:020000040000FA
:06000000B7EF5FF01200F3
:0600080004EF08F01200F5
:060018000CEF08F01200DD
:06100000B7EF5FF01200E3
:021006001200D6
:0610080087EF5AF0120010
:02100E001200CE
:02101000FEFFE1
:0410120000000000DA
:021016000000D8
:0610180074EF5AF0120013
:02101E000C00C4
:10102000161000003D0F0000020000005DC000002F
:10103000B60400004A0000005AC00000FB01000096
:101040000300000041C00000800200001900000001
:101050003BC00000D20200000600000034C00000C7
:10106000C5020000070000002EC00000CC020000F6
:10107000060000001BC00000280F00001300000045
:101080000AC00000990200001100000003C0000027
:10109000BE0200000700000012100000FB0000006C
:1010A00004000000101000003B0F000002000000D0
:1010B000D9CFE6FFE1CFD9FF0D0EE126040EDB6AA2
:1010C000200EF36E040EDBCFF4FFF350F45C13E25A
:1010D000040EDB50E76EFD0EDBCFE9FFFE0EDBCF2B
:1010E000EAFFE750E926000EEA22EF5001E103D0C3
:1010F000040EDB2AE5D7040EDB5004E1F368F46844
:10110000A5EF15F0200EF36E040EDBCFF4FFF350C5
:10111000F45C11E3200EE76EFD0EDBCFE9FFFE0E5F
:10112000DBCFEAFFE750E926000EEA22EF6AF36818
:10113000F468A5EF15F0050EDB6AFD0EDBCFE9FFC5
:10114000FE0EDBCFEAFFEF50400802E099EF15F00A
:10115000040EDB04E76EFD0EDBCFE9FFFE0EDBCFF6
:10116000EAFFE750E926000EEA22EF503F0802E0CE
:1011700099EF15F0010EE76EFD0EDBCFE9FFFE0ED5
:10118000DBCFEAFFE750E926000EEA22EF505308D2
:1011900001E07ED0020EE76EFD0EDBCFE9FFFE0E12
:1011A000DBCFEAFFE750E926000EEA22EF505408B1
:1011B0006FE1FAC100F0016A00BE016800C0E6FFFD
:1011C00001C0E6FF28CFE6FF29CFE6FF06C1E6FF14
:1011D00007C1E6FF04C1E6FF05C1E6FF02C1E6FF65
:1011E00003C1E6FF56C1E6FF57C1E6FF30C1E6FF87
:1011F00031C1E6FF0AC1E6FF0BC1E6FF54C1E6FFBD
:1012000055C1E6FF2EC1E6FF2FC1E6FF08C1E6FF8C
:1012100009C1E6FF8250020B01E0010EE66EE66AAC
:101220008250010BE66EE66AA0C202F0036A02BEBB
:10123000036802C0E6FF03C0E6FF9FC204F0056A30
:1012400004BE056804C0E6FF05C0E6FF9EC206F0C6
:10125000076A06BE076806C0E6FF07C0E6FF660E1F
:10126000E66EA40EE66E000EE66EFB0EDBCFE6FF2A
:10127000FC0EDBCFE6FFD0EC5CF0086E250EE15EE5
:101280000850010EF36E050EF3CFDBFF98EF15F05B
:10129000010EE76EFD0EDBCFE9FFFE0EDBCFEAFFAE
:1012A000E750E926000EEA22EF50540844E1020E0E
:1012B000E76EFD0EDBCFE9FFFE0EDBCFEAFFE75066
:1012C000E926000EEA22EF50440835E1EEC0E6FFC1
:1012D000EFC0E6FFECC0E6FFEDC0E6FFEAC0E6FFC8
:1012E000EBC0E6FFE8C0E6FFE9C0E6FFE6C0E6FFC8
:1012F000E7C0E6FFE4C0E6FFE5C0E6FFE2C0E6FFC8
:10130000E3C0E6FF490EE66EA40EE66E000EE66E42
:10131000FB0EDBCFE6FFFC0EDBCFE6FFD0EC5CF094
:10132000006E130EE15E0050010EF36E050EF3CF5A
:10133000DBFF98EF15F0010EE76EFD0EDBCFE9FF46
:10134000FE0EDBCFEAFFE750E926000EEA22EF505F
:10135000430802E0AAEF0DF0020EE76EFD0EDBCFB0
:10136000E9FFFE0EDBCFEAFFE750E926000EEA2296
:10137000EF504E0801E0EED3080EF36E040EDBCF03
:10138000F4FFF350F45C01E2E5D3030EE76EFD0ECB
:10139000DBCFE9FFFE0EDBCFEAFFE750E926000EC8
:1013A000EA22EF50200801E0D5D3050EE76EFD0ECE
:1013B000DBCFE9FFFE0EDBCFEAFFE750E926000EA8
:1013C000EA22EF503A0801E0C5D3FD0EDBCFE6FF7D
:1013D000FE0EDBCFE6FFFB0EDBCFE6FFFC0EDBCF26
:1013E000E6FFFEEC59F0E552E552E552E552010EFA
:1013F000F36E050EF3CFDBFF0201805103E1050E12
:10140000DB68A6D3040EE76EFD0EDBCFE9FFFE0E10
:10141000DBCFEAFFE750E926000EEA22EF506C0826
:1014200027E1060EE76EFD0EDBCFE9FFFE0EDBCFF8
:10143000EAFFE750E926000EEA22EF50300803E108
:1014400018EC3EF014D0060EE76EFD0EDBCFE9FF80
:10145000FE0EDBCFEAFFE750E926000EEA22EF504E
:10146000310803E116EC3EF002D0050EDB6870D3C4
:10147000040EE76EFD0EDBCFE9FFFE0EDBCFEAFFC9
:10148000E750E926000EEA22EF50680827E1060E31
:10149000E76EFD0EDBCFE9FFFE0EDBCFEAFFE75084
:1014A000E926000EEA22EF50300803E1FAEC3DF0A5
:1014B00014D0060EE76EFD0EDBCFE9FFFE0EDBCF8C
:1014C000EAFFE750E926000EEA22EF50310803E177
:1014D000C8EC3DF002D0050EDB683AD3040EE76E8F
:1014E000FD0EDBCFE9FFFE0EDBCFEAFFE750E9267A
:1014F000000EEA22EF50730801E058D1040EDB50D1
:101500000F0801E053D1080EE76EFD0EDBCFE9FFB7
:10151000FE0EDBCFEAFFE750E926000EEA22EF508D
:101520002C0801E043D10B0EE76EFD0EDBCFE9FF87
:10153000FE0EDBCFEAFFE750E926000EEA22EF506D
:101540002C0801E033D1060EE76EFD0EDBCF00F074
:10155000FE0EDBCF01F0E7500026000E012200C096
:10156000E6FF01C0E6FF6AEC58F0E552E552070ECF
:10157000F3CFDBFF080EF4CFDBFFD950070FE96E86
:10158000DACFEAFFEE50ED1003E1050EDB6841D043
:10159000070EDBCF00F0080EDBCF01F00101085190
:1015A000001802E10951011834E0070EDBCF00F00A
:1015B000080EDBCF01F0013404E200503C08000EBD
:1015C000015407E23C0EF36E070EF3CFDBFF080E6B
:1015D000DB6A070EDBCF00F0080EDBCF01F0D890FE
:1015E000015004E6190E005C000E015807E2190EC6
:1015F000F36E070EF3CFDBFF080EDB6A070EDBCFBF
:1016000008F1080EDBCF09F10201A16BA26B01EC1E
:101610002FF0090EE76EFD0EDBCF00F0FE0EDBCFE4
:1016200001F0E7500026000E012200C0E6FF01C0D5
:10163000E6FF6AEC58F0E552E552070EF3CFDBFF08
:10164000080EF4CFDBFFD950070FE96EDACFEAFFBF
:10165000EE50ED1003E1050EDB6841D0070EDBCF45
:1016600000F0080EDBCF01F001012E51001802E15D
:101670002F51011834E0070EDBCF00F0080EDBCF4E
:1016800001F0013404E200504108000E015407E269
:10169000410EF36E070EF3CFDBFF080EDB6A070E79
:1016A000DBCF00F0080EDBCF01F0D890015004E64C
:1016B000190E005C000E015807E2190EF36E070EBA
:1016C000F3CFDBFF080EDB6A070EDBCF2EF1080E2F
:1016D000DBCF2FF10201A36BA46B01EC2FF00C0EFA
:1016E000E76EFD0EDBCF00F0FE0EDBCF01F0E75022
:1016F0000026000E012200C0E6FF01C0E6FF6AECF2
:1017000058F0E552E552070EF3CFDBFF080EF4CF99
:10171000DBFFD950070FE96EDACFEAFFEE50ED108C
:1017200003E1050EDB6841D0070EDBCF00F0080EA9
:10173000DBCF01F001015451001802E155510118AD
:1017400034E0070EDBCF00F0080EDBCF01F00134F0
:1017500004E200504108000E015407E2410EF36E0E
:10176000070EF3CFDBFF080EDB6A070EDBCF00F0BE
:10177000080EDBCF01F0D890015004E6190E005C92
:10178000000E015807E2190EF36E070EF3CFDBFFD0
:10179000080EDB6A070EDBCF54F1080EDBCF55F1E4
:1017A0000201A56BA66B01EC2FF0D2D1040EE76EFF
:1017B000FD0EDBCFE9FFFE0EDBCFEAFFE750E926A7
:1017C000000EEA22EF50640801E03DD1040EDB5028
:1017D0000F0801E038D1080EE76EFD0EDBCFE9FF00
:1017E000FE0EDBCFEAFFE750E926000EEA22EF50BB
:1017F0002C0801E028D10B0EE76EFD0EDBCFE9FFD0
:10180000FE0EDBCFEAFFE750E926000EEA22EF509A
:101810002C0801E018D1060EE76EFD0EDBCF00F0BC
:10182000FE0EDBCF01F0E7500026000E012200C0C3
:10183000E6FF01C0E6FF6AEC58F0E552E552070EFC
:10184000F3CFDBFF080EF4CFDBFFD950070FE96EB3
:10185000DACFEAFFEE50ED1003E1050EDB6829D088
:10186000070EDBCF00F0080EDBCF01F0013404E2FD
:1018700000503C08000E015407E23C0EF36E070EC8
:10188000F3CFDBFF080EDB6A070EDBCF00F0080E9C
:10189000DBCF01F0D890015004E6190E005C000E79
:1018A000015807E2190EF36E070EF3CFDBFF080EA7
:1018B000DB6A090EE76EFD0EDBCF00F0FE0EDBCF1C
:1018C00001F0E7500026000E012200C0E6FF01C033
:1018D000E6FF6AEC58F0E552E552090EF3CFDBFF64
:1018E0000A0EF4CFDBFFD950090FE96EDACFEAFF19
:1018F000EE50ED1003E1050EDB6829D0090EDBCFB9
:1019000000F00A0EDBCF01F0013404E20050410880
:10191000000E015407E2410EF36E070EF3CFDBFF1A
:10192000080EDB6A090EDBCF00F00A0EDBCF01F0F8
:10193000D890015004E6190E005C000E015807E231
:10194000190EF36E070EF3CFDBFF080EDB6A0C0EE9
:10195000E76EFD0EDBCF00F0FE0EDBCF01F0E750AF
:101960000026000E012200C0E6FF01C0E6FF6AEC7F
:1019700058F0E552E5520B0EF3CFDBFF0C0EF4CF1F
:10198000DBFFD9500B0FE96EDACFEAFFEE50ED1016
:1019900003E1050EDB6829D00B0EDBCF00F00C0E47
:1019A000DBCF01F0013404E200504108000E015485
:1019B00007E2410EF36E070EF3CFDBFF080EDB6A82
:1019C0000B0EDBCF00F00C0EDBCF01F0D8900150F6
:1019D00004E6190E005C000E015807E2190EF36EC2
:1019E000070EF3CFDBFF080EDB6A050EDB042AE1EE
:1019F0000B0EDBCFE6FF0C0EDBCFE6FF090EDBCFD5
:101A0000E6FF0A0EDBCFE6FF070EDBCFE6FF080E90
:101A1000DBCFE6FFF4EC27F0006E060EE15E00502F
:101A2000070EDBCF02F1080EDBCF03F1090EDBCF8F
:101A300004F10A0EDBCF05F10B0EDBCF06F10C0E25
:101A4000DBCF07F185D0040EE76EFD0EDBCFE9FF9B
:101A5000FE0EDBCFEAFFE750E926000EEA22EF5048
:101A6000690821E1060EE76EFD0EDBCF00F0FE0EE9
:101A7000DBCF01F0E7500026000E012200C0E6FF98
:101A800001C0E6FF6AEC58F0E552E552F3CF28FFBB
:101A9000F4CF29FF28CFE6FF29CFE6FFBEEC28F0E0
:101AA000E552E55255D0040EE76EFD0EDBCFE9FF9F
:101AB000FE0EDBCFEAFFE750E926000EEA22EF50E8
:101AC000610842E1060EE76EFD0EDBCFE9FFFE0E78
:101AD000DBCFEAFFE750E926000EEA22EF5030089C
:101AE00010E10101FA6BFAC100F0016A00BE016861
:101AF00000C0E6FF01C0E6FF4CEC2AF0E552E552DB
:101B000022D0060EE76EFD0EDBCFE9FFFE0EDBCF27
:101B1000EAFFE750E926000EEA22EF50310811E112
:101B20000101010EFA6FFAC100F0016A00BE0168FE
:101B300000C0E6FF01C0E6FF4CEC2AF0E552E5529A
:101B400002D0050EDB6804D00000050EDB68000043
:101B500098EF15F0010EE76EFD0EDBCFE9FFFE0EEC
:101B6000DBCFEAFFE750E926000EEA22EF504908F2
:101B700001E09CD0020EE76EFD0EDBCFE9FFFE0E0A
:101B8000DBCFEAFFE750E926000EEA22EF504408D7
:101B900001E08CD0450EE66EA40EE66E000EE66EF9
:101BA000FB0EDBCFE6FFFC0EDBCFE6FF1FEC5AF0AF
:101BB000006E050EE15E0050D5C2E6FFD6C2E6FF1C
:101BC000D7C2E6FFFB0EDBCFE6FFFC0EDBCFE6FF66
:101BD000E2EC59F0006E050EE15E0050430EE66E39
:101BE000A40EE66E000EE66EFB0EDBCFE6FFFC0EEB
:101BF000DBCFE6FFE2EC59F0006E050EE15E00502F
:101C00004CEC28F0F3CF00F0F4CF01F000C0E6FF79
:101C100001C0E6FFFB0EDBCFE6FFFC0EDBCFE6FFED
:101C2000BEEC59F0E552E552E552E552430EE66E40
:101C3000A40EE66E000EE66EFB0EDBCFE6FFFC0E9A
:101C4000DBCFE6FFE2EC59F0006E050EE15E0050DE
:101C5000D2C2E6FFD3C2E6FFD4C2E6FFFB0EDBCF63
:101C6000E6FFFC0EDBCFE6FFE2EC59F0006E050E5E
:101C7000E15E00500201805112E0400EE66EA40EBB
:101C8000E66E000EE66EFB0EDBCFE6FFFC0EDBCF52
:101C9000E6FFE2EC59F0006E050EE15E0050010E29
:101CA000F36E050EF3CFDBFF98EF15F0010EE76E34
:101CB000FD0EDBCFE9FFFE0EDBCFEAFFE750E926A2
:101CC000000EEA22EF50520801E0CFD0020EE76E7C
:101CD000FD0EDBCFE9FFFE0EDBCFEAFFE750E92682
:101CE000000EEA22EF504D0801E0BFD0400EF36E27
:101CF000050EF3CFDBFF040EE76EFD0EDBCF00F029
:101D0000FE0EDBCF01F0E7500026000E012200C0DE
:101D1000E6FF01C0E6FF6AEC58F0E552E552090E15
:101D2000F3CFDBFF0A0EF4CFDBFF060EE76EFD0EEE
:101D3000DBCF00F0FE0EDBCF01F0E7500026000EF7
:101D4000012200C0E6FF01C0E6FF6AEC58F0E55250
:101D5000E552070EF3CFDBFF080EF4CFDBFFD950BF
:101D6000090FE96EDACFEAFFEE50ED1010E1070E31
:101D7000DBCFE6FF080EDBCFE6FF000EE66E020EBD
:101D8000E66EC4EC4DF0E552E552E552E552090E1F
:101D9000DBCF00F00A0EDBCF01F00001800E011452
:101DA0004EE1090EDBCF02F00A0EDBCF03F0D89034
:101DB000035004E6040E025C000E035840E2200EBD
:101DC000E66EE66A090EDBCF00F00A0EDBCF01F00B
:101DD000050ED89000360136E806FBE1000E00261D
:101DE000020E012200C0E6FF01C0E6FF200EE76EF2
:101DF000FB0EDBCF02F0FC0EDBCF03F0E750022638
:101E0000000E032202C0E6FF03C0E6FF79EC59F0A2
:101E1000046E060EE15E0450FD0EDBCFE6FFFE0E03
:101E2000DBCFE6FFFB0EDBCFE6FFFC0EDBCFE6FFF2
:101E3000FEEC59F0E552E552E552E55214D0050E9C
:101E4000DB683A0EE66EA40EE66E000EE66EFB0E42
:101E5000DBCFE6FFFC0EDBCFE6FF1FEC5AF0006E97
:101E6000050EE15E005098EF15F0010EE76EFD0ED5
:101E7000DBCFE9FFFE0EDBCFEAFFE750E926000EDD
:101E8000EA22EF50570801E0BFD0020EE76EFD0EC8
:101E9000DBCFE9FFFE0EDBCFEAFFE750E926000EBD
:101EA000EA22EF504D0801E0AFD0400EF36E050E70
:101EB000F3CFDBFF040EE76EFD0EDBCF00F0FE0E6E
:101EC000DBCF01F0E7500026000E012200C0E6FF44
:101ED00001C0E6FF6AEC58F0E552E552090EF3CF77
:101EE000DBFF0A0EF4CFDBFF060EE76EFD0EDBCF45
:101EF00000F0FE0EDBCF01F0E7500026000E0122BD
:101F000000C0E6FF01C0E6FF6AEC58F0E552E5527A
:101F1000070EF3CFDBFF080EF4CFDBFF090EDBCF9C
:101F200000F00A0EDBCF01F00001800E011468E121
:101F3000090EDBCF02F00A0EDBCF03F0D89003507E
:101F400004E6040E025C000E03585AE2200EE66E10
:101F5000E66A200EE76EFD0EDBCF00F0FE0EDBCF53
:101F600001F0E7500026000E012200C0E6FF01C08C
:101F7000E6FF090EDBCF02F00A0EDBCF03F0050E01
:101F8000D89002360336E806FBE1000E0226020E68
:101F9000032202C0E6FF03C0E6FF79EC59F0046EAD
:101FA000060EE15E0450D950090FE96EDACFEAFF60
:101FB000030EEE1801E1ED5010E1070EDBCFE6FF56
:101FC000080EDBCFE6FF000EE66E020EE66E84EC36
:101FD0004BF0E552E552E552E552FD0EDBCFE6FF50
:101FE000FE0EDBCFE6FFFB0EDBCFE6FFFC0EDBCF0A
:101FF000E6FFFEEC59F0E552E552E552E55202D01B
:10200000050EDB6898EF15F0010EE76EFD0EDBCFD5
:10201000E9FFFE0EDBCFEAFFE750E926000EEA22D9
:10202000EF5045082AE1020EE76EFD0EDBCFE9FF17
:10203000FE0EDBCFEAFFE750E926000EEA22EF5062
:1020400043081BE17EEC46F0FD0EDBCFE6FFFE0E03
:10205000DBCFE6FFFB0EDBCFE6FFFC0EDBCFE6FFC0
:10206000FEEC59F0E552E552E552E552010EF36EF1
:10207000050EF3CFDBFF98EF15F0010EE76EFD0EB6
:10208000DBCFE9FFFE0EDBCFEAFFE750E926000ECB
:10209000EA22EF5045082AE1020EE76EFD0EDBCF83
:1020A000E9FFFE0EDBCFEAFFE750E926000EEA2249
:1020B000EF5050081BE119EC47F0FD0EDBCFE6FFB7
:1020C000FE0EDBCFE6FFFB0EDBCFE6FFFC0EDBCF29
:1020D000E6FFFEEC59F0E552E552E552E552010EFD
:1020E000F36E050EF3CFDBFF98EF15F0010EE76EF0
:1020F000FD0EDBCFE9FFFE0EDBCFEAFFE750E9265E
:10210000000EEA22EF5045082AE1020EE76EFD0EAE
:10211000DBCFE9FFFE0EDBCFEAFFE750E926000E3A
:10212000EA22EF5051081BE1BEEC47F0FD0EDBCF79
:10213000E6FFFE0EDBCFE6FFFB0EDBCFE6FFFC0E7D
:10214000DBCFE6FFFEEC59F0E552E552E552E552F1
:10215000010EF36E050EF3CFDBFF98EF15F0010EC5
:10216000E76EFD0EDBCFE9FFFE0EDBCFEAFFE750A7
:10217000E926000EEA22EF50540801E05FD1020E7A
:10218000E76EFD0EDBCFE9FFFE0EDBCFEAFFE75087
:10219000E926000EEA22EF50530801E04FD1FD0E70
:1021A000DBCFE6FFFE0EDBCFE6FF38EC5AF0E55260
:1021B000E552F3CF00F0F4CF01F0120E001801E168
:1021C000015001E03AD1020EDB6A030EE76EFD0E0C
:1021D000DBCFE9FFFE0EDBCFEAFFE750E926000E7A
:1021E000EA22EFCFDFFF040EE76EFD0EDBCFE9FF43
:1021F000FE0EDBCFEAFFE750E926000EEA22010ED1
:10220000EFCFDBFFD9CFE6FFDACFE6FF6AEC58F07D
:10221000E552E552F3CFE2F0F4CFE3F0050EE76EBE
:10222000FD0EDBCFE9FFFE0EDBCFEAFFE750E9262C
:10223000000EEA22EFCFDFFF060EE76EFD0EDBCFCA
:10224000E9FFFE0EDBCFEAFFE750E926000EEA22A7
:10225000010EEFCFDBFFD9CFE6FFDACFE6FF6AEC66
:1022600058F0E552E552F3CFE4F0F4CFE5F0070E75
:10227000E76EFD0EDBCFE9FFFE0EDBCFEAFFE75096
:10228000E926000EEA22EFCFDFFF080EE76EFD0E13
:10229000DBCFE9FFFE0EDBCFEAFFE750E926000EB9
:1022A000EA22010EEFCFDBFFD9CFE6FFDACFE6FF60
:1022B0006AEC58F0E552E552F3CFE6F0F4CFE7F0E0
:1022C000090EE76EFD0EDBCFE9FFFE0EDBCFEAFF66
:1022D000E750E926000EEA22EFCFDFFF0A0EE76E95
:1022E000FD0EDBCFE9FFFE0EDBCFEAFFE750E9266C
:1022F000000EEA22010EEFCFDBFFD9CFE6FFDACFE7
:10230000E6FF6AEC58F0E552E552F3CFE8F0F4CF7F
:10231000E9F00B0EE76EFD0EDBCFE9FFFE0EDBCF23
:10232000EAFFE750E926000EEA22EFCFDFFF0C0EAE
:10233000E76EFD0EDBCFE9FFFE0EDBCFEAFFE750D5
:10234000E926000EEA22010EEFCFDBFFD9CFE6FF30
:10235000DACFE6FF6AEC58F0E552E552F3CFEAF047
:10236000F4CFEBF00D0EE76EFD0EDBCFE9FFFE0EB6
:10237000DBCFEAFFE750E926000EEA22EFCFDFFFCE
:102380000E0EE76EFD0EDBCFE9FFFE0EDBCFEAFFA0
:10239000E750E926000EEA22010EEFCFDBFFD9CF8E
:1023A000E6FFDACFE6FF6AEC58F0E552E552F3CFEC
:1023B000ECF0F4CFEDF00F0EE76EFD0EDBCFE9FF92
:1023C000FE0EDBCFEAFFE750E926000EEA22EFCF50
:1023D000DFFF100EE76EFD0EDBCFE9FFFE0EDBCF59
:1023E000EAFFE750E926000EEA22010EEFCFDBFFFD
:1023F000D9CFE6FFDACFE6FF6AEC58F0E552E552B6
:10240000F3CFEEF0F4CFEFF095EC41F0FD0EDBCF23
:10241000E6FFFE0EDBCFE6FFFB0EDBCFE6FFFC0E9A
:10242000DBCFE6FFFEEC59F0E552E552E552E5520E
:10243000010EF36E050EF3CFDBFF7AD3010EE76ECC
:10244000FD0EDBCFE9FFFE0EDBCFEAFFE750E9260A
:10245000000EEA22EF5043082AE1020EE76EFD0E5D
:10246000DBCFE9FFFE0EDBCFEAFFE750E926000EE7
:10247000EA22EF504D081BE10201010EC36FFD0E71
:10248000DBCFE6FFFE0EDBCFE6FFFB0EDBCFE6FF8A
:10249000FC0EDBCFE6FFFEEC59F0E552E552E552CB
:1024A000E552010EF36E050EF3CFDBFF41D3010EB3
:1024B000E76EFD0EDBCFE9FFFE0EDBCFEAFFE75054
:1024C000E926000EEA22EF50430829E1020EE76EEA
:1024D000FD0EDBCFE9FFFE0EDBCFEAFFE750E9267A
:1024E000000EEA22EF5045081AE10201C36BFD0E0F
:1024F000DBCFE6FFFE0EDBCFE6FFFB0EDBCFE6FF1A
:10250000FC0EDBCFE6FFFEEC59F0E552E552E5525A
:10251000E552010EF36E050EF3CFDBFF09D3010E7A
:10252000E76EFD0EDBCFE9FFFE0EDBCFEAFFE750E3
:10253000E926000EEA22EF50520873E1020EE76E20
:10254000FD0EDBCFE9FFFE0EDBCFEAFFE750E92609
:10255000000EEA22EF50460864E1FD0EDBCFE6FFF5
:10256000FE0EDBCFE6FFFB0EDBCFE6FFFC0EDBCF84
:10257000E6FFFEEC59F0E552E552E552E552FD0E5C
:10258000DBCFE6FFFE0EDBCFE6FF38EC5AF0E5527C
:10259000E552F3CF00F0F4CF01F0060E001801E190
:1025A00001502AE1040EE76EFD0EDBCF00F0FE0EB7
:1025B000DBCF01F0E7500026000E012200C0E6FF4D
:1025C00001C0E6FF6AEC58F0E552E552070EF3CF82
:1025D000DBFF080EF4CFDBFFD950070FE96EDACF2F
:1025E000EAFFEE50ED1002E1A9EC2FF0010EF36EC0
:1025F000050EF3CFDBFF14D0330EE66EA40EE66EAD
:10260000000EE66EFB0EDBCFE6FFFC0EDBCFE6FF37
:10261000E2EC59F0006E050EE15E0050050EDB683D
:1026200087D2010EE76EFD0EDBCFE9FFFE0EDBCF9A
:10263000EAFFE750E926000EEA22EF504C0801E0DD
:1026400058D1020EE76EFD0EDBCFE9FFFE0EDBCFA9
:10265000EAFFE750E926000EEA22EF50470801E0C2
:1026600048D1040EE76EFD0EDBCFE9FFFE0EDBCF97
:10267000EAFFE750E926000EEA22EF50470801E0A2
:1026800035D1050EE76EFD0EDBCFE9FFFE0EDBCF89
:10269000EAFFE750E926000EEA22EF504E0801E07B
:1026A00025D1070EE76EFD0EDBCFE9FFFE0EDBCF77
:1026B000EAFFE750E926000EEA22EF50D00FE76E5E
:1026C000060EE7CFDBFFFD0EDBCFE6FFFE0EDBCF16
:1026D000E6FFFB0EDBCFE6FFFC0EDBCFE6FFFEECFA
:1026E00059F0E552E552E552E552010EF36E050E42
:1026F000F3CFDBFF060EDB044DE1240EE76EFD0E8B
:10270000DBCFE9FFFE0EDBCFEAFFE750E926000E44
:10271000EA22EF50E66E230EE76EFD0EDBCFE9FFF7
:10272000FE0EDBCFEAFFE750E926000EEA22EF506B
:10273000E66E220EE76EFD0EDBCFE9FFFE0EDBCF6D
:10274000EAFFE750E926000EEA22EF50E66E210E7E
:10275000E76EFD0EDBCFE9FFFE0EDBCFEAFFE750B1
:10276000E926000EEA22EF50E66E200EE76EFD0E1F
:10277000DBCFE9FFFE0EDBCFEAFFE750E926000ED4
:10278000EA22EF50E66E5BEC47F0006E050EE15E6C
:102790000050ABD0060EDB5002084DE1240EE76E70
:1027A000FD0EDBCFE9FFFE0EDBCFEAFFE750E926A7
:1027B000000EEA22EF50E66E230EE76EFD0EDBCF31
:1027C000E9FFFE0EDBCFEAFFE750E926000EEA2222
:1027D000EF50E66E220EE76EFD0EDBCFE9FFFE0E38
:1027E000DBCFEAFFE750E926000EEA22EF50E66E63
:1027F000210EE76EFD0EDBCFE9FFFE0EDBCFEAFF19
:10280000E750E926000EEA22EF50E66E200EE76E52
:10281000FD0EDBCFE9FFFE0EDBCFEAFFE750E92636
:10282000000EEA22EF50E66EC0EC46F0006E050E98
:10283000E15E00505AD0060EDB5003084DE1240E35
:10284000E76EFD0EDBCFE9FFFE0EDBCFEAFFE750C0
:10285000E926000EEA22EF50E66E230EE76EFD0E2B
:10286000DBCFE9FFFE0EDBCFEAFFE750E926000EE3
:10287000EA22EF50E66E220EE76EFD0EDBCFE9FF97
:10288000FE0EDBCFEAFFE750E926000EEA22EF500A
:10289000E66E210EE76EFD0EDBCFE9FFFE0EDBCF0D
:1028A000EAFFE750E926000EEA22EF50E66E200E1E
:1028B000E76EFD0EDBCFE9FFFE0EDBCFEAFFE75050
:1028C000E926000EEA22EF50E66E1DEC46F0006E9F
:1028D000050EE15E005009D0FB0EDBCFE9FFFC0ED8
:1028E000DBCFEAFFEF6A050EDB6802D0050EDB687E
:1028F0001FD1010EE76EFD0EDBCFE9FFFE0EDBCF31
:10290000EAFFE750E926000EEA22EF50450801E011
:10291000AFD0020EE76EFD0EDBCFE9FFFE0EDBCF80
:10292000EAFFE750E926000EEA22EF50520801E0E4
:102930009FD0FD0EDBCFE6FFFE0EDBCFE6FFFB0EEA
:10294000DBCFE6FFFC0EDBCFE6FFFEEC59F0E552F5
:10295000E552E552E552010EF36E050EF3CFDBFFB3
:10296000040EE76EFD0EDBCFE9FFFE0EDBCFEAFFC4
:10297000E750E926000EEA22EF50530821E1050E48
:10298000E76EFD0EDBCFE9FFFE0EDBCFEAFFE7507F
:10299000E926000EEA22EF50540812E1070EE76E16
:1029A000FD0EDBCFE9FFFE0EDBCFEAFFE750E926A5
:1029B000000EEA22EF50E66E48EC57F0E55257D091
:1029C000040EE76EFD0EDBCFE9FFFE0EDBCFEAFF64
:1029D000E750E926000EEA22EF5047081EE1050EF7
:1029E000E76EFD0EDBCFE9FFFE0EDBCFEAFFE7501F
:1029F000E926000EEA22EF5054080FE1200EE76EA0
:102A0000FB0EDBCFE9FFFC0EDBCFEAFFE750E92648
:102A1000000EEA22FDC1EFFF2AD0040EE76EFD0E84
:102A2000DBCFE9FFFE0EDBCFEAFFE750E926000E21
:102A3000EA22EF50430812E1050EE76EFD0EDBCFF0
:102A4000E9FFFE0EDBCFEAFFE750E926000EEA229F
:102A5000EF504C0803E134EC58F009D0FB0EDBCF0B
:102A6000E9FFFC0EDBCFEAFFEF6A050EDB6860D002
:102A7000010EE76EFD0EDBCFE9FFFE0EDBCFEAFFB6
:102A8000E750E926000EEA22EF5052083AE1020E22
:102A9000E76EFD0EDBCFE9FFFE0EDBCFEAFFE7506E
:102AA000E926000EEA22EF5053082BE1040EDB501A
:102AB000060827E1040EE76EFD0EDBCFE9FFFE0EF0
:102AC000DBCFEAFFE750E926000EEA22EF5030089C
:102AD00003E1F29EFF0014D0040EE76EFD0EDBCF83
:102AE000E9FFFE0EDBCFEAFFE750E926000EEA22FF
:102AF000EF50310805E10000F29E0EEF00F00000FB
:102B000017D0230EE66EA40EE66E000EE66EFB0EE8
:102B1000DBCFE6FFFC0EDBCFE6FF1FEC5AF0006ECA
:102B2000050EE15E0050010EF36E050EF3CFDBFFE4
:102B300003D0F368F46809D0050EDB50006E016A1B
:102B400000C0F3FF01C0F4FF00D00D0EE15C02E213
:102B5000E16AE552E16EE552E7CFD9FF1200D9CF25
:102B6000E6FFE1CFD9FF0D0EE126FC0EDBCFE9FF3A
:102B7000FD0EDBCFEAFF010EEECFDBFF020EEECF44
:102B8000DBFF030EEECFDBFF040EEECFDBFFE76EC5
:102B9000FC0EDBCFE9FFFD0EDBCFEAFFE750E926B5
:102BA000000EEA22050EEECFDBFF060EEECFDBFFB6
:102BB000070EEECFDBFF080EEECFDBFF090EDB6A60
:102BC0000A0EDB6A0B0EDB6A0C0EDB6ADF6AFE0E96
:102BD000DB50DF5C01E338D1050EDBCF04F0060EDD
:102BE000DBCF05F0070EDBCF06F0080EDBCF07F0DA
:102BF000040E1F0B07E0D89004360536063607365C
:102C0000E806F9E1050EDBCF08F0060EDBCF09F090
:102C1000070EDBCF0AF0080EDBCF0BF0050ED890C5
:102C20000B320A3209320832E806F9E10850041A78
:102C30000950051A0A50061A0B50071AD950050FE9
:102C4000E96EDACFEAFF0450EE24006E0550EE2064
:102C5000016E0650EE20026E0750EE20036E030E4A
:102C6000106E116A126A136AD950090FE96EDACF31
:102C7000EAFFEE501016EE501116EE501216EE50FE
:102C8000131610C0E9FF11C0EAFFD890E936EA3602
:102C9000D890E936EA36850EE926020EEA22EECF12
:102CA0000CF0EECF0DF0EECF0EF0EFCF0FF0D950CD
:102CB000090FE96EDACFEAFFEE500C26EE500D2236
:102CC000EE500E22EE500F220C50001A0D50011A39
:102CD0000E50021A0F50031AD950010FE96EDACFC5
:102CE000EAFF0050EE260150EE220250EE22035081
:102CF000EE22D950090FE96EDACFEAFF02019551B1
:102D0000EE269651EE229751EE229851EE22010EB8
:102D1000DBCF04F0020EDBCF05F0030EDBCF06F0B5
:102D2000040EDBCF07F01F0B07E0D8900436053602
:102D300006360736E806F9E1010EDBCF08F0020E91
:102D4000DBCF09F0030EDBCF0AF0040EDBCF0BF074
:102D5000050ED8900B320A3209320832E806F9E142
:102D60000850041A0950051A0A50061A0B50071A7F
:102D7000D950010FE96EDACFEAFF0450EE24006E5D
:102D80000550EE20016E0650EE20026E0750EE2038
:102D9000036E090EDBCF10F00A0EDBCF11F00B0E25
:102DA000DBCF12F00C0EDBCF13F00B0ED8901332EA
:102DB000123211321032E806F9E1030E146E156A70
:102DC000166A176A1450101615501116165012165E
:102DD0001750131610C0E9FF11C0EAFFD890E9366A
:102DE000EA36D890E936EA36850EE926020EEA225E
:102DF000EECF0CF0EECF0DF0EECF0EF0EFCF0FF0E8
:102E0000D950090FE96EDACFEAFFEE500C26EE50EA
:102E10000D22EE500E22EE500F220C50001A0D50D3
:102E2000011A0E50021A0F50031AD950050FE96EFD
:102E3000DACFEAFF0050EE260150EE220250EE22D9
:102E40000350EE22DF2AC3D6FC0EDBCFE9FFFD0ED6
:102E5000DBCFEAFF010EDBCFEEFF020EDBCFEEFF92
:102E6000030EDBCFEEFF040EDBCFEEFFE76EFC0EB2
:102E7000DBCFE9FFFD0EDBCFEAFFE750E926000ECE
:102E8000EA22050EDBCFEEFF060EDBCFEEFF070ECC
:102E9000DBCFEEFF080EDBCFEEFF0D0EE15C02E2B2
:102EA000E16AE552E16EE552E7CFD9FF1200D9CFD2
:102EB000E6FFE1CFD9FF0D0EE126FC0EDBCFE9FFE7
:102EC000FD0EDBCFEAFF010EEECFDBFF020EEECFF1
:102ED000DBFF030EEECFDBFF040EEECFDBFFE76E72
:102EE000FC0EDBCFE9FFFD0EDBCFEAFFE750E92662
:102EF000000EEA22050EEECFDBFF060EEECFDBFF63
:102F0000070EEECFDBFF080EEECFDBFFFE0EDBCFB2
:102F100000F0016A026A036A95C21EF096C21FF0B1
:102F200097C220F098C221F000C023F001C024F025
:102F300002C025F003C026F0C0EC5EF0090E1AC0F6
:102F4000DBFF0A0E1BC0DBFF0B0E1CC0DBFF0C0EF1
:102F50001DC0DBFFDF6AFE0EDB50DF5C01E338D112
:102F6000010EDBCF04F0020EDBCF05F0030EDBCF4A
:102F700006F0040EDBCF07F01F0B07E0D8900436F5
:102F8000053606360736E806F9E1010EDBCF08F014
:102F9000020EDBCF09F0030EDBCF0AF0040EDBCF0D
:102FA0000BF0050ED8900B320A3209320832E806CF
:102FB000F9E10850041A0950051A0A50061A0B5074
:102FC000071AD950010FE96EDACFEAFF0450EE2458
:102FD000006E0550EE20016E0650EE20026E075086
:102FE000EE20036E090EDBCF10F00A0EDBCF11F0DE
:102FF0000B0EDBCF12F00C0EDBCF13F00B0ED890C4
:103000001332123211321032E806F9E1030E146E57
:10301000156A166A176A14501016155011161650B4
:1030200012161750131610C0E9FF11C0EAFFD8900E
:10303000E936EA36D890E936EA36850EE926020EF8
:10304000EA22EECF0CF0EECF0DF0EECF0EF0EFCF88
:103050000FF0D950090FE96EDACFEAFFEE500C26D7
:10306000EE500D22EE500E22EE500F220C50001AA0
:103070000D50011A0E50021A0F50031AD950050FA5
:10308000E96EDACFEAFF0050EE5E0150EE5A0250D0
:10309000EE5A0350EE5AD950090FE96EDACFEAFF23
:1030A00002019551EE5E9651EE5A9751EE5A9851A3
:1030B000EE5A050EDBCF04F0060EDBCF05F0070E4F
:1030C000DBCF06F0080EDBCF07F0040E1F0B07E086
:1030D000D8900436053606360736E806F9E1050EBF
:1030E000DBCF08F0060EDBCF09F0070EDBCF0AF0CE
:1030F000080EDBCF0BF0050ED8900B320A320932E6
:103100000832E806F9E10850041A0950051A0A5075
:10311000061A0B50071AD950050FE96EDACFEAFFED
:103120000450EE24006E0550EE20016E0650EE2095
:10313000026E0750EE20036E030E106E116A126AC3
:10314000136AD950090FE96EDACFEAFFEE50101674
:10315000EE501116EE501216EE50131610C0E9FF85
:1031600011C0EAFFD890E936EA36D890E936EA3657
:10317000850EE926020EEA22EECF0CF0EECF0DF01E
:10318000EECF0EF0EFCF0FF0D950090FE96EDACF86
:10319000EAFFEE500C26EE500D22EE500E22EE50BD
:1031A0000F220C50001A0D50011A0E50021A0F5027
:1031B000031AD950010FE96EDACFEAFF0050EE5E34
:1031C0000150EE5A0250EE5A0350EE5ADF2AC3D68F
:1031D000FC0EDBCFE9FFFD0EDBCFEAFF010EDBCFFC
:1031E000EEFF020EDBCFEEFF030EDBCFEEFF040E91
:1031F000DBCFEEFFE76EFC0EDBCFE9FFFD0EDBCF92
:10320000EAFFE750E926000EEA22050EDBCFEEFFCB
:10321000060EDBCFEEFF070EDBCFEEFF080EDBCF97
:10322000EEFF0D0EE15C02E2E16AE552E16EE5526D
:06323000E7CFD9FF1200F8
:0A323600D9CFE6FFE1CFD9FFE65241
:10324000A098636A626A0F01160E5F6F9F0E5D6F32
:103250007B0E5C6F658C5E6B010EE66EE66AE66A5D
:103260004D0EE66E0F0EE66EA4EC59F0006E050EE4
:10327000E15E0050659CDF6ADF50006E016A080E57
:10328000005C000E015810E2DF50040DF3CFE9FF9F
:10329000F4CFEAFF000EE926040EEA22EE6AEE6A97
:1032A000EE6AEE6ADF2AE8D70F01160E4C6F62A6AF
:1032B00002D06296FCD70F01146B196B1A6B1B6B53
:1032C0006598DF6A020EDF5C18E2EA6ADF34FE0B03
:1032D000EA36E96E0B0EE9260F0EEA22EE6AED6A77
:1032E000EA6ADF34FE0BEA36E96E070EE9260F0EB6
:1032F000EA22EE6AED6ADF2AE5D70F01080E0B6FAE
:10330000040E0C6F016B006BE552E552E7CFD9FF5D
:103310001200D9CFE6FFE1CFD9FFE6520F01000539
:1033200009E165BA07D0626A0F015C815C890F010F
:10333000020E006F6250040B06E00F015C51040B9B
:1033400002E06294C2D865A202D0A1988CD06250EB
:10335000010B17E00F015C51010B13E06CDFD08E05
:10336000A288A088F28E0F01040E006F0401200EC7
:10337000026F040E036F080E016F006B8C0E0013BA
:1033800062906250100B06E00F015C51100B02E0DE
:1033900089D862986250400B14E00F015C51400BD9
:1033A00010E0010EE66EE66A000EE66EE66A730E47
:1033B000E66EE66AFDEC56F0006E060EE15E005029
:1033C000629C6250200B05E00F015C51200B01E074
:1033D0004FD86250020B14E00F015C51020B10E059
:1033E000010EE66EE66A000EE66EE66AE6687F0E9D
:1033F000E66EFDEC56F0006E060EE15E0050636A6C
:10340000040E0F01E76E0019E8AE02D0E73402D0D7
:10341000E750005D02E2A19826D00F015CA722D000
:10342000DF6A040EDF5C1EE262A61BD064CF22FFBF
:103430006296780E0F01221502E15DD810D0000EC1
:10344000E66EE66A220EE66E0F0EE66E720EE66E0F
:10345000E66AFDEC56F0006E060EE15E0050DF2AD3
:10346000E0D700D0A198E552E552E7CFD9FF12008E
:103470000F014CA115D003CFE9FF04CFEAFFEF50B5
:1034800080080DE10BCFE9FF0CCFEAFFEF50840875
:1034900006E103CFE9FF04CFEAFF8C0EEF6E4C91FB
:1034A000629A12000F015C8562986582000EE66EDA
:1034B000E66AE66EE66A750EE66EE66AFDEC56F0C2
:1034C000006E060EE15E00501200000EE66EE66A27
:1034D000E66EE66A740EE66EE66AFDEC56F0006E85
:1034E000060EE15E005065920F015C9562A402D069
:1034F0006294FCD71200D9CFE6FFE1CFD9FFE652A4
:10350000FD0E0F0122155AE17E0E2215E8407F0BB9
:10351000040DF3CF03FFF4CF04FF000E0327040EC6
:10352000042303CF05FF04CF06FF057503CFE9FF92
:1035300004CFEAFFEF503C0BE842E8420D083CE1C3
:1035400003CFE9FF04CFEAFF020EE926000EEA22CC
:10355000EECF00F0EFCF01F0280E001802E1040ECC
:10356000011828E103CFE9FF04CFEAFF020EE926A4
:10357000000EEA22200EEE6E040EED6EDF6ADF50C2
:10358000006E016A080E005C000E015813E2DF5065
:10359000EA6A280FE96E040EEA22EF50E66EDF5069
:1035A000EA6A200FE96E040EEA22E552E750EF6E58
:1035B000DF2AE5D70DD801D02ED805D0FD0E221573
:1035C000040801E14FD8E552E552E7CFD9FF1200D8
:1035D0000BCFE9FF0CCFEAFFEF50800B05E00BCFDC
:1035E000E9FF0CCFEAFFEF6A0F010F6B106B156B51
:1035F000166B146BBDD8000EE66EE66AE66EE66AE0
:10360000030EE66EE66AFDEC56F0006E060EE15E15
:103610000050B0EF1DF0020E0F01105D03E113EC3E
:103620001FF01FD06FD80F0123511AE105CFE9FF1A
:1036300006CFEAFFEE52080EEF6E05CFE9FF06CF88
:10364000EAFF020EE926000EEA22200EEE6E040EBC
:10365000ED6E05CFE9FF06CFEAFF8C0EEF6E01D0CD
:10366000236B1200D9CFE6FFE1CFD9FFE6520BCF93
:10367000E9FF0CCFEAFFEF50400B01E0010EDF6ED7
:103680000F010B75080E005D0DE122C45EFF0F01F6
:103690005E51000804E20F01100E006F03D00F010D
:1036A000040E006F100528E10BCFE9FF0CCFEAFFF5
:1036B000020EE926000EEA22280EEE6E040EED6ED2
:1036C00024DB020E0F010F5D07E10BCFE9FF0CCFEA
:1036D000EAFF840EEF6E0FD0DF5007E10BCFE9FF5A
:1036E0000CCFEAFFC80EEF6E06D00BCFE9FF0CCF70
:1036F000EAFF880EEF6E01D005D8E552E552E7CF1C
:10370000D9FF1200D9CFE6FFE1CFD9FF020EE126A3
:103710000F01106B0BCFE9FF0CCFEAFFEF6A040E2D
:103720000B19006E0CCF01F000C0DEFF01C0DDFF01
:10373000DECFE9FFDDCFEAFFEF6A19AF0FD01C51F2
:103740001D111E1109E007D01ECFFBFF1DCFFAFF90
:103750000F011C51F96EF8DF0F01199F020EE15C99
:1037600002E2E16AE552E16EE552E7CFD9FF1200CD
:1037700004012051600BE842E842E842E842E84296
:10378000000901E058D021510C0A54E00B0A43E033
:103790000C0A35E0010A26E00B0A22E0020A20E0CA
:1037A000030A1CE0080A10E0010A0CE00F0A08E016
:1037B000030A01E03FD00F01148F080E006F3BD0C9
:1037C000C7D839D0D0DB37D00F01010E116F0F0EE3
:1037D000126F1481010E156F148F2DD060D92BD06C
:1037E0002BD829D024510F01116F126B020E112713
:1037F0000F0E12231481010E156F148F1CD00F01B0
:10380000148F04012451EA6A020FE96E0F0EEA22B6
:1038100022C4EFFF10D0000EE66EE66AE66EE66A9E
:10382000020EE66EE66AFDEC56F0006E060EE15EF4
:10383000005001D000D01200D9CFE6FFE1CFD9FF70
:10384000040EE1260401220510E120511F0B00099E
:103850000CE10F01148F030E0401215D04E10F013F
:10386000010E216F02D00F01216B0401225166E18C
:1038700020511F0B020862E124510F0B00095EE08A
:103880000F01148F040124BF10D024510F0BE96ED7
:10389000EA6AD890E936EA36070EE9260F0EEA22E0
:1038A000EECFDEFFEDCFDDFF0FD024510F0BE96E21
:1038B000EA6AD890E936EA360B0EE9260F0EEA22BC
:1038C000EECFDEFFEDCFDDFF030E215D07E1DECFA2
:1038D000E9FFDDCFEAFF840EEF6E30D024510F0BED
:1038E000016A4C0F006E0F0E0122020E00C0DBFFBA
:1038F000030E01C0DBFF020EDBCFE9FF030EDBCFBF
:10390000EAFFEF9024AF0DD0DECFE9FFDDCFEAFF75
:10391000EF6ADF74DECFE9FFDDCFEAFF400EEF6E26
:103920000DD0DECFE9FFDDCFEAFF880EEF6EDF744A
:10393000DECFE9FFDDCFEAFFC80EEF6E040EE15CDB
:1039400002E2E16AE552E16EE552E7CFD9FF1200EB
:10395000800E0401205D01E0A1D00F01C00E146FA4
:1039600004012351030A56E0010A10E0030A03E0B0
:103970000F01146B93D00F01D00E116FB80E126FA0
:10398000000E136F120E156F166B88D0940E006E1A
:10399000B90E016E000E026E22C403F0046A056ABD
:1039A000030E246E256A266A03C01FF004C020F0AF
:1039B00005C021F0ACEC5BF01CC003F01DC004F0AE
:1039C0001EC005F000500324F36E01500420F46E75
:1039D00002500520F86EF4CFF7FFF3CFF6FF090091
:1039E000F5CF11FF0900F5CF12FF0800F5CF13FF47
:1039F00011CFF6FF12CFF7FF13CFF8FF020EF62616
:103A0000000EF722F8220900F5CF15FF0A00F5CFC6
:103A100016FF44D0030E225D3EE2970E006EB90EF3
:103A2000016E000E026E22C403F0046A056A030EE2
:103A3000246E256A266A03C01FF004C020F005C06A
:103A400021F0ACEC5BF01CC003F01DC004F01EC004
:103A500005F000500324F36E01500420F46E025070
:103A60000520F86EF4CFF7FFF3CFF6FF0900F5CF8E
:103A700011FF0900F5CF12FF0800F5CF13FF11CF9A
:103A8000F6FF12CFF7FF13CFF8FF0800F5500F0134
:103A9000156F166B02D00F01146B00D01200D9CF36
:103AA000E6FFE1CFD9FF020EE1260401286B296B66
:103AB00020511F0B020A12E0030A0DE0010A01E087
:103AC0003BD00F01148F040128810F01210502E171
:103AD0000401288331D00F01148F2ED00F01148FD1
:103AE000040124BF10D024510F0BE96EEA6AD8906C
:103AF000E936EA36070EE9260F0EEA22EECFDEFFA0
:103B0000EDCFDDFF0FD024510F0BE96EEA6AD8909C
:103B1000E936EA360B0EE9260F0EEA22EECFDEFF7B
:103B2000EDCFDDFFDECFE9FFDDCFEAFFEF50040B85
:103B300002E0010E286F00D00F0114AF07D0280E4D
:103B4000116F040E126F1481020E156F020EE15CEC
:103B500002E2E16AE552E16EE552E7CFD9FF1200D9
:103B600065980F0114BF4AD019AF28D0020E106F0C
:103B70000BCFE9FF0CCFEAFFEE52EF6A0BCFE9FF64
:103B80000CCFEAFFC80EEF6E05CFE9FF06CFEAFFC4
:103B9000EE52080EEF6E05CFE9FF06CFEAFF020EE8
:103BA000E926000EEA22280EEE6E040EED6E05CF19
:103BB000E9FF06CFEAFFC80EEF6E1FD005CFE9FF81
:103BC00006CFEAFFEE52080EEF6E05CFE9FF06CFF3
:103BD000EAFF020EE926000EEA22200EEE6E040E27
:103BE000ED6E05CFE9FF06CFEAFF8C0EEF6E0BCF2F
:103BF000E9FF0CCFEAFF840EEF6E86D019BF84D0A8
:103C0000040120AF59D00F0115510401265D0F01A9
:103C100016510401275904E226C415FF27C416FFD4
:103C200074D80F01010E106F05CFE9FF06CFEAFF30
:103C3000EE52080EEF6E05CFE9FF06CFEAFF020E47
:103C4000E926000EEA22200EEE6E040EED6E05CF80
:103C5000E9FF06CFEAFF800EEF6E236B03CFE9FF8B
:103C600004CFEAFFEE52080EEF6E03CFE9FF04CF58
:103C7000EAFF020EE926000EEA22200EEE6E040E86
:103C8000ED6E03CFE9FF04CFEAFF840EEF6E010E65
:103C9000236F0BCFE9FF0CCFEAFF020EE926000EDF
:103CA000EA22280EEE6E040EED6E0BCFE9FF0CCF6C
:103CB000EAFFC80EEF6E28D00F01020E106F0BCF77
:103CC000E9FF0CCFEAFFEE52EF6A0BCFE9FF0CCF12
:103CD000EAFFC80EEF6E05CFE9FF06CFEAFFEE520E
:103CE000080EEF6E05CFE9FF06CFEAFF020EE926C8
:103CF000000EEA22280EEE6E040EED6E05CFE9FFEF
:103D000006CFEAFFC80EEF6E1200D9CFE6FFE1CF73
:103D1000D9FF020EE1260F01080E155D000E16599F
:103D20000EE215CFDEFF16CFDDFF0F5103E1010ECE
:103D30000F6F04D00F0502E1020E0F6F03D0080EC3
:103D4000DE6EDD6A0BCFE9FF0CCFEAFFEF920BCFFF
:103D5000E9FF0CCFEAFFEF900BCFE9FF0CCFEAFFB2
:103D6000010EDB50EF120BCFE9FF0CCFEAFFEE5252
:103D7000DFCFEFFF000EDB50155F010EDB50165B4F
:103D8000280E1F6F040E206F14B124D0D9CFE9FF85
:103D9000DACFEAFFEE50ED101CE011CFF6FF112B49
:103DA00012CFF7FF000E122313CFF8FF13230800E2
:103DB000F550E66E1FCFE9FF20CFEAFF1F2B000E64
:103DC0002023E552E750EF6EDF06010E01E2DB062D
:103DD000DDD71FD0D9CFE9FFDACFEAFFEE50ED10E3
:103DE00018E011CFE9FF12CFEAFF112B000E1223CA
:103DF000EF50E66E1FCFE9FF20CFEAFF1F2B000E2A
:103E00002023E552E750EF6EDF06010E01E2DB06EC
:103E1000E1D7020EE15C02E2E16AE552E16EE552B1
:103E2000E7CFD9FF1200D9CFE6FFE1CFD9FF020ECD
:103E3000E12603CFE9FF04CFEAFFEE52EFCFDFFF29
:103E4000DFCF00F000500F011A5D000E1B5902E297
:103E50001ACFDFFFDF50006E016A00501A5D1A6F43
:103E600001501B591B6F010EDB6ADF50F36E010E10
:103E7000DBCFF4FFF350F45C16E2010EDB50EA6A8C
:103E8000280FE96E040EEA22EF50E66E17CFE9FF25
:103E900018CFEAFF172B000E1823E552E750EF6EFC
:103EA000010EDB2AE2D7000ED8801A55000E1B55F2
:103EB00028E205CFE9FF06CFEAFFEE52080EEF6ECB
:103EC00005CFE9FF06CFEAFF020EE926000EEA223F
:103ED000280EEE6E040EED6E03CFE9FF04CFEAFF6D
:103EE000EF50400B07E105CFE9FF06CFEAFFC80E10
:103EF000EF6E06D005CFE9FF06CFEAFF880EEF6E22
:103F000028D005CFE9FF06CFEAFFEE52080EEF6E8C
:103F100005CFE9FF06CFEAFF020EE926000EEA22EE
:103F2000200EEE6E040EED6E05CFE9FF06CFEAFF20
:103F3000840EEF6E1C511D111E1109E007D01ECF1B
:103F4000FBFF1DCFFAFF0F011C51F96EF8DF0F01C7
:103F5000199F020EE15C02E2E16AE552E16EE55270
:103F6000E7CFD9FF1200D9CFE6FFE1CFD9FFE65264
:103F70000F01148F010EE66EE66AE66A4D0EE66EDC
:103F80000F0EE66EA4EC59F0006E050EE15E0050D7
:103F9000DF6ADF50006E016A080E005C000E0158F7
:103FA00010E2DF50040DF3CFE9FFF4CFEAFF000E7B
:103FB000E926040EEA22EE6AEE6AEE6AEE6ADF2A6B
:103FC000E8D7658C010EE66EE66AE66A020EE66EDA
:103FD0000F0EE66EA4EC59F0006E050EE15E005087
:103FE000659C0F01080E0B6F040E0C6F000E036F23
:103FF000040E046F03CF05FF04CF06FF22C401FFA8
:10400000015103E1100E006F13D0010EE66EE66A57
:10401000010EE66E0F0EE66E010EE66EE66AFDEC30
:1040200056F0006E060EE15E00500F01200E006F8C
:10403000E552E552E7CFD9FF1200D9CFE6FFE1CF35
:10404000D9FF020EE126000EDE6E040EDD6EFD0EBF
:10405000DB50E824026EFE0EDB50040DF350022408
:10406000040DF350006E016A020E0F0B05E0D890AC
:1040700001320032E806FBE1D89000360136D890D4
:1040800000360136D9CFE9FFDACFEAFF0050EE263D
:104090000150ED22DECFE9FFDDCFEAFFEF9EFD0EFE
:1040A000DB500FE1FE0EEA6ADB34FE0BEA36E96E06
:1040B000070EE9260F0EEA22DECFEEFFDDCFEDFF81
:1040C0000ED0FE0EEA6ADB34FE0BEA36E96E0B0E0A
:1040D000E9260F0EEA22DECFEEFFDDCFEDFFDECFC9
:1040E000E9FFDDCFEAFFEF9CDECFE9FFDDCFEAFF9E
:1040F000040EE926000EEA22EF8C020EE15C02E2D9
:10410000E16AE552E16EE552E7CFD9FF1200D9CF5F
:10411000E6FFE1CFD9FF020EE126FE0EDB50016A79
:104120004C0F006E0F0E012200C0DEFF01C0DDFF4C
:10413000DECFE9FFDDCFEAFFFD0EDBCFEFFFDBA433
:1041400007D0E66AFE0EDBCFE6FF77DFE552E552E9
:10415000FD0EDBA208D0010EE66EFE0EDBCFE6FF01
:104160006CDFE552E552020EE15C02E2E16AE552E3
:10417000E16EE552E7CFD9FF1200D9CFE6FFE1CFDC
:10418000D9FF020EE126FE0EDB5020E105CFE9FF4C
:1041900006CFEAFFEE52080EEF6E05CFE9FF06CF1D
:1041A000EAFF020EE926000EEA22200EEE6E040E51
:1041B000ED6E05CFE9FF06CFEAFF8C0EEF6E0BCF59
:1041C000E9FF0CCFEAFF840EEF6E3DD0FD0EDB5011
:1041D000E824026EFE0EDB50040DF3500224040DA1
:1041E000F3CF00F0F4CF01F0000E0026040E012200
:1041F00000C0DEFF01C0DDFF840E006EDECFE9FFF0
:10420000DDCFEAFF0050EF12FD0EDB50E824026E16
:10421000FE0EDB50040DF3500224010F040DF3CF0A
:1042200000F0F4CF01F0000E0026040E012200C0C1
:10423000DEFF01C0DDFF840E006EDECFE9FFDDCFC3
:10424000EAFF0050EF12020EE15C02E2E16AE55281
:10425000E16EE552E7CFD9FF1200D9CFE6FFE1CFFB
:10426000D9FF020EE126FD0EDB500FE0FE0EEA6ADA
:10427000DB34FE0BEA36E96E0B0EE9260F0EEA225E
:10428000EECFDEFFEDCFDDFF0ED0FE0EEA6ADB34AF
:10429000FE0BEA36E96E070EE9260F0EEA22EECF94
:1042A000DEFFEDCFDDFFD9CFE9FFDACFEAFFEE5039
:1042B000ED1003E1F36AF46A49D0DECFE9FFDDCF08
:1042C000EAFF020EE926000EEA22FB0EDBCFEEFF2C
:1042D000FC0EDBCFEDFFDECFE9FFDDCFEAFFEE52D4
:1042E000FA0EDBCFEFFF400E006EDECFE9FFDDCF31
:1042F000EAFF0050EF16880E006EDECFE9FFDDCF3B
:10430000EAFF0050EF12FD0EDB500CE0FE0EEA6AF1
:10431000DB34FE0BEA36E96E0B0EE9260F0EEA22BD
:10432000EF740BD0FE0EEA6ADB34FE0BEA36E96E60
:10433000070EE9260F0EEA22EF74DECF00F0DDCF84
:1043400001F000C0F3FF01C0F4FF00D0020EE15CF9
:1043500002E2E16AE552E16EE552E7CFD9FF1200D1
:10436000D9CFE6FFE1CFD9FF65A84ED0FE0EEA6AAD
:10437000DB34FE0BEA36E96E0B0EE9260F0EEA225D
:10438000EE50EFCFEAFFE96E400EEE16EE6AEE6AEF
:10439000EE6AFE0EEA6ADB34FE0BEA36E96E0B0EBD
:1043A000E9260F0EEA22EE50EFCFEAFFE96EEE7C2F
:1043B000FE0EEA6ADB34FE0BEA36E96E0B0EE926E6
:1043C0000F0EEA22EF74400E006EFE0EEA6ADB3436
:1043D000FE0BEA36E96E0B0EE9260F0EEA22EE50CE
:1043E000EFCFEAFFE96E0050EF16FE0EEA6ADB340B
:1043F000FE0BEA36E96E0B0EE9260F0EEA22EE50AE
:10440000EFCFEAFFE96EEF7CE552E7CFD9FF12006C
:10441000656A0F015C6B0F01006B00D012000F0189
:10442000005114E1656A0F015C6B160E5F6F9F0E01
:104430005D6F7B0E5C6FD08EA288A088F28E65B611
:0E44400002D06586FCD70F01010E006F12003E
:02444E00D9CFC4
:10445000E6FFE1CFD9FF0B0EE126040EDB6A050E65
:10446000DB6A000EE66EE66A360EE66E040EE66E57
:10447000C4EC4DF0E552E552E552E552360EDE6EE3
:10448000040EDD6E060EDB6ADBCF00F0200EE76E59
:104490000018E8AE02D0E73402D0E750005C1AE220
:1044A000DECFE9FFDDCFEAFFE9CF00F0EACF01F090
:1044B000060EDBCF02F0036A02BE0368005002243E
:1044C000E96E01500320EA6EEF5001E103D0060EC1
:1044D000DB2ADAD7060EDBCF00F0200EE76E0018DD
:1044E000E8AE02D0E73402D0E750005C10E2DECF45
:1044F000E9FFDDCFEAFFEFCF01F0300E015C07E30B
:10450000DECFE9FFDDCFEAFFEF507A081DE2A60E0D
:10451000E66EA40EE66E000EE66EDECFE9FFDDCF9E
:10452000EAFFE9CF00F0EACF01F000C0E6FF01C0EA
:10453000E6FF1FEC5AF0026E050EE15E0250010E1E
:10454000F36E040EF3CFDBFFDECFE9FFDDCFEAFF32
:10455000200EE926000EEA22EECF00F0EFCF01F0A8
:10456000D890015004E6190E005C000E015813E3C8
:10457000DECFE9FFDDCFEAFF200EE926000EEA22BA
:10458000EECF02F0EFCF03F0033404E202503C0818
:10459000000E035410E2DECFE9FFDDCFEAFF200E6C
:1045A000E926000EEA222A0EEE6EED6A010EF36E87
:1045B000040EF3CFDBFFDECFE9FFDDCFEAFF220EF3
:1045C000E926000EEA22EECF00F0EFCF01F0D890FE
:1045D000015004E6190E005C000E015813E3DECF13
:1045E000E9FFDDCFEAFF220EE926000EEA22EECF38
:1045F00002F0EFCF03F0033404E202504108000E52
:10460000035410E2DECFE9FFDDCFEAFF220EE926F8
:10461000000EEA22370EEE6EED6A010EF36E040E06
:10462000F3CFDBFFDECFE9FFDDCFEAFF240EE92683
:10463000000EEA22EECF00F0EFCF01F0D89001504B
:1046400004E6190E005C000E015813E3DECFE9FF0B
:10465000DDCFEAFF240EE926000EEA22EECF02F0BB
:10466000EFCF03F0033404E202504108000E03547C
:1046700010E2DECFE9FFDDCFEAFF240EE926000ECF
:10468000EA222A0EEE6EED6A010EF36E040EF3CFEF
:10469000DBFFDECFE9FFDDCFEAFF300EE926000EBB
:1046A000EA22EECF00F0EFCF01F0013404E2005037
:1046B0000008000E015414E2DECFE9FFDDCFEAFF6F
:1046C000300EE926000EEA22EECF02F0EFCF03F023
:1046D000033404E2025000087D0E035401E389D044
:1046E000DECFE9FFDDCFEAFF300EE926000EEA2239
:1046F000140EEE6EED6ADECFE9FFDDCFEAFF320E7B
:10470000E926000EEA22400EEE6EED6ADECFE9FFEA
:10471000DDCFEAFF340EE926000EEA220A0EEE6E25
:10472000ED6ADECFE9FFDDCFEAFF360EE926000EA7
:10473000EA22320EEE6EED6ADECFE9FFDDCFEAFF50
:10474000380EE926000EEA22200EEE6EED6ADECF6C
:10475000E9FFDDCFEAFF3A0EE926000EEA22800EDD
:10476000EE6EED6ADECFE9FFDDCFEAFF3C0EE92613
:10477000000EEA220A0EEE6EED6ADECFE9FFDDCF13
:10478000EAFF3E0EE926000EEA22460EEE6EED6AC4
:10479000DECFE9FFDDCFEAFF400EE926000EEA2278
:1047A000200EEE6EED6ADECFE9FFDDCFEAFF420EAE
:1047B000E926000EEA22800EEE6EED6ADECFE9FFFA
:1047C000DDCFEAFF440EE926000EEA220A0EEE6E65
:1047D000ED6ADECFE9FFDDCFEAFF460EE926000EE7
:1047E000EA223C0EEE6EED6A010EF36E040EF3CF7C
:1047F000DBFFDECFE9FFDDCFEAFF480EE926000E42
:10480000EA22EECF00F0EFCF01F0D880015004E7AC
:10481000EC0E005CFF0E015840E3DECFE9FFDDCF78
:10482000EAFF480EE926000EEA22EECF02F0EFCFB3
:1048300003F0033404E202501408000E03542DE385
:10484000DECFE9FFDDCFEAFF480EE926000EEA22BF
:10485000FF0EEE1802E1FF0EED1801E0CBD0DECF27
:10486000E9FFDDCFEAFF500EE926000EEA22FF0E37
:10487000EE1802E1FF0EED1801E0BCD0DECFE9FF3B
:10488000DDCFEAFF580EE926000EEA22FF0EEE18F1
:1048900002E1FF0EED1801E0ADD0DECFE9FFDDCF84
:1048A000EAFF480EE926000EEA22010EEE6EED6ADE
:1048B000DECFE9FFDDCFEAFF480EE926000EEA224F
:1048C000020EE926000EEA22020EEE6EED6ADECF3F
:1048D000E9FFDDCFEAFF480EE926000EEA22040ECA
:1048E000E926000EEA22030EEE6EED6ADECFE9FF46
:1048F000DDCFEAFF480EE926000EEA22060EE92681
:10490000000EEA22040EEE6EED6ADECFE9FFDDCF87
:10491000EAFF500EE926000EEA22FD0EEE6EED686B
:10492000DECFE9FFDDCFEAFF500EE926000EEA22D6
:10493000020EE926000EEA22FD0EEE6EED68DECFD5
:10494000E9FFDDCFEAFF500EE926000EEA22040E51
:10495000E926000EEA22FC0EEE6EED68DECFE9FFDE
:10496000DDCFEAFF500EE926000EEA22060EE92608
:10497000000EEA22FB0EEE6EED68DECFE9FFDDCF22
:10498000EAFF580EE926000EEA22FD0EEE6EED68F3
:10499000DECFE9FFDDCFEAFF580EE926000EEA225E
:1049A000020EE926000EEA22FC0EEE6EED68DECF66
:1049B000E9FFDDCFEAFF580EE926000EEA22040ED9
:1049C000E926000EEA22FB0EEE6EED68DECFE9FF6F
:1049D000DDCFEAFF580EE926000EEA22060EE92690
:1049E000000EEA22FB0EEE6EED68010EF36E040E71
:1049F000F3CFDBFFDECFE9FFDDCFEAFF6A0EE9266A
:104A0000000EEA22EE50ED101AE0DECFE9FFDDCF16
:104A1000EAFF6A0EE926000EEA22010EEE1801E115
:104A2000ED500DE0DECFE9FFDDCFEAFF6A0EEB6A65
:104A30006B0EEB6A010EF36E040EF3CFDBFFDECFDD
:104A4000E9FFDDCFEAFF700EE926000EEA22EECF85
:104A500000F0EFCF01F00001800E011414E1DECF71
:104A6000E9FFDDCFEAFF700EE926000EEA22EECF65
:104A700002F0EFCF03F0D890035004E6A00E025CE2
:104A8000050E03580DE3DECFE9FFDDCFEAFF700E20
:104A9000EB6A710EEB6A010EF36E040EF3CFDBFFCF
:104AA000DECFE9FFDDCFEAFF780EE926000EEA222D
:104AB000E868EE1808E1E868EE1805E1E868EE1825
:104AC00002E1E868EE1800E1DECFE9FFDDCFEAFFA2
:104AD000760EE926000EEA22EE50ED101AE0DECF47
:104AE000E9FFDDCFEAFF760EE926000EEA22010E8D
:104AF000EE1801E1ED500DE0DECFE9FFDDCFEAFF7A
:104B0000760EEB6A770EEB6A010EF36E040EF3CFAE
:104B1000DBFF040EDB500DE0000EE66EE66A360E9B
:104B2000E66E040EE66E84EC4BF0E552E552E5527B
:104B3000E552010EE66EE66A360EE66E040EE66E8D
:104B4000C4EC4DF0E552E552E552E552D950020F62
:104B5000E96EDACFEAFF360EEE6E040EED6E060E4B
:104B6000DB6ADBCF00F0070EE76E0018E8AE02D07C
:104B7000E73402D0E750005C01E382D1020EDBCFC4
:104B8000E9FF030EDBCFEAFFE9CF02F0EACF03F043
:104B9000060EDBCF04F0056A04BE0568D890043623
:104BA000053602500424E96E03500520EA6EEECF6C
:104BB00000F0EFCF01F0000E0001015C60E3020E97
:104BC000DBCFE9FF030EDBCFEAFFE9CF08F0EACF46
:104BD00009F0060EDBCF0AF00B6A0ABE0B68D8900C
:104BE0000A360B3608500A24E96E09500B20EA6E8B
:104BF000EECF06F0EFCF07F0180E075C40E2020E92
:104C0000DBCFE9FF030EDBCFEAFFE9CF0EF0EACFFF
:104C10000FF0060EDBCF10F0116A10BE1168D890AD
:104C2000103611360E501024E96E0F501120EA6E26
:104C3000EECF0CF0EFCF0DF0000E0C5C20E3020E77
:104C4000DBCFE9FF030EDBCFEAFFE9CF14F0EACFB9
:104C500015F0060EDBCF16F0176A16BE1768D8904F
:104C60001636173614501624E96E15501720EA6EC2
:104C7000EECF12F0EFCF13F03C0E125C21E3020EE8
:104C8000DBCFE9FF030EDBCFEAFFE9CF00F0EACF8D
:104C900001F0060EDBCF02F0036A02BE0368D89073
:104CA0000236033600500224E96E01500320EA6EFA
:104CB000EE6A080EED6E010EF36E050EF3CFDBFF0C
:104CC000020EDBCFE9FF030EDBCFEAFF0E0EE92673
:104CD000000EEA22E9CF02F0EACF03F0060EDBCFA6
:104CE00004F0056A04BE0568D89004360536025003
:104CF0000424E96E03500520EA6EEECF00F0EFCFFA
:104D000001F0000E015C6CE3020EDBCFE9FF030E45
:104D1000DBCFEAFF0E0EE926000EEA22E9CF08F00B
:104D2000EACF09F0060EDBCF0AF00B6A0ABE0B6869
:104D3000D8900A360B3608500A24E96E09500B2029
:104D4000EA6EEECF06F0EFCF07F0180E075C48E2F0
:104D5000020EDBCFE9FF030EDBCFEAFF0E0EE926E2
:104D6000000EEA22E9CF0EF0EACF0FF0060EDBCFFD
:104D700010F0116A10BE1168D890103611360E501E
:104D80001024E96E0F501120EA6EEECF0CF0EFCF39
:104D90000DF0000E0C5C24E3020EDBCFE9FF030EE6
:104DA000DBCFEAFF0E0EE926000EEA22E9CF14F06F
:104DB000EACF15F0060EDBCF16F0176A16BE17689D
:104DC000D8901636173614501624E96E1550172051
:104DD000EA6EEECF12F0EFCF13F03C0E125C4DE313
:104DE000060EDB5004E0060EDB50060821E1020E41
:104DF000DBCFE9FF030EDBCFEAFF0E0EE926000E44
:104E0000EA22E9CF00F0EACF01F0060EDBCF02F094
:104E1000036A02BE0368D8900236033600500224AB
:104E2000E96E01500320EA6EEE6A080EED6E20D0A6
:104E3000020EDBCFE9FF030EDBCFEAFF0E0EE92601
:104E4000000EEA22E9CF00F0EACF01F0060EDBCF38
:104E500002F0036A02BE0368D8900236033600509F
:104E60000224E96E01500320EA6EEE6A110EED6E27
:104E7000010EF36E050EF3CFDBFF060EDB2A71D6B3
:104E8000020EDBCFE9FF030EDBCFEAFF1C0EE926A3
:104E9000000EEA22EE50ED101EE0020EDBCFE9FF1D
:104EA000030EDBCFEAFF1C0EE926000EEA22010EFC
:104EB000EE1801E1ED500FE0020EDBCFE9FF030E2B
:104EC000DBCFEAFF1C0EEB6A1D0EEB6A010EF36EE0
:104ED000050EF3CFDBFF050EDB500DE0010EE66E95
:104EE000E66A360EE66E040EE66E84EC4BF0E55292
:104EF000E552E552E552040EDB5005E1050EDB50AC
:104F000002E1000E01D0010E006E0B0EE15C03E227
:104F100000D0E16AE552E16E0050E552E7CFD9FFDB
:104F20001200D9CFE6FFE1CFD9FF020EE126000E35
:104F3000E66EE66A360EE66E040EE66EC4EC4DF0E2
:104F4000E552E552E552E552360EDE6E040EDD6E98
:104F5000DECFE9FFDDCFEAFF200EE926000EEA22D0
:104F6000EECF00F0EFCF01F0FD0EDBCFE9FFFE0E3C
:104F7000DBCFEAFF00C0EEFF01C0EDFFDECFE9FFAF
:104F8000DDCFEAFF220EE926000EEA22EECF00F086
:104F9000EFCF01F0FB0EDBCFE9FFFC0EDBCFEAFF2A
:104FA00000C0EEFF01C0EDFFDECFE9FFDDCFEAFF7D
:104FB000240EE926000EEA22EECF00F0EFCF01F03A
:104FC000F90EDBCFE9FFFA0EDBCFEAFF00C0EEFF00
:104FD00001C0EDFF020EE15C02E2E16AE552E16E22
:104FE000E552E7CFD9FF1200D9CFE6FFE1CFD9FFD5
:104FF000020EE126000EE66EE66A360EE66E040E3E
:10500000E66EC4EC4DF0E552E552E552E552360E3F
:10501000DE6E040EDD6EDECFE9FFDDCFEAFF200E8F
:10502000E926000EEA22FD0EDBCFEEFFFE0EDBCFFF
:10503000EDFFDECFE9FFDDCFEAFF220EE926000E0D
:10504000EA22FB0EDBCFEEFFFC0EDBCFEDFFDECF67
:10505000E9FFDDCFEAFF240EE926000EEA22F90E71
:10506000DBCFEEFFFA0EDBCFEDFF000EE66EE66A59
:10507000360EE66E040EE66E84EC4BF0E552E55219
:10508000E552E552020EE15C02E2E16AE552E16EB0
:10509000E552E7CFD9FF1200D9CFE6FFE1CFD9FF24
:1050A000020EE126000EE66EE66A360EE66E040E8D
:1050B000E66EC4EC4DF0E552E552E552E552360E8F
:1050C000DE6E040EDD6EDECFE9FFDDCFEAFFEF50CE
:1050D000FF0804E1F36AF46A0ED00DD0DECFE9FFD9
:1050E000DDCFEAFFE9CF00F0EACF01F000C0F3FF27
:1050F00001C0F4FF00D0020EE15C02E2E16AE55279
:10510000E16EE552E7CFD9FF1200D9CFE6FFE1CF3C
:10511000D9FF020EE126000EE66EE66A360EE66E56
:10512000040EE66EC4EC4DF0E552E552E552E55250
:10513000360EDE6E040EDD6E0201805112E0DECF0F
:10514000E9FFDDCFEAFF700EE926000EEA22EECF7E
:1051500000F0EFCF01F000C0F3FF01C0F4FF04D076
:1051600003D0F36AF46A00D0020EE15C02E2E16A65
:10517000E552E16EE552E7CFD9FF1200D9CFE6FF45
:10518000E1CFD9FF020EE126000EE66EE66A360E8A
:10519000E66E040EE66EC4EC4DF0E552E552E552C3
:1051A000E552360EDE6E040EDD6EDECFE9FFDDCF9A
:1051B000EAFF700EE926000EEA22FD0EDBCFEEFFBD
:1051C000FE0EDBCFEDFF000EE66EE66A360EE66EF3
:1051D000040EE66E84EC4BF0E552E552E552E552E2
:1051E000020EE15C02E2E16AE552E16EE552E7CFD0
:1051F000D9FF1200D9CFE6FFE1CFD9FF020EE12699
:10520000000EE66EE66A360EE66E040EE66EC4EC3E
:105210004DF0E552E552E552E552360EDE6E040ED3
:10522000DD6EDECFE9FFDDCFEAFF760EE926000E68
:10523000EA22010EEE1801E1ED5002E1010E01D06B
:10524000000E006E020EE15C03E200D0E16AE5525E
:10525000E16E0050E552E7CFD9FF1200D9CFE6FF4B
:10526000E1CFD9FF060EE1260201806B0201816BBE
:10527000826B836B846B000EE66EE66A360EE66E1A
:10528000040EE66EC4EC4DF0E552E552E552E552EF
:10529000360EDE6E040EDD6EDECFE9FFDDCFEAFFF7
:1052A000780EE926000EEA22E9CF00F0EACF01F0FD
:1052B00000C0E6FF01C0E6FF200EE66E57EC17F0D7
:1052C000E552E552E55200680168026A036ADECFE2
:1052D000E9FFDDCFEAFF7C0EE926000EEA22EE5060
:1052E0000016EE500116EE500216EE500316420E56
:1052F000001806E1530E011803E1025001E10350CA
:1053000001E0C0D0006A016A026A0368DECFE9FFEB
:10531000DDCFEAFF780EE926000EEA22EE500016F5
:10532000EE500116EE500216EE500316005006E144
:10533000015004E1025002E1540E031801E0A2D032
:10534000DECFE9FFDDCFEAFF780EE926000EEA2284
:10535000EECF81F2EECF82F2EECF83F2EFCF84F286
:105360000201846BEEC000F0EFC001F0026A036A34
:1053700001AE02D002680368020E00C0DBFF030E1C
:1053800001C0DBFF040E02C0DBFF050E03C0DBFF24
:10539000020EDBCF00F0030EDBCF01F0040EDBCFFB
:1053A00002F0050EDBCF03F0080E1F0B07E0D890CC
:1053B0000036013602360336E806F9E1ECC004F0A7
:1053C000EDC005F0066A076A05AE02D006680768F8
:1053D0000450001205500112065002120750031229
:1053E000020E00C0DBFF030E01C0DBFF040E02C093
:1053F000DBFF050E03C0DBFF020EDBCF00F0030E68
:10540000DBCF01F0040EDBCF02F0050EDBCF03F0A3
:10541000080E1F0B07E0D89000360136023603361F
:10542000E806F9E1EAC004F0EBC005F0066A076A95
:1054300005AE02D00668076804500012055001123C
:105440000650021207500312020E00C0DBFF030ECB
:1054500001C0DBFF040E02C0DBFF050E03C0DBFF53
:10546000D950020FE96EDACFEAFFEE500201815DFA
:10547000EE508259EE508359EE50845903E30201F5
:10548000010E806F060EE15C02E2E16AE552E16E18
:10549000E552E7CFD9FF1200D9CFE6FFE1CFD9FF20
:1054A000020EE126010EE66EE66A360EE66E040E88
:1054B000E66EC4EC4DF0E552E552E552E552360E8B
:1054C000DE6E040EDD6EDECFE9FFDDCFEAFF1C0EDF
:1054D000E926000EEA22FD0EDBCFEEFFFE0EDBCF4B
:1054E000EDFF010EE66EE66A360EE66E040EE66E1F
:1054F00084EC4BF0E552E552E552E552020EE15CD8
:1055000002E2E16AE552E16EE552E7CFD9FF12000F
:10551000D9CFE6FFE1CFD9FF020EE126FE0EDB5028
:10552000020A0FE0030A08E0010A01E010D1080EA8
:10553000DE6E010EDD6E0AD02E0EDE6E010EDD6E09
:1055400005D0540EDE6E010EDD6E00D0DECFE9FF19
:10555000DDCFEAFF020EE926000EEA22EECF00F0D0
:10556000EFCF01F0DECFE9FFDDCFEAFF040EE92641
:10557000000EEA2200C0EEFF01C0EDFFFE0EDBCF01
:10558000E6FFF8EC4EF0E552006E016A00BE0168DD
:10559000DECFE9FFDDCFEAFF020EE926000EEA22A8
:1055A00000C0EEFF01C0EDFFDECFE9FFDDCFEAFF77
:1055B000020EE926000EEA22FF0EEE1802E1FF0EAF
:1055C000ED1822E1FE0EDBCFE6FF45EC3DF0E552A3
:1055D000FE0EDB50020A11E0030A09E0010A01E0B5
:1055E00012D0320EE66E48EC57F0E5520CD0330E76
:1055F000E66E48EC57F0E55206D0340EE66E48EC05
:1056000057F0E55200D0A3D00201C35101E09FD072
:10561000DECFE9FFDDCFEAFFEECF00F0EFCF01F004
:10562000D890015004E6320E005C000E015819E2D9
:10563000DECFE9FFDDCFEAFF1E0EE926000EEA22EB
:10564000EECF00F0EFCF01F0DECFE9FFDDCFEAFFD4
:10565000020EE926000EEA220050EE260150ED224D
:1056600076D0DECFE9FFDDCFEAFFEECF00F0EFCF5F
:1056700001F0D890015004E63A0E005C000E01588B
:105680001DE2DECFE9FFDDCFEAFF1E0EE926000EA8
:10569000EA22020EE926000EEA22EECF00F0EFCF5A
:1056A00001F0DECFE9FFDDCFEAFF020EE926000EB2
:1056B000EA220050EE260150ED2249D0DECFE9FF6C
:1056C000DDCFEAFFEECF00F0EFCF01F0D890015030
:1056D00004E63F0E005C000E01581DE2DECFE9FF3C
:1056E000DDCFEAFF1E0EE926000EEA22040EE926AF
:1056F000000EEA22EECF00F0EFCF01F0DECFE9FF9F
:10570000DDCFEAFF020EE926000EEA220050EE2667
:105710000150ED221CD0DECFE9FFDDCFEAFF1E0EE7
:10572000E926000EEA22060EE926000EEA22EECF56
:1057300000F0EFCF01F0DECFE9FFDDCFEAFF020E90
:10574000E926000EEA220050EE260150ED22020E5C
:10575000E15C02E2E16AE552E16EE552E7CFD9FF92
:105760001200D9CFE6FFE1CFD9FF020EE126D950D2
:10577000FD0FE96EFF0EDA20EA6EEE50ED1001E14A
:1057800030D2FD0EDBCFE9FFFE0EDBCFEAFFEECF1E
:1057900002F0EFCF03F0FD0EDBCFE9FFFE0EDBCF13
:1057A000EAFF020EE926000EEA22EE50025C006ECD
:1057B000EE500358016EFD0EDBCFE9FFFE0EDBCF8E
:1057C000EAFF0C0EE926000EEA2200C0EEFF01C03F
:1057D000EDFFFD0EDBCFE9FFFE0EDBCFEAFF100E83
:1057E000E926000EEA22EECF02F0EFCF03F0FD0E25
:1057F000DBCFE9FFFE0EDBCFEAFF0C0EE926000E41
:10580000EA22EECF04F0EFCF05F0000104500202CF
:10581000F3CF00F0F4CF01F00302F350012605505E
:105820000202F3500126FD0EDBCFE9FFFE0EDBCFB7
:10583000EAFF060EE926000EEA2200C0EEFF01C0D4
:10584000EDFFFD0EDBCFE9FFFE0EDBCFEAFF0C0E16
:10585000E926000EEA22EECF00F0EFCF01F001348E
:1058600004E200500008000E015446E2FD0EDBCFBA
:10587000E9FFFE0EDBCFEAFF120EE926000EEA2258
:10588000EECF02F0EFCF03F0020E256E266A02C0C3
:1058900020F003C021F03BEC5BF020C002F021C0FF
:1058A00003F0FD0EDBCFE9FFFE0EDBCFEAFF0C0EAF
:1058B000E926000EEA22EECF04F0EFCF05F000015A
:1058C00004500202F3CF00F0F4CF01F00302F350D2
:1058D000012605500202F3500126FD0EDBCFE9FF41
:1058E000FE0EDBCFEAFF0A0EE926000EEA22005088
:1058F000EE260150ED2245D0FD0EDBCFE9FFFE0E76
:10590000DBCFEAFF180EE926000EEA22EECF02F006
:10591000EFCF03F0020E256E266A02C020F003C00E
:1059200021F03BEC5BF020C002F021C003F0FD0E43
:10593000DBCFE9FFFE0EDBCFEAFF0C0EE926000EFF
:10594000EA22EECF04F0EFCF05F00001045002028E
:10595000F3CF00F0F4CF01F00302F350012605501D
:105960000202F3500126FD0EDBCFE9FFFE0EDBCF76
:10597000EAFF0A0EE926000EEA220050EE26015048
:10598000ED220201C25149E1FD0EDBCFE9FFFE0E1F
:10599000DBCFEAFF0A0EE926000EEA22EECF00F086
:1059A000EFCF01F0013404E2005060086D0E0154A5
:1059B0000FE2FD0EDBCFE9FFFE0EDBCFEAFF0A0EA2
:1059C000E926000EEA22600EEE6E6D0EED6E24D01A
:1059D000FD0EDBCFE9FFFE0EDBCFEAFF0A0EE92664
:1059E000000EEA22EECF00F0EFCF01F0D880015098
:1059F00004E7A00E005C920E01580EE2FD0EDBCF14
:105A0000E9FFFE0EDBCFEAFF0A0EE926000EEA22CE
:105A1000A00EEE6E920EED6E48D0FD0EDBCFE9FFCC
:105A2000FE0EDBCFEAFF0A0EE926000EEA22EECFD9
:105A300000F0EFCF01F0013404E200501808790EB5
:105A400001540FE2FD0EDBCFE9FFFE0EDBCFEAFFD4
:105A50000A0EE926000EEA22180EEE6E790EED6EA1
:105A600024D0FD0EDBCFE9FFFE0EDBCFEAFF0A0EEE
:105A7000E926000EEA22EECF00F0EFCF01F0D88049
:105A8000015004E7E80E005C860E01580EE2FD0EA0
:105A9000DBCFE9FFFE0EDBCFEAFF0A0EE926000EA0
:105AA000EA22E80EEE6E860EED6EFD0EDBCFE9FF0C
:105AB000FE0EDBCFEAFF020EE926000EEA22EECF51
:105AC00002F0EFCF03F0FD0EDBCFE9FFFE0EDBCFE0
:105AD000EAFF040EE926000EEA22EE50025C006E98
:105AE000EE500358016E00C0DEFF01C0DDFFDECFC7
:105AF00000F0DDCF01F0013404E200500008000E98
:105B0000015438E2FD0EDBCFE9FFFE0EDBCFEAFFEA
:105B10001A0EE926000EEA22EECF02F0EFCF03F0D4
:105B2000020E256E266A02C020F003C021F03BEC75
:105B30005BF020C002F021C003F002C020F003C0DF
:105B400021F0DECF25F0DDCF26F061EC5BF01EC04A
:105B500000F01FC001F0FD0EDBCFE9FFFE0EDBCF32
:105B6000EAFF080EE926000EEA2200C0EEFF01C09F
:105B7000EDFF37D0FD0EDBCFE9FFFE0EDBCFEAFFF6
:105B8000140EE926000EEA22EECF02F0EFCF03F06A
:105B9000020E256E266A02C020F003C021F03BEC05
:105BA0005BF020C002F021C003F002C020F003C06F
:105BB00021F0DECF25F0DDCF26F061EC5BF01EC0DA
:105BC00000F01FC001F0FD0EDBCFE9FFFE0EDBCFC2
:105BD000EAFF080EE926000EEA2200C0EEFF01C02F
:105BE000EDFF020EE15C02E2E16AE552E16EE55290
:105BF000E7CFD9FF1200D9CFE6FFE1CFD9FF020EE0
:105C0000E126FE0EDB5001E064D012C102F013C1A8
:105C100003F0256A010E266E02C020F003C021F0B9
:105C20003BEC5BF020C002F021C003F001010E51FB
:105C30000224006E0F510320016E1051005C166F9C
:105C400011510158176F820EDE6EDD6A093504E2CC
:105C500008513608000E09550AE20B3504E20A51D4
:105C60003608000E0B5503E2AA0EDE6EDD6A17350C
:105C700004E216518208000E175504E2DECF16F139
:105C8000DDCF17F1800E171502E0166B176B153577
:105C900004E214510A08000E155505E2DECF16F194
:105CA000DDCF17F10AD0D880155104E7FA0E145D44
:105CB000FF0E155902E2166B176B153504E21451ED
:105CC0000608000E155504E224C112F125C113F196
:105CD00000D0020EE15C02E2E16AE552E16EE552BB
:105CE000E7CFD9FF12000201BF5101011719E8AE39
:105CF00002D0173507D016510201BE5D01011751C0
:105D00000201BF5914E2E66A1EEC3EF0E552F3CF01
:105D100000F0F4CF01F00050011009E002019E05EF
:105D200006E1010EE66E5FEC3CF0E55205D0010E97
:105D3000E66EA5EC3CF0E552120002019E5101E135
:105D400060D80201C25135E102019E0532E1010134
:105D50000A51081902E10B5109192AE10201C12B6C
:105D6000020EE76EC119E8AE02D0E73402D0E75068
:105D7000C15D1AE3020EC16F010EC26F1AEC3EF054
:105D8000EE0E206E020E216E08C125F009C126F02C
:105D900061EC5BF01EC012F11FC013F10101D80EBF
:105DA000125F590E135B04D01CEC3EF00201C26B73
:105DB00027D00201C20524E1010108510A5D006EED
:105DC0000B510955016E013404E200500408000E25
:105DD000015410E30A51085D026E09510B55036E20
:105DE000033404E202500808000E035403E30201E6
:105DF0009E5106E106D8310EE66E48EC57F0E552AA
:105E000012000201C16BC26B12000201C451C42B0B
:105E1000006E140E005C06E34CEC3EF056EC40F0D5
:105E20000201C46BE2C0E6FFE3C0E6FFE4C0E6FFA8
:105E3000E5C0E6FFE6C0E6FFE7C0E6FFEE0EE66E71
:105E4000A30EE66E000EE66E75EC5DF0006E090EB8
:105E5000E15E005060C1E6FF61C1E6FF56C1E6FFAA
:105E600057C1E6FF54C1E6FF55C1E6FF3AC1E6FF60
:105E70003BC1E6FF30C1E6FF31C1E6FF2EC1E6FFC0
:105E80002FC1E6FF14C1E6FF15C1E6FF0AC1E6FF18
:105E90000BC1E6FF08C1E6FF09C1E6FFBF0EE66ED3
:105EA000A30EE66E000EE66E75EC5DF0006E150E4C
:105EB000E15E0050C2C200F0016A00BE016800C08D
:105EC000E6FF01C0E6FFFDC102F0036A02BE0368FF
:105ED00002C0E6FF03C0E6FF62C1E6FF63C1E6FF62
:105EE0003CC1E6FF3DC1E6FF16C1E6FF17C1E6FF74
:105EF0005CC1E6FF5DC1E6FF5EC1E6FF5FC1E6FF94
:105F00005AC1E6FF5BC1E6FF36C1E6FF37C1E6FFD7
:105F100038C1E6FF39C1E6FF34C1E6FF35C1E6FF0F
:105F200010C1E6FF11C1E6FF12C1E6FF13C1E6FF93
:105F30000EC1E6FF0FC1E6FF790EE66EA30EE66E18
:105F4000000EE66E75EC5DF0046E1F0EE15E04500F
:105F50001200D9CFE6FFE1CFD9FF030EE126000EF4
:105F6000E66EE66A360EE66E040EE66EC4EC4DF0A2
:105F7000E552E552E552E552D950010FE96EDACF0C
:105F8000EAFF360EEE6E040EED6E010EDBCFE9FF7A
:105F9000020EDBCFEAFF300EE926000EEA22EECF3A
:105FA00018F1EDCF19F1010EDBCFE9FF020EDBCFC7
:105FB000EAFF320EE926000EEA22EECF1AF1EDCF0B
:105FC0001BF1010EDBCFE9FF020EDBCFEAFF340E3F
:105FD000E926000EEA22EECF1CF1EDCF1DF1010EF5
:105FE000DBCFE9FF020EDBCFEAFF360EE926000E1B
:105FF000EA22EECF1EF1EDCF1FF1010EDBCFE9FF5C
:10600000020EDBCFEAFF320EE926000EEA22EECFC7
:1060100020F1EFCF21F10101D89020372137010E77
:10602000DBCFE9FF020EDBCFEAFF340EE926000EDC
:10603000EA22EECF22F1EFCF23F1030E2303F3CFB9
:1060400023F12203F3CF22F1F45023271C0E246FF7
:10605000250E256F010EDBCFE9FF020EDBCFEAFF35
:10606000380EE926000EEA22EECF3EF1EDCF3FF1E9
:10607000010EDBCFE9FF020EDBCFEAFF3A0EE92685
:10608000000EEA22EECF40F1EDCF41F1010EDBCF61
:10609000E9FF020EDBCFEAFF3C0EE926000EEA2202
:1060A000EECF42F1EDCF43F1010EDBCFE9FF020E5F
:1060B000DBCFEAFF3E0EE926000EEA22EECF44F1E6
:1060C000EDCF45F1010EDBCFE9FF020EDBCFEAFF9A
:1060D0003A0EE926000EEA22EECF46F1EDCF47F167
:1060E000010EDBCFE9FF020EDBCFEAFF3C0EE92613
:1060F000000EEA22EECF48F1EFCF49F10101030E85
:106100004903F3CF49F14803F3CF48F1F45049274D
:10611000680E4A6F420E4B6F010EDBCFE9FF020E95
:10612000DBCFEAFF400EE926000EEA22EECF64F153
:10613000EDCF65F1010EDBCFE9FF020EDBCFEAFF09
:10614000420EE926000EEA22EECF66F1EDCF67F1AE
:10615000010EDBCFE9FF020EDBCFEAFF440EE9269A
:10616000000EEA22EECF68F1EDCF69F1010EDBCF30
:10617000E9FF020EDBCFEAFF460EE926000EEA2217
:10618000EECF6AF1EDCF6BF1010EDBCFE9FF020E2E
:10619000DBCFEAFF420EE926000EEA22EECF6CF1D9
:1061A000EDCF6DF1010EDBCFE9FF020EDBCFEAFF91
:1061B000440EE926000EEA22EECF6EF1EFCF6FF12A
:1061C0000101030E6F03F3CF6FF16E03F3CF6EF196
:1061D000F4506F27800E706F3E0E716FDF6A040EF1
:1061E000DF5C01E377D0010EDBCFE9FF020EDBCFEE
:1061F000EAFF480EE926000EEA22E9CF02F0EACFD4
:1062000003F0DF50020D0250F324E96E0350F42036
:10621000EA6EEECF00F0EFCF01F0EA6ADF34FE0B5A
:10622000EA36E96E260EE926010EEA2200C0EEFFEC
:1062300001C0EDFF010EDBCFE9FF020EDBCFEAFF6D
:10624000500EE926000EEA22E9CF02F0EACF03F071
:10625000DF50020D0250F324E96E0350F420EA6E81
:10626000EECF00F0EFCF01F0EA6ADF34FE0BEA3642
:10627000E96E4C0EE926010EEA2200C0EEFF01C0D5
:10628000EDFF010EDBCFE9FF020EDBCFEAFF580E78
:10629000E926000EEA22E9CF02F0EACF03F0DF5050
:1062A000020D0250F324E96E0350F420EA6EEECFA3
:1062B00000F0EFCF01F0EA6ADF34FE0BEA36E96E58
:1062C000720EE926010EEA2200C0EEFF01C0EDFFCA
:1062D000DF2A85D7030EE15C02E2E16AE552E16E56
:0862E000E552E7CFD9FF1200DF
:0862E800B0EC36F0FB0EDBCF39
:1062F000F3FFDB06F35000090AE0FEEC36F0FA0E7D
:1063000069EC37F0F3E1011CF1E1010E01D0000E60
:10631000DFEF36F0B0EC36F03B0EE12402E3E1684B
:10632000E652E16E010EDB6A020EDB6AF90EDBCF8C
:10633000F6FFFA0EDBCFF7FFFB0EDBCFF8FF08000E
:10634000F550DF6EDF5002E103EF36F0250EDF5C23
:1063500002E0F6EF35F0030EDB6A040EDB6A050E91
:10636000DB6A060EDB6A070EDB6A18EC36F02D0ED0
:10637000DF5C0CE02B0EDF5C09E0200EDF5C06E04A
:10638000230EDF5C03E0300EDF5C1AE1DF50300AE1
:1063900014E0130A0FE0030A0AE00B0A05E0060AFC
:1063A000E4E1030EDB80E1D7030EDB82DED7030ED0
:1063B000DB84DBD7030EDB86D8D7030EDB88D5D78B
:1063C0002A0EDF5C1BE114EC36F062EC36F010E0D4
:1063D000030EDB8020682168130EDBCF25F0140E3E
:1063E000DBCF26F061EC5BF0040E1EC0DBFF03D0B8
:1063F000130E4BEC36F018EC36F00BD0090EDB6ABE
:10640000B9EC36F003E02DEC37F0FAD7090E4BEC7F
:1064100036F0030EDBB0DB982E0EDF5C1BE118ECD0
:1064200036F02A0EDF5C0BE114EC36F062EC36F04D
:1064300003E1130E9DEC36F018EC36F00BD0090E8C
:10644000DB6AB9EC36F003E02DEC37F0FAD7090E31
:106450009DEC36F0680EDF5C07E118EC36F0680E54
:10646000DF5C1DE1030E18D0740EDF5C17E07A0EBE
:10647000DF5C14E0480EDF5C06E0540EDF5C03E0F6
:106480005A0EDF5C02E1020E07D06C0EDF5C03E007
:106490006A0EDF5C04E1010EF0EC36F0C9DBDF5080
:1064A0006E0A01E17FD31E0A01E192D1200A01E1C7
:1064B0008FD13F0A01E149D11A0A01E146D10D0A03
:1064C00001E143D1200A01E140D13A0A01E13DD185
:1064D000200A01E13AD1260A01E135D10D0A01E194
:1064E00032D11A0A01E1D9D0200A4AE0300A1FE06D
:1064F000460A0EE0250A01E083D3D950F90FE96E70
:10650000FF0EDA20EA6E010EEE5E000EEE5AEE5A33
:10651000FEEC36F0250EE66E95DB03E1011C01E191
:1065200069D3FAEC36F001E26BD3DB2A69D3080EAB
:10653000DB6A040EDB50010806E2040EDB04C2EC49
:1065400036F0DB508BDB080EDB5009E0030EDB502E
:10655000010B05E172DB01E04DD3080EDB6A64DB61
:10656000EFCFDFFF72EC37F003E1011C01E142D312
:10657000FAEC36F001E3DB2A60DB01E141D33AD3E8
:10658000070EDB5002080FE13EEC37F0030E05EC7E
:1065900037F00E0EEECFDBFF0F0EEECFDBFF100E4F
:1065A000EECFDBFF20D0F70EDBCF03F0F80EDBCF12
:1065B00004F0020E035E000E045AF70E03C0DBFF68
:1065C000F80E04C0DBFF03C0E9FF04C0EAFFF5ECEE
:1065D00036F0026A0E0E00C0DBFF0F0E01C0DBFFBB
:1065E000100E02C0DBFF0E0EDBCFE6FF0F0EDBCF7F
:1065F000E6FF100EDBCFE6FF46EC5AF0E552E5521F
:10660000E552130E1FC0DBFF140E20C0DBFF060E89
:10661000DB5005E0130E39EC37F001E26ADB5DEC8C
:1066200037F002E2130E37DB20EC37F006E0040E01
:1066300039EC37F002E2050E2EDB030EDBB005D09D
:10664000FCDA01E0D7D2080EDB6A090EDB6A0E0E17
:10665000DBCFF6FF0F0EDBCFF7FF100EDBCFF8FF1F
:106660000800F550DF6EDF5014E063EC37F011E204
:1066700072EC37F003E1011C01E1BCD2BBDB01E3AA
:10668000DB2A090EDB2AD9500E0FE96E000ECBDB98
:10669000E7D7D3DA01E1B4D2ADD2C6DA110EEECF2C
:1066A000DBFF120EEDCFDBFF110EDBCFE6FF120E8C
:1066B000DBCFE6FF38EC5AF0E552E552130EF3CF8C
:1066C000DBFF140EF4CFDBFF060EDB5004E0130EED
:1066D000D0DB01E20EDB5DEC37F002E2130EDBDA19
:1066E000AFDB05E0040EC5DB02E2050ED4DA030ED3
:1066F000DBB005D0A2DA01E07DD2080EDB6A090E1C
:10670000DB6A110EDBCFE9FF120EDBCFEAFFEFCF22
:10671000DFFFDF5014E0D7DB12E2E4DB03E1011C12
:1067200001E168D267DB01E3DB2A090EDB2A110EE7
:10673000DB2ADBCFE9FF120EE8E3DB2AE6D77DDABE
:1067400001E15ED257D2030EDB8E070EDB0410E1AF
:1067500095DB040E5ADB0A0EEECFDBFF0B0EEECFFD
:10676000DBFF0C0EEECFDBFF0D0EEECFDBFF6CD0B0
:10677000070EDB5003082CE1030EDBAE0DD0B2DABE
:10678000020E76DAEFCF00F0016A026A036A00AE09
:1067900039D00168026835D0F70EDBCF01F0F80E72
:1067A000DBCF02F0020E015E000E025AF70E01C0AE
:1067B000DBFFF80E02C0DBFF01C0E9FF02C0EAFF09
:1067C000EFCF00F00A0E00C0DBFF0B0EDB6A38D003
:1067D000070EDB50020809E1030EDBAE04D059DBE3
:1067E00002AE10D00ED055DB0DD0030EDBAE12D0B2
:1067F00079DA020E3DDAF9DA026A036A01AE02D0F2
:1068000002680368E2DA0C0E02C0DBFF0D0E03C063
:10681000DBFF1AD0F70EDBCF02F0F80EDBCF03F070
:10682000020E025E000E035AF70E02C0DBFFF80EE6
:1068300003C0DBFF02C0E9FF03C0EAFFD6DAC5DA16
:106840000C0EDB6A0D0EDB6A060EDB5005E1010E55
:10685000F36E050EF3CFDBFF150EDB6A160EDB6A57
:10686000D950370F006E000EDA20016E390E00C0CD
:10687000DBFF3A0E01C0DBFF380EDB6A080EDB6A75
:106880000A0EAEDADF50780A12E0200A10E0280A79
:106890000CE0200A0AE03F0A06E00D0A02E0200AA6
:1068A00008E1020E05D0080E03D0080EDF26100EF8
:1068B00097DA030EDBBE02D0DB92DB94DB50800B59
:1068C00024E08ADAD890030EEB50000A08E6000EA6
:1068D000EE5C000EEE58000EEE58000EEE5815E27B
:1068E00013DA2368246825682668C0EC5EF00A0E77
:1068F0001AC0DBFF0B0E1BC0DBFF0C0E1CC0DBFF46
:106900000D0E1DC0DBFF2D0E08D0030EDBA202D042
:106910002B0E03D0DBA408D0200EF36E170EF3CF9E
:10692000DBFF150EDB2A02D0170EDB6A050EDB50EB
:1069300003E1B7D901E189D0F20E006EBF0E016EFE
:10694000000E026E070EDBCF03F0046A056A066ACA
:1069500003C023F004C024F005C025F006C026F0D3
:10696000D3D91EEC5FF000501A24F36E01501B20A7
:10697000F46E02501C20F86EF4CFF7FFF3CFF6FF51
:106980000800090EF5CFDBFF580EDF5C0FE1610E4A
:10699000F36E090E7BD90AE3200E006E090EDBCFE1
:1069A000E7FF0050E75E090EE7CFDBFF070EDBCF06
:1069B00000F0016A026A036A0FDA00C023F001C026
:1069C00024F002C025F003C026F0EECF1EF0EECF7B
:1069D0001FF0EECF20F0EFCF21F01EEC5FF021C0D2
:1069E000EDFF20C0EDFF1FC0EDFF1EC0EFFF390E11
:1069F000DBCFE9FFDB063A0EDBCFEAFF01E2DB0685
:106A0000090EDBCFEFFF150EDB2A4BD995E1030E04
:106A1000DBA61DD06F0EDF5C06E1C1D918E3150EB1
:106A2000DB285BDA14D0780EDF5C09E0580EDF5CFF
:106A300006E0620EDF5C03E0420EDF5C08E1020E5E
:106A4000F36E160EF3CFDBFF02D0150EDB6A030EDA
:106A5000DB50100B0EE0040EDBCF00F0050EDB5018
:106A6000D880005406E2060EDB5003E1040EDB5032
:106A700034DA95D90AE2050EDBCFE7FF150EDB50BD
:106A8000E75E050EE7CFDBFF02D0050EDB6A040EE2
:106A9000DBCF00F0160E45D9D880005414E2160E54
:106AA000DBCFE6FF150EDBCFE6FF040EDBCFE6FF04
:106AB000050EDB50E552E75CE552D880E754E5521D
:106AC000D880E7545FD9030EDB50010B0BE1080EB1
:106AD000DB5008E0B2D801E08DD0080EDB50BED804
:106AE000080EDB6A170EDB5007E088D9170EF1D9C4
:106AF00003E1011C01E17ED0160EDB5016E07ED9C9
:106B0000300EE66E9FD802E1011C74E077D9DFCF2A
:106B1000E6FF03EC5EF0E552E552E552F4CF01F0FA
:106B20000001F31C02E1011C65E0050EDBCF00F063
:106B3000160EDB50D880005409E2050EDBCFE7FFCC
:106B4000160EDB50E75E050EE7CFDBFF300EE66E7C
:106B5000050ECBD94FE1390EDB2ADBCFE9FF3A0E28
:106B600001E3DB2ADBCFEAFF090EEFCFDBFFDB50CF
:106B70000EE044D9090EADD902E1011C3BE0390E0B
:106B8000DB2ADBCFE9FF3A0EEDE3DB2AEBD755D862
:106B900031E1160EDBCFE6FF080EC3D8E552E7243D
:106BA0005DD82ED0070EDB50030A1CE0010A14E06A
:106BB000030A07E07BD9DBCFEEFF020EDBCFEDFF50
:106BC0001FD0F5D8056A03AE02D0046805682CD83A
:106BD000BCD805C0EEFF14D0EAD803BE046824D8A0
:106BE000B4D80ED063D9DBCFEFFF0AD07BD905E153
:106BF000011C03E1F368F46810D0FCD801E3DB2A40
:106C000079D99FEF31F0010EDBCF00F0020EDBCF20
:106C100001F000C0F3FF01C0F4FF3B0EE15C02E2B3
:106C2000E16AE552E16ECBD029D9020E05EF37F0CB
:106C300061D90800F550DF6E1200200EE66E080ED6
:106C400075EF37F003EC5EF0E552E552E552F3CF15
:106C500000F0F4CF01F00001F31C1200006E016A95
:106C6000D950010F4DD90050EE260150ED221200EF
:106C7000045E000E055AF70E04C0DBFFF80E05C0D7
:106C8000DBFF04C0E9FF05C0EAFF1200DBCFF4FF21
:106C9000F350F45C1200DB50E76E040EE7CFDBFF2D
:106CA00012000A0EDBCF00F00B0EDBCF01F00C0E52
:106CB000DBCF02F00D0EDBCF03F00050011002100D
:106CC00003101200130EEECFDBFF140EEDCFDBFF2F
:106CD000130EDBCF00F0140EDBCF01F00001800EAD
:106CE00001141200F70EDBCF04F0F80EDBCF05F035
:106CF0001200050EDB50E66ED950130F01D9E55294
:106D0000E750EE6EED6A12000A0EDBCF1EF00B0E9E
:106D1000DBCF1FF00C0EDBCF20F00D0EDBCF21F010
:106D20001200DBCFE6FF150EDBCFE6FF050EDB50D2
:106D3000E552E724E552E7241200DB50CED8010EDD
:106D4000F36E060EF3CFDBFF1200EE50EFCFEAFF3B
:106D5000E96E02C0EEFF03C0EEFF04C0EEFF1200BA
:106D6000D9CFE6FFDACFE6FFE1CFD9FFE2CFDAFFF6
:106D70001200DFCFE6FFE66A0CEC5FF0E552E55269
:106D8000F3501200E76E080EE7CFDBFF1200EECFE4
:106D900000F0EECF01F0EFCF02F0036A1200050E13
:106DA000DBCF00F0150EDB50D88000541200010E2E
:106DB000DBCF02F0020EDBCF03F0046A1200E552D3
:106DC000E5CFDAFFE7CFD9FF12000A0E00C0DBFFE4
:106DD0000B0E01C0DBFF1200D9500A0F80EF37F015
:106DE000F36E070EF3CFDBFF1200EECF00F0EFCF14
:106DF00001F01200010EDB2A020E1200FC0EDBCFA6
:106E0000E6FFFD0EDBCFE6FF1200005E000E015A2A
:106E1000F70E00C0DBFFF80E01C0DBFF00C0E9FF8A
:106E200001C0EAFF1200DA20EA6EEF2AEECFF6FF89
:106E3000000EEF22EECFF7FFEF22EECFF8FF1200A9
:106E4000040EDBCFE6FF130EDB50E552E75C9ADF62
:106E5000DB5004DF060EDB501200090EDB500A0D7A
:106E6000F350DF24D00FE76E090EE7CFDBFF18EFFA
:106E700036F0DB50F36E050E46EF36F0F70EDBCF43
:106E800000F0F80EDBCF01F01200DFCFE6FF22EFBB
:106E900036F028DF030EECDEC7EF36F074EC31F08D
:106EA000E552E552E552E55200091200BDDEEE5012
:106EB000EFCFEAFFE96E010E1200130EDB50F36E06
:106EC000040E46EF36F0040EDB50F36E090E46EF6B
:106ED00036F0DBCFE6FF22EF36F0E76E050EE7CFA8
:106EE000DBFF12008BDF45EF37F0DBCFE6FF86DFFD
:106EF0004EEF37F0D950F90FE96EFF0E13EF37F070
:0A6F0000E96E000EDA20EA6E1200BE
:066F0A00D9CFE6FFE1CF44
:106F1000D9FFE652FEC4E9FFEA6AE9BEEA68F40E68
:106F2000E926040EEA22EFCF00F0016A00BE0168F4
:106F300000C0E6FF01C0E6FFF8EC5EF0E552E55266
:106F4000F350DF6EDF50200A01E115D10D0A01E197
:106F50000ED1070A01E108D1700A01E100D1030A4C
:106F600001E1F8D0010A01E1F0D00F0A01E1E8D017
:106F7000010A01E1E0D0030A01E1D9D0010A01E1EF
:106F8000D1D0070A01E1C9D0010A01E1C1D0030A49
:106F900001E1B9D0010A01E1B1D01F0A01E1AAD093
:106FA000010A01E1A2D0030A01E19AD0010A01E13C
:106FB00093D0070A01E18BD0010A01E184D0030AD2
:106FC00001E17CD0010A75E00F0A6EE0010A67E07A
:106FD000030A60E0010A59E0070A53E0010A4CE0A5
:106FE000030A45E0780A3EE0010A37E00F0A31E083
:106FF000010A2AE0030A23E0010A1CE0070A15E05F
:10700000010A0EE0030A08E0010A01E0B7D0BF0E52
:107010008D6E080E906EB4D0060E8D6E906AB0D054
:107020001B0E8D6E110E906EABD00F0E8D6E010E7D
:10703000906EA6D0260E8D6E110E906EA1D00D0E04
:107040008D6E210E906E9CD03D0E8D6E110E906E49
:1070500097D0070E8D6E906A93D03F0E8D6E110EF5
:10706000906E8ED02F0E8D6E110E906E89D0370ED1
:107070008D6E110E906E84D04F0E8D6E050E906E3B
:107080007FD0390E8D6E906A7BD04F0E8D6E040EC0
:10709000906E76D0390E8D6E110E906E71D0310ECD
:1070A0008D6E100E906E6CD03D0E8D6E010E906E3A
:1070B00067D0360E8D6E110E906E62D0400E8D6EC2
:1070C000040E906E5DD01E0E8D6E906A59D0B00E7B
:1070D0008D6E120E906E54D0380E8D6E906A50D018
:1070E000B60E8D6E200E906E4BD0360E8D6E220E2B
:1070F000906E46D03F0E8D6E906A42D0330E8D6EEC
:10710000110E906E3DD03F0E8D6E020E906E38D0F7
:10711000330E8D6E130E906E33D02D0E8D6E110EBC
:10712000906E2ED0410E8D6E040E906E29D03E0EC4
:107130008D6E906A25D0B00E8D6E080E906E20D0A8
:10714000360E8D6E0A0E906E1BD0800E8D6E2A0E3E
:10715000906E16D0800E8D6E240E906E11D0890E1A
:107160008D6E080E906E0CD08D68906809D08D6A77
:10717000110E906E05D08D6A906A02D08D6A906A69
:10718000810E91160401FE51050A26E0010A19E05C
:10719000070A0DE0010A09E0030A05E0010A01E01F
:1071A0001DD088821BD0888419D0888617D0888803
:1071B000FA0505E1320EFC5D02E1908C01D0909C55
:1071C0000DD0888AFA0505E1320EFC5D02E1908C53
:1071D00001D0909C03D002D0888C00D00401FE51D5
:1071E000FE2B060801E1FE6BE552E552E7CFD9FF21
:1071F0001200D9CFE6FFE1CFD9FF090EE126040145
:10720000FB513D0A6BE0380A5AE0010A49E0070ADF
:1072100038E0010A27E0030A16E0010A05E0DE5221
:10722000200EDD6EDF6E78D0D9CFE6FFDACFE6FF35
:1072300008C1E6FF09C1E6FFDFEC58F0E552E55270
:10724000E552E55269D0D9CFE6FFDACFE6FF2EC18D
:10725000E6FF2FC1E6FFDFEC58F0E552E552E552BC
:10726000E5525AD0D9CFE6FFDACFE6FF54C1E6FFA8
:1072700055C1E6FFDFEC58F0E552E552E552E55224
:107280004BD0D9CFE6FFDACFE6FF0AC1E6FF0BC14C
:10729000E6FFDFEC58F0E552E552E552E5523CD00E
:1072A000D9CFE6FFDACFE6FF30C1E6FF31C1E6FF16
:1072B000DFEC58F0E552E552E552E5522DD0D9CF3A
:1072C000E6FFDACFE6FF56C1E6FF57C1E6FFDFEC87
:1072D00058F0E552E552E552E5521ED0D2C2F6FF13
:1072E000D3C2F7FFD4C2F8FF060EF626000EF7222F
:1072F000F8220800F550DF6ED2C2F6FFD3C2F7FFC6
:10730000D4C2F8FF070EF626000EF722F822080076
:10731000010EF5CFDBFF00D0DFCFF4F4010EDBCFA1
:10732000F5F40401FC513D0A01E176D1010A01E1C5
:1073300062D17A0A01E157D1750A01E179D0010AD7
:1073400001E09DD1070EE6C0DBFF080EE7C0DBFFC2
:10735000B65121E1D950070FE96EDACFEAFF0C0EE2
:10736000256E266AEECF20F0EDCF21F03BEC5BF0EE
:107370001CC0EEFF1DC0EDFFD950070FE96EDACF3C
:10738000EAFFEE50ED1007E10C0EF36E070EF3CF9F
:10739000DBFF080EDB6AD9CFE6FFDACFE6FF070E88
:1073A000DBCFE6FF080EDBCFE6FFDFEC58F0E5525F
:1073B000E552E552E552070EDBCF00F0080EDBCFB9
:1073C00001F0D890015004E60A0E005C000E01584E
:1073D00006E20401200EF66FDFCFF7F405D0DFCF11
:1073E000F6F4010EDBCFF7F4D9CFE6FFDACFE6FFF4
:1073F000E4C0E6FFE5C0E6FFDFEC58F0E552E552F9
:10740000E552E5520A0E0001E5AF02D0D89003D054
:10741000E45D000EE55906E20401300EF86FDFCF9F
:10742000F9F405D0DFCFF8F4010EDBCFF9F427D162
:10743000FB51020A01E188D0070A01E185D0040A64
:1074400045E0050A43E0040A03E0030A01E0BAD07C
:10745000B7510FE1D9CFE6FFDACFE6FFEEC4E6FF82
:10746000EFC4E6FFDFEC58F0E552E552E552E55295
:107470002CD0D9CFE6FFDACFE6FFEEC400F0EFC4A0
:1074800001F0090E0102F3CF01F00002F3CF00F08A
:10749000F4500126050E256E266A00C020F001C0BA
:1074A00021F03BEC5BF020C000F021C001F0200E89
:1074B0000026000E012200C0E6FF01C0E6FFDFEC5F
:1074C00058F0E552E552E552E5527CD0B7510FE154
:1074D000D9CFE6FFDACFE6FFF0C4E6FFF1C4E6FF5E
:1074E000DFEC58F0E552E552E552E5522CD0D9CF09
:1074F000E6FFDACFE6FFF0C400F0F1C401F0090EB8
:107500000102F3CF01F00002F3CF00F0F4500126A6
:10751000050E256E266A00C020F001C021F03BEC6C
:107520005BF020C000F021C001F0200E0026000E0C
:10753000012200C0E6FF01C0E6FFDFEC58F0E55293
:10754000E552E552E5523ED0B7510FE1D9CFE6FF03
:10755000DACFE6FFF2C4E6FFF3C4E6FFDFEC58F053
:10756000E552E552E552E5522CD0D9CFE6FFDACF0D
:10757000E6FFF2C400F0F3C401F0090E0102F3CFFC
:1075800001F00002F3CF00F0F4500126050E256E45
:10759000266A00C020F001C021F03BEC5BF020C067
:1075A00000F021C001F0200E0026000E012200C0D4
:1075B000E6FF01C0E6FFDFEC58F0E552E552E55288
:1075C000E55200D0DFCFF6F4010EDBCFF7F4020E68
:1075D000DBCFF8F40401B75103E1430EF96F02D099
:1075E000460EF96F4CD0450EF66F520EF76FF86FDE
:1075F000FDC1F9F444D0D5C2E6FFD6C2E6FFD7C23A
:10760000E6FFF60EE66E040EE66E1FEC5AF0006E14
:10761000050EE15E005033D0D2C2F6FFD3C2F7FFB1
:10762000D4C2F8FF0800F5CFF6F4D2C2F6FFD3C2F9
:10763000F7FFD4C2F8FFF62A000EF722F82208005E
:10764000F5CFF7F4D2C2F6FFD3C2F7FFD4C2F8FFEA
:10765000030EF626000EF722F8220800F5CFF8F404
:10766000D2C2F6FFD3C2F7FFD4C2F8FF040EF6264B
:10767000000EF722F8220800F5CFF9F400D0090E29
:10768000E15C02E2E16AE552E16EE552E7CFD9FF43
:107690001200D9CFE6FFE1CFD9FFE652DF6ADFCF94
:1076A00000F0080EE76E0018E8AE02D0E73402D012
:1076B000E750005C32E2DFCFE9FFEA6AE9BEEA6840
:1076C000D890E936EA36B80EE926040EEA220AC155
:1076D000EEFF0BC1EDFFDFCFE9FFEA6AE9BEEA6822
:1076E000D890E936EA36C80EE926040EEA2230C1FF
:1076F000EEFF31C1EDFFDFCFE9FFEA6AE9BEEA68DC
:10770000D890E936EA36D80EE926040EEA2256C1A8
:10771000EEFF57C1EDFFDF2AC2D7E552E552E7CFB2
:10772000D9FF1200D9CFE6FFE1CFD9FFE65204011D
:10773000FF51E96EEA6AD890E936EA36B80EE926D2
:10774000040EEA220AC1EEFF0BC1EDFFFF51E96E04
:10775000EA6AD890E936EA36C80EE926040EEA222B
:1077600030C1EEFF31C1EDFFFF51E96EEA6AD890FA
:10777000E936EA36D80EE926040EEA2256C1EEFFB3
:1077800057C1EDFF000EF26FF36BF06FF16BEE6F10
:10779000EF6BDF6A080EDF5C29E2EA6ADF34FE0B7A
:1077A000EA36E96EB80EE926040EEA22EE50EE271C
:1077B000EE50EF23EA6ADF34FE0BEA36E96EC80EBC
:1077C000E926040EEA22EE50F027EE50F123EA6A91
:1077D000DF34FE0BEA36E96ED80EE926040EEA2203
:1077E000EE50F227EE50F323DF2AD4D7050EEE2514
:1077F000EE6F000EEF21EF6F080E256E266AEEC4C5
:1078000020F0EFC421F03BEC5BF020C0EEF421C08F
:10781000EFF4050E0401F025F06F000EF121F16F79
:10782000080E256E266AF0C420F0F1C421F03BEC6E
:107830005BF020C0F0F421C0F1F4050E0401F22544
:10784000F26F000EF321F36F080E256E266AF2C464
:1078500020F0F3C421F03BEC5BF020C0F2F421C037
:10786000F3F40401FF2B070EFF17E552E552E7CFB3
:10787000D9FF12000401B65103E1010EB66F01D029
:10788000B66B12000401B75103E1010EB76F01D0CE
:04789000B76B1200C0
:0C78940082841E0EE66E7AEC5FF0E55276
:1078A000829412008284780EE66E7AEC5FF0E552E4
:1078B000780EE66E7AEC5FF0E55282941200D9CF32
:1078C000E6FFE1CFD9FFFE0EDB50080A39E00F0AD0
:1078D00031E0010A29E0030A21E0010A19E0070A60
:1078E00011E0010A09E0030A01E02BD0010E0201B8
:1078F0009911996F816E25D0020E02019911996F2D
:10790000816E1FD0040E02019911996F816E19D0FA
:10791000080E02019911996F816E13D0100E0201A9
:107920009911996F816E0DD0200E02019911996FF6
:10793000816E07D0400E02019911996F816E01D0BE
:1079400000D0E552E7CFD9FF1200D9CFE6FFE1CF53
:10795000D9FFFE0EDB50080A3CE00F0A34E0010AB2
:107960002CE0030A24E0010A1CE0070A14E0010AE3
:107970000CE0030A04E00201996B816A2BD01E0E11
:1079800002019915996F816E25D0FD0E020199159E
:10799000996F816E1FD0FB0E02019915996F816E50
:1079A00019D0F70E02019915996F816E13D0EF0E61
:1079B00002019915996F816E0DD0DF0E02019915A4
:1079C000996F816E07D0BF0E02019915996F816E74
:1079D00001D000D0E552E7CFD9FF1200D9CFE6FFA2
:1079E000E1CFD9FFFE0EDB5001E04AD00101165174
:1079F000171102E11669176B02019E513DE1E66A1B
:107A0000E66A08C1E6FF0AC1E6FF040EE66EC0ECB6
:107A100046F0006E050EE15E0050E66AE66A08C1B7
:107A2000E6FF0AC1E6FF020EE66E5BEC47F0006E71
:107A3000050EE15E0050E66A56C1E6FF30C1E6FF82
:107A40000AC1E6FFE66A5BEC47F0006E050EE15EF8
:107A5000005028CF2AFF29CF2BFF020180510CE0D4
:107A600002C108F103C109F104C12EF105C12FF1D2
:107A700006C154F107C155F10201010E9E6F00D0FD
:107A8000D5D8E552E7CFD9FF1200D9CFE6FFE1CF35
:107A9000D9FFFE0EDB50020A3CE0030A30E0010A87
:107AA00007E00101166B176B02019E0549E13BD00F
:107AB0000101166B176B02019E051AE1E66AE66A80
:107AC000E66A0AC1E6FF050EE66EC0EC46F0006EFF
:107AD000050EE15E0050E66AE66AE66A0AC1E6FF64
:107AE000030EE66E5BEC47F0006E050EE15E0050A3
:107AF00002019E6B010EE66E28DFE5523AD00101CD
:107B00003C6B3D6B02019F6B020EE66E1EDFE55281
:107B100030D00101626B636B0201A06B030EE66E55
:107B200014DFE55226D0E66AE66AE66A010EE66EE2
:107B3000030EE66E5BEC47F0006E050EE15E005052
:107B400002019E6B010EE66E00DFE55201013C6B07
:107B50003D6B02019F6B020EE66EF7DEE5520101FE
:107B6000626B636B0201A06B030EE66EEEDEE55204
:107B700000D002019E5108E102019F5105E102017E
:107B8000A05102E155D858D8E552E7CFD9FF1200ED
:107B900001EC2FF0E66A22DFE5520AC112F10BC1B7
:107BA00013F10101140E125F000E135B260E130376
:107BB000F3CF13F1020E1203F3501327260E120314
:107BC000F3CF12F1F4501327800E131502E0126B5D
:107BD000136B0201A8510DE0A80EE66EA60EE66E2C
:107BE000000EE66E75EC5DF0E552E552E55205ECEF
:107BF0002FF01200E66A49DFE552010EE66E45DF1E
:107C0000E552020EE66E41DFE5520201A8510DE099
:107C1000980EE66EA60EE66E000EE66E75EC5DF052
:107C2000E552E552E55205EC2FF012008B80120070
:107C30008B9012008880120088901200D9CFE6FF46
:107C4000E1CFD9FF82B205D0010EF36EF46A04D001
:107C500003D0F36AF46A00D0E552E7CFD9FF1200EF
:107C6000D9CFE6FFE1CFD9FFE652C00EF214DF6EA6
:107C7000F29CF29EDF5000D0E552E552E7CFD9FFEB
:107C80001200D9CFE6FFE1CFD9FFFE0EDB50F21292
:107C9000E552E7CFD9FF1200930EE66EA60EE66E10
:107CA000000EE66E75EC5DF0E552E552E5520C0E05
:107CB0000001EC1901E1ED5101E1C0D00B0EEC190E
:107CC00001E1ED5101E1AED00A0EEC1901E1ED51F7
:107CD00001E19CD0090EEC1901E1ED5101E18AD0DE
:107CE000080EEC1901E1ED5101E178D0070EEC1915
:107CF00001E1ED5167E0060EEC1901E1ED5156E0AE
:107D0000050EEC1901E1ED5145E0040EEC1901E11D
:107D1000ED5134E0030EEC1901E1ED5123E0020EC8
:107D2000EC1901E1ED5112E0010EEC1901E1ED5108
:107D300001E090D08A0EE66EA60EE66E000EE66EAC
:107D400075EC5DF0E552E552E55284D0800EE66EAA
:107D5000A60EE66E000EE66E75EC5DF0E552E5529D
:107D6000E55278D0790EE66EA60EE66E000EE66E4F
:107D700075EC5DF0E552E552E5526CD0720EE66EA0
:107D8000A60EE66E000EE66E75EC5DF0E552E5526D
:107D9000E55260D06D0EE66EA60EE66E000EE66E43
:107DA00075EC5DF0E552E552E55254D0670EE66E93
:107DB000A60EE66E000EE66E75EC5DF0E552E5523D
:107DC000E55248D0610EE66EA60EE66E000EE66E37
:107DD00075EC5DF0E552E552E5523CD0590EE66E89
:107DE000A60EE66E000EE66E75EC5DF0E552E5520D
:107DF000E55230D04E0EE66EA60EE66E000EE66E32
:107E000075EC5DF0E552E552E55224D0450EE66E84
:107E1000A60EE66E000EE66E75EC5DF0E552E552DC
:107E2000E55218D03B0EE66EA60EE66E000EE66E2C
:107E300075EC5DF0E552E552E5520CD0310EE66E80
:107E4000A60EE66E000EE66E75EC5DF0E552E552AC
:107E5000E55200D0EAC0E6FFEBC0E6FF2B0EE66E6F
:107E6000A60EE66E000EE66E75EC5DF0006E050E79
:107E7000E15E0050EEC0E6FFEFC0E6FF220EE66EC8
:107E8000A60EE66E000EE66E75EC5DF0006E050E59
:107E9000E15E0050070E0001E81901E1E95167E0D9
:107EA000060EE81901E1E95156E0050EE81901E175
:107EB000E95145E0040EE81901E1E95134E0030E0F
:107EC000E81901E1E95123E0020EE81901E1E95165
:107ED00012E0010EE81901E1E95101E054D01A0E57
:107EE000E66EA60EE66E000EE66E75EC5DF0E552EF
:107EF000E552E55248D0120EE66EA60EE66E000E72
:107F0000E66E75EC5DF0E552E552E5523CD0090EA7
:107F1000E66EA60EE66E000EE66E75EC5DF0E552BE
:107F2000E552E55230D0FE0EE66EA50EE66E000E6E
:107F3000E66E75EC5DF0E552E552E55224D0F40EA4
:107F4000E66EA50EE66E000EE66E75EC5DF0E5528F
:107F5000E552E55218D0EC0EE66EA50EE66E000E68
:107F6000E66E75EC5DF0E552E552E5520CD0E20E9E
:107F7000E66EA50EE66E000EE66E75EC5DF0E5525F
:107F8000E552E55200D00001E73504E2E6510C0865
:107F9000000EE75544E2E6C000F0E7C001F00C0E29
:107FA000005E000E015A00C0E6FF01C0E6FFDD0ED4
:107FB000E66EA50EE66E000EE66E75EC5DF0026EE6
:107FC000050EE15E0250E4C0E6FFE5C0E6FFD70E15
:107FD000E66EA50EE66E000EE66E75EC5DF0006EC8
:107FE000050EE15E0050E2C0E6FFE3C0E6FFD10E01
:107FF000E66EA50EE66E000EE66E75EC5DF0006EA8
:10800000050EE15E0050CB0EE66EA50EE66E000E8C
:10801000E66E75EC5DF0E552E552E5523BD0E6C008
:10802000E6FFE7C0E6FFDD0EE66EA50EE66E000E8B
:10803000E66E75EC5DF0006E050EE15E0050E4C08A
:10804000E6FFE5C0E6FFD70EE66EA50EE66E000E73
:10805000E66E75EC5DF0006E050EE15E0050E2C06C
:10806000E6FFE3C0E6FFD10EE66EA50EE66E000E5B
:10807000E66E75EC5DF0006E050EE15E0050C50E1B
:10808000E66EA50EE66E000EE66E75EC5DF0E5524E
:10809000E552E552C20EE66EA50EE66E000EE66EE5
:1080A00075EC5DF0E552E552E55212003C0EE66ECD
:1080B000A50EE66E000EE66E75EC5DF0E552E5523B
:1080C000E552B70EE66EA40EE66E000EE66E75EC97
:0A80D0005DF0E552E552E5521200A2
:0680DA00D9CFE6FFE1CF63
:1080E000D9FF020EE126DF6A010EDB6AC750040BDE
:1080F00001E0010E006E1F0EC514001001E0F6D75E
:10810000C580C5B0FED7C5B0FED7D00EE66E45EC33
:108110005EF0E552C750040B01E0010E006E1F0E29
:10812000C514001001E0F6D7E66A45EC5EF0E552B2
:10813000C750040B01E0010E006E1F0EC5140010A5
:1081400001E0F6D7C582C5B2FED7C5B2FED7D10EC3
:10815000E66E45EC5EF0E552C750040B01E0010EFF
:10816000006E1F0EC514001001E0F6D7080EE66E73
:10817000F20EE66E000EE66E85EC5EF0E552E5521C
:10818000E552C58AC588C5B8FED7C5B8FED7C5842F
:10819000C5B4FED7C5B4FED7700E0001F215E8389D
:1081A0000F0BDF6E0F0EF215E76E010EE7CFDBFF50
:1081B000DBCFE6FF0A0EDF02F350E552E724E26F61
:1081C000E36B800B01E0E3690F013D510001E4190D
:1081D00004E10F013E510001E51920E00F012A07DB
:1081E000000E2B5B2B3504E22A510008000E2B55A4
:1081F00015E328CF2AFF29CF2BFF02019E050EE1B0
:10820000E66A56C1E6FF30C1E6FF0AC1E6FFE66A4C
:108210005BEC47F0006E050EE15E0050E4C03DFFF0
:10822000E5C03EFF700E0001F315E8380F0BDF6E5E
:108230000F0EF315E76E010EE7CFDBFFDBCFE6FF96
:108240000A0EDF02F350E552E724E46FE56B800B82
:1082500001E0E569300EF415E8380F0BDF6E0F0E04
:10826000F415E76E010EE7CFDBFFDBCFE6FF0A0E6A
:10827000DF02F350E552E724E66FE76B800B01E085
:10828000E769070EF515E86FE96B300EF615E8386B
:108290000F0BDF6E0F0EF615E76E010EE7CFDBFF5B
:1082A000DBCFE6FF0A0EDF02F350E552E724EA6F68
:1082B000EB6B800B01E0EB69100EF715E8380F0B44
:1082C000DF6E0F0EF715E76E010EE7CFDBFFDBCF9A
:1082D000E6FF0A0EDF02F350E552E724EC6FED6B88
:1082E000800B01E0ED69F8390F0BDF6E0F0EF8150A
:1082F000E76E010EE7CFDBFFDBCFE6FF0A0EDF0202
:10830000F350E552E724EE6FEF6B800B01E0EF696D
:10831000F951F06FF16B020EE15C02E2E16AE552A5
:10832000E16EE552E7CFD9FF1200D9CFE6FFE1CFEA
:10833000D9FF090EE1260A0E0001E3AF02D0D89062
:1083400003D0E25D000EE35904E2030EE2C0DBFF5E
:108350001BD0D9CFE6FFDACFE6FFE2C0E6FFE3C0ED
:10836000E6FFDFEC58F0E552E552E552E552010E2A
:10837000DB50D00F006E300EDF5C100DF350002488
:10838000E76E030EE7CFDBFF0A0E0001E5AF02D078
:10839000D89003D0E45D000EE55904E2040EE4C079
:1083A000DBFF1BD0D9CFE6FFDACFE6FFE4C0E6FF64
:1083B000E5C0E6FFDFEC58F0E552E552E552E55244
:1083C000010EDB50D00F006E300EDF5C100DF3504D
:1083D0000024E76E040EE7CFDBFF0A0E0001E7AFD3
:1083E00002D0D89003D0E65D000EE75904E2050EF6
:1083F000E6C0DBFF1BD0D9CFE6FFDACFE6FFE6C051
:10840000E6FFE7C0E6FFDFEC58F0E552E552E55243
:10841000E552010EDB50D00F006E300EDF5C100D08
:10842000F3500024E76E050EE7CFDBFF0A0E0001D4
:10843000EBAF02D0D89003D0EA5D000EEB5904E216
:10844000060EEAC0DBFF1BD0D9CFE6FFDACFE6FF8E
:10845000EAC0E6FFEBC0E6FFDFEC58F0E552E5527C
:10846000E552E552010EDB50D00F006E300EDF5C9E
:10847000100DF3500024E76E060EE7CFDBFF0A0E67
:108480000001EDAF02D0D89003D0EC5D000EED59A5
:1084900004E2070EECC0DBFF1BD0D9CFE6FFDACF3A
:1084A000E6FFECC0E6FFEDC0E6FFDFEC58F0E5527A
:1084B000E552E552E552010EDB50D00F006E300E52
:1084C000DF5C100DF3500024E76E070EE7CFDBFFF3
:1084D0000A0E0001EFAF02D0D89003D0EE5D000E7F
:1084E000EF5904E2080EEEC0DBFF1BD0D9CFE6FF48
:1084F000DACFE6FFEEC0E6FFEFC0E6FFDFEC58F0B4
:10850000E552E552E552E552010EDB50D00F006E08
:10851000300EDF5C100DF3500024E76E080EE7CF3D
:10852000DBFFC750040B01E0010E006E1F0EC514E7
:10853000001001E0F6D7C580C5B0FED7C5B0FED7A4
:10854000D00EE66E45EC5EF0E552C750040B01E03C
:10855000010E006E1F0EC514001001E0F6D7E66A8A
:1085600045EC5EF0E552C750040B01E0010E006ED1
:108570001F0EC514001001E0F6D7030EDBCFE6FF97
:1085800045EC5EF0E552C750040B01E0010E006EB1
:108590001F0EC514001001E0F6D7040EDBCFE6FF76
:1085A00045EC5EF0E552C750040B01E0010E006E91
:1085B0001F0EC514001001E0F6D7050EDBCFE6FF55
:1085C00045EC5EF0E552C750040B01E0010E006E71
:1085D0001F0EC514001001E0F6D7E8C0E6FF45EC19
:1085E0005EF0E552C750040B01E0010E006E1F0E55
:1085F000C514001001E0F6D7060EDBCFE6FF45EC10
:108600005EF0E552C750040B01E0010E006E1F0E34
:10861000C514001001E0F6D7070EDBCFE6FF45ECEE
:108620005EF0E552C750040B01E0010E006E1F0E14
:10863000C514001001E0F6D7080EDBCFE6FF45ECCD
:108640005EF0E552C750040B01E0010E006E1F0EF4
:10865000C514001001E0F6D7C584C5B4FED7C5B473
:10866000FED7090EE15C02E2E16AE552E16EE552F5
:10867000E7CFD9FF1200D9CFE6FFE1CFD9FFC7502E
:10868000040B01E0010E006E1F0EC514001001E086
:10869000F6D7C580C5B0FED7C5B0FED7D00EE66E02
:1086A00045EC5EF0E552C750040B01E0010E006E90
:1086B0001F0EC514001001E0F6D7070EE66E45EC5C
:1086C0005EF0E552C750040B01E0010E006E1F0E74
:1086D000C514001001E0F6D7400E0001F011E66E5F
:1086E00045EC5EF0E552C750040B01E0010E006E50
:1086F0001F0EC514001001E0F6D7C584C5B4FED71F
:10870000C5B4FED7E552E7CFD9FF1200D9CFE6FFB7
:10871000E1CFD9FFC750040B01E0010E006E1F0E20
:10872000C514001001E0F6D7C580C5B0FED7C5B0AE
:10873000FED7D00EE66E45EC5EF0E552C750040B56
:1087400001E0010E006E1F0EC514001001E0F6D707
:10875000070EE66E45EC5EF0E552C750040B01E0F3
:10876000010E006E1F0EC514001001E0F6D7DF0EDB
:108770000001F015E66E45EC5EF0E552C750040BC3
:1087800001E0010E006E1F0EC514001001E0F6D7C7
:10879000C584C5B4FED7C5B4FED7E552E7CFD9FF2F
:1087A0001200D9CFE6FFE1CFD9FFC750040B01E09B
:1087B000010E006E1F0EC514001001E0F6D7C58033
:1087C000C5B0FED7C5B0FED7D00EE66E45EC5EF064
:1087D000E552C750040B01E0010E006E1F0EC514D8
:1087E000001001E0F6D7070EE66E45EC5EF0E552AC
:1087F000C750040B01E0010E006E1F0EC5140010DF
:1088000001E0F6D7F0C0E6FF45EC5EF0E552C75058
:10881000040B01E0010E006E1F0EC514001001E0F4
:10882000F6D7C584C5B4FED7C5B4FED7E552E7CFA9
:10883000D9FF12000001E42B000EE523E53504E228
:10884000E4513B08000EE55502E2E46BE56B95EF61
:1088500041F00001E62B000EE723E73504E2E65184
:108860001708000EE75502E2E66BE76B95EF41F063
:10887000D9CFE6FFE1CFD9FF080EE126010EF36E56
:10888000050EF3CFDBFF040EDB6A080EDE6EDD6A39
:10889000DECF00F0DDCF01F0100E005C000E0158BD
:1088A00001E378D0DECFE6FFDDCFE6FF360EE66EE1
:1088B000040EE66EC4EC4DF0E552E552E552E55289
:1088C000020EDB6A030EDB6A020EDBCF00F0030E42
:1088D000DBCF01F0780E005C000E015852E2020E70
:1088E000DBCF00F0030EDBCF01F0360E0026040EC6
:1088F0000122060E00C0DBFF070E01C0DBFF060EE3
:10890000DBCFE9FF070EDBCFEAFFEF50FF0806E100
:10891000010EF36E040EF3CFDBFF33D0050EDB50F8
:1089200011E0060EDBCFE9FF070EDBCFEAFF030EF7
:10893000E926000EEA22EF50800B0F01306F050E82
:10894000DB6A15D0060EDBCFE9FF070EDBCFEAFFAF
:10895000030EE926000EEA22EF50800B0F01305D76
:1089600006E0010EF36E040EF3CFDBFF0AD0D95000
:10897000020FE96EDACFEAFF0A0EEE26000EED22B4
:10898000A3D7040EDB5001E005D0DF2A010E01E37E
:10899000DB2A7ED7040EDB500BE0DECF2CFFDDCFD1
:1089A0002DFF020EDBCF2EFF030EDBCF2FFF02D0F9
:1089B0000F01307F010EF36E050EF3CFDBFF040EC7
:1089C000DB6A100EDE6EDD6ADECF00F0DDCF01F077
:1089D000200E005C000E015801E378D0DECFE6FFE8
:1089E000DDCFE6FF360EE66E040EE66EC4EC4DF00B
:1089F000E552E552E552E552020EDB6A030EDB6AF0
:108A0000020EDBCF00F0030EDBCF01F0780E005C2E
:108A1000000E015852E2020EDBCF00F0030EDBCF56
:108A200001F0360E0026040E0122060E00C0DBFF08
:108A3000070E01C0DBFF060EDBCFE9FF070EDBCF21
:108A4000EAFFEF50FF0806E1010EF36E040EF3CFCC
:108A5000DBFF33D0050EDB5011E0060EDBCFE9FF64
:108A6000070EDBCFEAFF030EE926000EEA22EF50E5
:108A7000800B0F01356F050EDB6A15D0060EDBCFBC
:108A8000E9FF070EDBCFEAFF030EE926000EEA221C
:108A9000EF50800B0F01355D06E0010EF36E040E02
:108AA000F3CFDBFF0AD0D950020FE96EDACFEAFF2D
:108AB0000A0EEE26000EED22A3D7040EDB5001E0D5
:108AC00005D0DF2A010E01E3DB2A7ED7040EDB503E
:108AD0000BE0DECF31FFDDCF32FF020EDBCF33FF05
:108AE000030EDBCF34FF02D00F01357F010EF36E92
:108AF000050EF3CFDBFF040EDB6A200EDE6EDD6AAF
:108B0000D9CFE9FFDACFEAFFFF0ED880EE54010E8D
:108B1000ED5401E278D0DECFE6FFDDCFE6FF360E82
:108B2000E66E040EE66EC4EC4DF0E552E552E552F9
:108B3000E552020EDB6A030EDB6A020EDBCF00F0A9
:108B4000030EDBCF01F0780E005C000E015852E2FC
:108B5000020EDBCF00F0030EDBCF01F0360E002655
:108B6000040E0122060E00C0DBFF070E01C0DBFF72
:108B7000060EDBCFE9FF070EDBCFEAFFEF50FF0861
:108B800006E1010EF36E040EF3CFDBFF33D0050ECA
:108B9000DB5011E0060EDBCFE9FF070EDBCFEAFF6B
:108BA000030EE926000EEA22EF50800B0F013A6F08
:108BB000050EDB6A15D0060EDBCFE9FF070EDBCF13
:108BC000EAFF030EE926000EEA22EF50800B0F01A8
:108BD0003A5D06E0010EF36E040EF3CFDBFF0AD020
:108BE000D950020FE96EDACFEAFF0A0EEE26000E28
:108BF000ED22A3D7040EDB5001E005D0DF2A010EE1
:108C000001E3DB2A7DD7040EDB500BE0DECF36FF1D
:108C1000DDCF37FF020EDBCF38FF030EDBCF39FF8E
:108C200002D00F013A7F080EE15C02E2E16AE552F0
:108C3000E16EE552E7CFD9FF1200D9CFE6FFE1CFD1
:108C4000D9FFFE0EDBCFB4F2E2C0B5F2E4C0B6F25B
:108C500030CF00F0016A00BE01680001E65100104B
:108C60000201B76FEAC0B8F2ECC0B9F2FD0EDBCF7B
:108C7000BAF2FC0EDBCFBBF2FB0EDBCFBCF2FA0E7E
:108C8000DBCFBDF20A0EE66EE66A2ECFE6FF2FCFEF
:108C9000E6FF2CCFE6FF2DCFE6FFB40EE66E020E08
:108CA000E66E46EC4CF0006E080EE15E0050060EDB
:108CB000E66ED3EC5FF0E5520A0E0F012E27000E90
:108CC0002F230A0E016A2E25006E2F510122800EDD
:108CD000005C000E01580EE32E6B2F6B2C2B000E48
:108CE0002D23100E2C5D000E2D5904E3080E2C6F61
:108CF0002D6B307FE552E7CFD9FF1200D9CFE6FFC9
:108D0000E1CFD9FF020EE126080EDE6EDD6ADECF6E
:108D100000F0DDCF01F0100E005C000E015814E2EF
:108D2000DECFE6FFDDCFE6FFE66810EC4DF0E55262
:108D3000E552E552060EE66ED3EC5FF0E552DF2A0F
:108D4000010E01E3DB2AE3D7080E0F012C6F2D6B18
:108D50002E6B2F6BE66AE66AE66A030EE66E090E74
:108D6000E66E0ED8006E050EE15E0050020EE15C6C
:108D700002E2E16AE552E16EE552E7CFD9FF120067
:108D8000D9CFE6FFE1CFD9FFFE0EDBCFB4F2E2C0D0
:108D9000B5F2E4C0B6F2E6C0B7F2EAC0B8F2ECC091
:108DA000B9F2FD0EDBCFBAF2FC0EDBCFBBF2FB0E4D
:108DB000DBCFBCF2FA0EDBCFBDF20A0EE66EE66A3E
:108DC00033CFE6FF34CFE6FF31CFE6FF32CFE6FF09
:108DD000B40EE66E020EE66E46EC4CF0006E080E27
:108DE000E15E0050060EE66ED3EC5FF0E5520A0E2F
:108DF0000F013327000E34230A0E016A3325006E5B
:108E000034510122800E005C000E01580EE3336BDA
:108E1000346B312B000E3223200E315D000E32599F
:108E200004E3100E316F326B357FE552E7CFD9FF87
:108E30001200D9CFE6FFE1CFD9FF020EE126100ED6
:108E4000DE6EDD6ADECF00F0DDCF01F0200E005CCB
:108E5000000E015814E2DECFE6FFDDCFE6FFE66844
:108E600010EC4DF0E552E552E552060EE66ED3ECFD
:108E70005FF0E552DF2A010E01E3DB2AE3D7100E93
:108E80000F01316F326B336B346BE66AE66AE66A68
:108E9000020EE66E090EE66E73DF006E050EE15EF1
:108EA0000050020EE15C02E2E16AE552E16EE55239
:108EB000E7CFD9FF1200D9CFE6FFE1CFD9FF0201FA
:108EC000805101E157D00F012851291101E152D001
:108ED000FE0EDBCFB4F2E2C0B5F2E4C0B6F2E6C0FB
:108EE000B7F2EAC0B8F2ECC0B9F2FD0EDBCFBAF2CD
:108EF000FC0EDBCFBBF2FB0EDBCFBCF2FA0EDBCFFE
:108F0000BDF20A0EE66EE66A38CFE6FF39CFE6FF1D
:108F100036CFE6FF37CFE6FFB40EE66E020EE66E02
:108F200046EC4CF0006E080EE15E0050060EE66E58
:108F3000D3EC5FF0E5520A0E0F013827000E3923FB
:108F40000A0E016A3825006E39510122800E005C3C
:108F5000000E01580FE3386B396B362B000E3723A8
:108F6000FF0ED8803655010E375504E2200E366FBD
:108F7000376B3A7FE552E7CFD9FF1200D9CFE6FF32
:108F8000E1CFD9FF020EE126200EDE6EDD6AD9CFD9
:108F9000E9FFDACFEAFFFF0ED880EE54010EED5460
:108FA00014E3DECFE6FFDDCFE6FFE66810EC4DF020
:108FB000E552E552E552060EE66ED3EC5FF0E5525F
:108FC000DF2A010E01E3DB2AE2D7200E0F01366F04
:108FD000376B386B396BE66AE66AE66A010EE66E55
:108FE000090EE66ECDDE006E050EE15E0050020E4B
:108FF000E15C02E2E16AE552E16EE552E7CFD9FFBA
:0290000012005C
:0E900200D9CFE6FFE1CFD9FF020EE126000034
:1090100000000000D0CF00F1FCCF01F1D082D08061
:10902000D08AD088FC9EFC9C91EC53F0000000009C
:109030002FEC56F0F9EC38F00201C75104E00201C0
:10904000C76BC5EC54F00201C85104E00201C86BC3
:109050006DEC40F00201C05101E122D10201C06B70
:1090600058D9E66A88EC2AF0E552010EE66E45EC26
:109070003DF0E552020EE66E45EC3DF0E552020190
:109080009E0559E1080EE66E010EE66EB1EC2BF07E
:10909000E552E552E66AFBEC2DF0E5529DEC2EF030
:1090A00001010A510101081904E101010B510101FB
:1090B000091905E00201A12B000EA22303D0020131
:1090C000A16BA26B040E206E216A08C125F009C1B4
:1090D00026F061EC5BF01EC000F01FC001F0020141
:1090E000A2510118E8AE02D0013404D00050A15DB5
:1090F0000150A25912E30101153504E2145105088B
:10910000000E155507E2350EE66E48EC57F0E552B5
:10911000F0D803D00201A16BA26B01010B3504E270
:109120000A513E08000E0B5506E2390EE66E48EC79
:1091300057F0E552DED802019F0552E12E0EE66E91
:10914000010EE66EB1EC2BF0E552E552010EE66E33
:10915000FBEC2DF0E5520101313504E230514708B6
:10916000000E315506E2410EE66E48EC57F0E5522E
:10917000C0D80101305101012E1904E10101315122
:1091800001012F1905E00201A32B000EA42303D037
:109190000201A36BA46B500E0201A4AF02D0D890C1
:1091A00003D0A35D000EA4591BE301013B3504E28B
:1091B0003A510508000E3B5509E30101D8803B51A7
:1091C00004E7F60E3A5DFF0E3B5907E2360EE66EF7
:1091D00048EC57F0E5528DD803D00201A36BA46B85
:1091E0000201A00552E1540EE66E010EE66EB1ECEE
:1091F0002BF0E552E552020EE66EFBEC2DF0E55247
:109200000101573504E256514508000E575506E254
:10921000430EE66E48EC57F0E5526BD8010156510B
:109220000101541904E1010157510101551905E0EB
:109230000201A52B000EA62303D00201A56BA66B8D
:10924000500E0201A6AF02D0D89003D0A55D000E4B
:10925000A6591BE30101613504E260510508000EC7
:10926000615509E30101D880615104E7F40E605DA6
:10927000FF0E615907E2370EE66E48EC57F0E552F3
:1092800038D803D00201A56BA66B0201A85102E0F9
:1092900005EC2FF092EC3BF00101FD5101E029D8E3
:1092A00073EC2EF00101FD5119E0E66A45EC3DF04A
:1092B000E552010EE66E45EC3DF0E552020EE66E1B
:1092C00045EC3DF0E5520201A16BA26B0201A36BDC
:1092D000A46B0201A56BA66B01EC2FF0A9D6020EC0
:1092E000E15C02E2E16AE552E16EE552E7CFD9FFC7
:1092F000120052EC3CF05A0EE66E7AEC5FF0E5524A
:1093000052EC3CF05A0EE66E7AEC5FF0E55252EF0A
:109310003CF0D9CFE6FFE1CFD9FF020EE126010EE6
:10932000E66EE66A7A0EE66E010EE66EC4EC4DF06D
:10933000E552E552E552E5527A0EDE6E010EDD6E23
:10934000DECFE9FFDDCFEAFF1C0EE926000EEA22A0
:10935000EFCFFAF10101FA5103E00201805103E17C
:109360000201A96B17D020D801080BE10201A95115
:1093700007E19E5102E1C8EC3DF00201010EA96F28
:1093800009D00201A90506E19E0502E1FAEC3DF0D3
:109390000201A96B020EE15C02E2E16AE552E16EB4
:1093A000E552E7CFD9FF1200D9CFE6FFE1CFD9FFD1
:1093B0000E0EE126D9500A0FE96EDACFEAFF7A0ED7
:1093C000EE6E010EED6EE8C000F0E9C001F000069F
:1093D000000E015A00C0DEFF01C0DDFFE6C003F051
:1093E000026A02500001E411006E0350E511016EA3
:1093F000040E00C0DBFF050E01C0DBFF0C0EDB6AB4
:109400000A0EDBCFE9FF0B0EDBCFEAFFE9CF00F05E
:10941000EACF01F0020E206E216ADECF25F0DDCF0B
:1094200026F061EC5BF000501E24E96E01501F2015
:10943000EA6E060EEECFDBFF070EEDCFDBFF0A0E66
:10944000DBCFE9FF0B0EDBCFEAFF0E0EE926000EA5
:10945000EA22E9CF00F0EACF01F0020E206E216A85
:10946000DECF25F0DDCF26F061EC5BF000501E244E
:10947000E96E01501F20EA6E080EEECFDBFF090EE9
:10948000EDCFDBFF060EDBCF00F0070EDBCF01F0E8
:10949000080EDB50001803E1090EDB50011801E152
:1094A0007DD0040EDBCF00F0050EDBCF01F0060E01
:1094B000DBCF02F0070EDBCF03F001500318E8AE5C
:1094C00002D0033404D00250005C0350015833E34F
:1094D000040EDBCF04F0050EDBCF05F0080EDBCF6A
:1094E00006F0090EDBCF07F005500718E8AE02D0F2
:1094F000073404D00650045C075005581CE3080EDE
:10950000DBCF00F0090EDBCF01F0060EDBCF02F05F
:10951000070EDBCF03F003500118E8AE02D0013490
:1095200004D00050025C0150035803E2000EE0D06A
:1095300035D0010EDDD0040EDBCF00F0050EDBCF01
:1095400001F0060EDBCF02F0070EDBCF03F0015077
:109550000318E8AE02D0033404D00250005C03507C
:10956000015803E3010EC4D019D0040EDBCF00F084
:10957000050EDBCF01F0080EDBCF02F0090EDBCFCA
:1095800003F001500318E8AE02D0033404D00250B7
:10959000005C0350015802E3000EAAD0010EF36EE6
:1095A0000D0EF3CFDBFFDBCF00F0070EE76E0018E8
:1095B000E8AE02D0E73402D0E750005C01E396D079
:1095C0000D0EDBCF02F0036A02BE03680250DE5CC0
:1095D000006E0350DD58016E020E00C0DBFF030E6B
:1095E00001C0DBFF020EDBCF00F0030EDBCF01F08A
:1095F0000001800E011409E0D950020FE96EDACFA4
:10960000EAFF070EEE26000EED220A0EDBCFE9FF81
:109610000B0EDBCFEAFFE9CF00F0EACF01F0020E3C
:10962000206E216ADBCF25F0030EDBCF26F061EC44
:109630005BF000501E24E96E01501F20EA6E060EFA
:10964000EECFDBFF070EEDCFDBFF0A0EDBCFE9FF2E
:109650000B0EDBCFEAFF0E0EE926000EEA22E9CF61
:1096600000F0EACF01F0020E206E216ADBCF25F078
:10967000030EDBCF26F061EC5BF000501E24E96E98
:1096800001501F20EA6E080EEECFDBFF090EEDCF72
:10969000DBFF060EDBCF00F0070EDBCF01F0080E7C
:1096A000DB50001803E1090EDB5001181CE0080E26
:1096B000DBCF00F0090EDBCF01F0060EDBCF02F0AE
:1096C000070EDBCF03F003500118E8AE02D00134DF
:1096D00004D00050025C0150035803E2000E08D091
:1096E00002D0010E05D00D0EDB2A5DD7000E00D092
:1096F000006E0E0EE15C02E2E16AE552E16E00509E
:08970000E552E7CFD9FF12008A
:08970800D9CFE6FFE1CFD9FF44
:10971000060EE126DE6ADD6A800E206E216AFB0EEF
:10972000DBCF25F0FC0EDBCF26F08EEC5BF0040ED9
:109730001EC0DBFF050E1FC0DBFFFF0EE76E040E31
:10974000DBCF00F0050EDBCF01F0E7500016016A19
:10975000030E00C0DBFF040EDBCF00F0050EDBCFF5
:1097600001F001C000F0016A020E00C0DBFFC7502B
:10977000040B01E0010E006E1F0EC514001001E085
:10978000F6D7C580C5B0FED7C5B0FED7AE0EE66E23
:1097900045EC5EF0E552C750040B01E0010E006E8F
:1097A0001F0EC514001001E0F6D7020EDBCFE6FF56
:1097B00045EC5EF0E552C750040B01E0010E006E6F
:1097C0001F0EC514001001E0F6D7030EDBCFE6FF35
:1097D00045EC5EF0E552C750040B01E0010E006E4F
:1097E0001F0EC514001001E0F6D7DE6ADD6ADECF79
:1097F00000F0DDCF01F0800E005C000E015824E285
:10980000FD0EDBCF00F0FE0EDBCF01F0DE500024BA
:10981000E96EDD500120EA6EEF50E66E45EC5EF039
:10982000E552C750040B01E0010E006E1F0EC51477
:10983000001001E0F6D7C5AC02D0FE0E1BD0DF2A27
:10984000010E01E3DB2AD3D7C750040B01E0010E60
:10985000006E1F0EC514001001E0F6D7C584C5B414
:10986000FED7C5B4FED7060EE66E7AEC5FF0E55281
:10987000000E00D0006E060EE15C02E2E16AE552E5
:10988000E16E0050E552E7CFD9FF1200D9CFE6FFD5
:10989000E1CFD9FF050EE126DF6AFB0EDBCF02F038
:1098A000FC0EDBCF03F0070ED89002360336E80635
:1098B000FBE1F90EDB500224006EFA0EDB500320B0
:1098C000016E030E00C0DBFF040E01C0DBFFFF0EC4
:1098D000E76E030EDBCF00F0040EDBCF01F0E750A4
:1098E0000016016A020E00C0DBFF030EDBCF00F0A2
:1098F000040EDBCF01F001C000F0016A010E00C0D0
:10990000DBFFC750040B01E0010E006E1F0EC514F3
:10991000001001E0F6D7C580C5B0FED7C5B0FED7B0
:10992000AE0EE66E45EC5EF0E552C750040B01E06A
:10993000010E006E1F0EC514001001E0F6D7010ED7
:10994000DBCFE6FF45EC5EF0E552C750040B01E0CB
:10995000010E006E1F0EC514001001E0F6D7020EB6
:10996000DBCFE6FF45EC5EF0E552C750040B01E0AB
:10997000010E006E1F0EC514001001E0F6D7DF6A5D
:10998000DFCF00F0F70EDBCF01F0F80EDBCF02F0F7
:109990000150005C000E025421E2DF50E76EFD0E24
:1099A000DBCFE9FFFE0EDBCFEAFFE750E926000E32
:1099B000EA22EF50E66E45EC5EF0E552C750040B2C
:1099C00001E0010E006E1F0EC514001001E0F6D775
:1099D000C5AC02D0FE0E18D0DF2AD2D7C750040B78
:1099E00001E0010E006E1F0EC514001001E0F6D755
:1099F000C584C5B4FED7C5B4FED7060EE66E7AECB4
:109A00005FF0E552000E00D0006E050EE15C02E250
:109A1000E16AE552E16E0050E552E7CFD9FF12004E
:109A2000D9CFE6FFE1CFD9FF050EE126DF6A800E30
:109A3000206E216AFC0EDBCF25F0FD0EDBCF26F079
:109A40008EEC5BF0030E1EC0DBFF040E1FC0DBFFBD
:109A5000FF0EE76E030EDBCF00F0040EDBCF01F04C
:109A6000E7500016016A020E00C0DBFF030EDBCFD9
:109A700000F0040EDBCF01F001C000F0016A010E1E
:109A800000C0DBFFC750040B01E0010E006E1F0E8B
:109A9000C514001001E0F6D7C580C5B0FED7C5B02B
:109AA000FED7AE0EE66E45EC5EF0E552C750040BF5
:109AB00001E0010E006E1F0EC514001001E0F6D784
:109AC000010EDBCFE6FF45EC5EF0E552C750040B1C
:109AD00001E0010E006E1F0EC514001001E0F6D764
:109AE000020EDBCFE6FF45EC5EF0E552C750040BFB
:109AF00001E0010E006E1F0EC514001001E0F6D744
:109B0000DF6ADF50006E016AD890015004E6800ED3
:109B1000005C000E015816E2FE0EDBCFE6FF45ECBE
:109B20005EF0E552C750040B01E0010E006E1F0EFF
:109B3000C514001001E0F6D7C5AC02D0FE0E18D057
:109B4000DF2ADFD7C750040B01E0010E006E1F0EA5
:109B5000C514001001E0F6D7C584C5B4FED7C5B45E
:109B6000FED7060EE66E7AEC5FF0E552000E00D0EE
:109B7000006E050EE15C02E2E16AE552E16E005022
:109B8000E552E7CFD9FF1200D9CFE6FFE1CFD9FFE9
:109B9000060EE126DE6ADD6A800E206E216AFB0E6B
:109BA000DBCF25F0FC0EDBCF26F08EEC5BF0040E55
:109BB0001EC0DBFF050E1FC0DBFFFF0EE76E040EAD
:109BC000DBCF00F0050EDBCF01F0E7500016016A95
:109BD000030E00C0DBFF040EDBCF00F0050EDBCF71
:109BE00001F001C000F0016A020E00C0DBFF060EAA
:109BF000E66EEEEC5FF0E552C750040B01E0010E9B
:109C0000006E1F0EC514001001E0F6D7C580C5B068
:109C1000FED7C5B0FED7AE0EE66E45EC5EF0E5525F
:109C2000C750040B01E0010E006E1F0EC51400109A
:109C300001E0F6D7020EDBCFE6FF45EC5EF0E55221
:109C4000C750040B01E0010E006E1F0EC51400107A
:109C500001E0F6D7030EDBCFE6FF45EC5EF0E55200
:109C6000C750040B01E0010E006E1F0EC51400105A
:109C700001E0F6D7C582C5B2FED7C5B2FED7AF0E9A
:109C8000E66E45EC5EF0E552C750040B01E0010EB4
:109C9000006E1F0EC514001001E0F6D7800EE66EB0
:109CA000FD0EDBCFE6FFFE0EDBCFE6FF85EC5EF0C0
:109CB000E552E552E552C58AC588C5B8FED7C5B894
:109CC000FED7C584C5B4FED7C5B4FED7000E006E5E
:109CD000060EE15C03E200D0E16AE552E16E00505D
:109CE000E552E7CFD9FF1200D9CFE6FFE1CFD9FF88
:109CF000020EE126FF0EE76EFC0EDBCF00F0FD0E3C
:109D0000DBCF01F0E7500016016A010E00C0DBFF57
:109D1000FC0EDBCF00F0FD0EDBCF01F001C000F048
:109D2000016A0050DF6EC750040B01E0010E006EA7
:109D30001F0EC514001001E0F6D7C580C5B0FED7D0
:109D4000C5B0FED7AE0EE66E45EC5EF0E552C750EC
:109D5000040B01E0010E006E1F0EC514001001E09F
:109D6000F6D7DFCFE6FF45EC5EF0E552C750040BB7
:109D700001E0010E006E1F0EC514001001E0F6D7C1
:109D8000010EDBCFE6FF45EC5EF0E552C750040B59
:109D900001E0010E006E1F0EC514001001E0F6D7A1
:109DA000FE0EDBCFE6FF45EC5EF0E552C750040B3C
:109DB00001E0010E006E1F0EC514001001E0F6D781
:109DC000C584C5B4FED7C5B4FED7060EE66E7AECE0
:109DD0005FF0E552000E006E020EE15C03E200D07F
:109DE000E16AE552E16E0050E552E7CFD9FF12007B
:109DF000D9CFE6FFE1CFD9FF030EE126C750040B10
:109E000001E0010E006E1F0EC514001001E0F6D730
:109E1000C580C5B0FED7C5B0FED7FE0EDB50020A26
:109E200011E0030A09E0010A01E012D0920EE66E89
:109E300045EC5EF0E5520CD0940EE66E45EC5EF01B
:109E4000E55206D0960EE66E45EC5EF0E55200D087
:109E5000C750040B01E0010E006E1F0EC514001068
:109E600001E0F6D7E66A45EC5EF0E552C750040B18
:109E700001E0010E006E1F0EC514001001E0F6D7C0
:109E8000C582C5B2FED7C5B0FED7FE0EDB50020AB2
:109E900011E0030A09E0010A01E012D0930EE66E18
:109EA00045EC5EF0E5520CD0950EE66E45EC5EF0AA
:109EB000E55206D0970EE66E45EC5EF0E55200D016
:109EC000C750040B01E0010E006E1F0EC5140010F8
:109ED00001E0F6D7E1EC5FF0DF6EC750040B01E064
:109EE000010E006E1F0EC514001001E0F6D7E1EC64
:109EF0005FF0E76E010EE7CFDBFFC58AC588C5B806
:109F0000FED7C5B8FED7C584C5B4FED7C5B4FED745
:109F1000DF50006E030EE15C03E200D0E16AE5521F
:109F2000E16E0050E552E7CFD9FF1200D9CFE6FF2E
:109F3000E1CFD9FF050EE126030EDB6A040EDB6AD2
:109F4000C750040B01E0010E006E1F0EC514001077
:109F500001E0F6D7C580C5B0FED7C5B0FED7FE0E6E
:109F6000DB50020A11E0030A09E0010A01E012D005
:109F7000920EE66E45EC5EF0E5520CD0940EE66E65
:109F800045EC5EF0E55206D0960EE66E45EC5EF0CE
:109F9000E55200D0C750040B01E0010E006E1F0E09
:109FA000C514001001E0F6D7E66A45EC5EF0E55214
:109FB000C750040B01E0010E006E1F0EC514001007
:109FC00001E0F6D7C582C5B2FED7C5B0FED7FE0EFA
:109FD000DB50020A11E0030A09E0010A01E012D095
:109FE000930EE66E45EC5EF0E5520CD0950EE66EF3
:109FF00045EC5EF0E55206D0970EE66E45EC5EF05D
:10A00000E55200D0C750040B01E0010E006E1F0E98
:10A01000C514001001E0F6D7E1EC5FF0DF6EC75029
:10A02000040B01E0010E006E1F0EC514001001E0CC
:10A03000F6D7E1EC5FF0E76E010EE7CFDBFFC58AF4
:10A04000C588C5B8FED7C5B8FED7C584C5B4FED788
:10A05000C5B4FED7DFCF00F0016A00BE0168030E71
:10A0600000C0DBFF040E01C0DBFF030EDBCF00F0FE
:10A07000040EDBCF01F000C001F0006AD950030FDD
:10A08000E96EDACFEAFFEE50ED1005E1010EDB508C
:10A0900002E1000E01D0010E030EDBCF00F0040E32
:10A0A000DBCF01F000C0F3FF01C0F4FF050EE15C5F
:10A0B00003E200D0E16AE552E16EE552E7CFD9FF55
:10A0C0001200D9CFE6FFE1CFD9FFC750040B01E062
:10A0D000010E006E1F0EC514001001E0F6D7C580FA
:10A0E000C5B0FED7C5B0FED7FE0EDB50020A11E0A8
:10A0F000030A09E0010A01E012D0920EE66E45EC77
:10A100005EF0E5520CD0940EE66E45EC5EF0E55242
:10A1100006D0960EE66E45EC5EF0E55200D0C750D4
:10A12000040B01E0010E006E1F0EC514001001E0CB
:10A13000F6D7010EE66E45EC5EF0E552C750040B13
:10A1400001E0010E006E1F0EC514001001E0F6D7ED
:10A15000FD0EDBCFE6FF45EC5EF0E552E552E7CFC2
:10A16000D9FF1200D9CFE6FFE1CFD9FF030EE126D8
:10A17000C750040B01E0010E006E1F0EC514001045
:10A1800001E0F6D7C580C5B0FED7C5B0FED7FE0E3C
:10A19000DB50020A11E0030A09E0010A01E012D0D3
:10A1A000920EE66E45EC5EF0E5520CD0940EE66E33
:10A1B00045EC5EF0E55206D0960EE66E45EC5EF09C
:10A1C000E55200D0C750040B01E0010E006E1F0ED7
:10A1D000C514001001E0F6D7010EE66E45EC5EF006
:10A1E000E552C750040B01E0010E006E1F0EC514AE
:10A1F000001001E0F6D7C582C5B2FED7C5B0FED7C4
:10A20000FE0EDB50020A11E0030A09E0010A01E038
:10A2100012D0930EE66E45EC5EF0E5520CD0950E32
:10A22000E66E45EC5EF0E55206D0970EE66E45EC24
:10A230005EF0E55200D0C750040B01E0010E006E45
:10A240001F0EC514001001E0F6D7E1EC5FF0DF6EE1
:10A25000C58AC588C5B8FED7C5B8FED7C584C5B4FC
:10A26000FED7C5B4FED7DF50006E030EE15C03E2FB
:10A2700000D0E16AE552E16E0050E552E7CFD9FF28
:10A280001200D9CFE6FFE1CFD9FFE652AA0EDF6E6A
:10A29000C750040B01E0010E006E1F0EC514001024
:10A2A00001E0F6D7C580C5B0FED7C5B0FED79A0E7F
:10A2B000E66E45EC5EF0E552C750040B01E0010E7E
:10A2C000006E1F0EC514001001E0F6D7E66A45ECDB
:10A2D0005EF0E552C750040B01E0010E006E1F0E48
:10A2E000C514001001E0F6D7C582C5B2FED7C5B2CD
:10A2F000FED79B0EE66E45EC5EF0E552C750040BB0
:10A3000001E0010E006E1F0EC514001001E0F6D72B
:10A31000E1EC5FF0DF6EC58AC588C5B8FED7C5B869
:10A32000FED7C584C5B4FED7C5B4FED7DF5000D074
:0AA33000E552E552E7CFD9FF120015
:06A33A00576174657262B8
:10A3400061746820696E697420636F6D706C6574E8
:10A35000652E2052434F4E3A253032782053544BCD
:10A360005054523A253032780A0D00544642530078
:10A3700076312E31302E306100253564202536644B
:10A380002025346420253564202536642025346456
:10A39000202535642025366420253464202025338B
:10A3A00064202020253364202020253364202025AC
:10A3B0003268686420202025686864200A0D002522
:10A3C000326420202532642025336420202020257B
:10A3D0003264202025326420253364202020202070
:10A3E0002532642020253264202533642000253066
:10A3F00032643A253032643A2530326420200048F5
:10A40000616E646C65496D73436F6D6D616E642040
:10A4100072657475726E6564206572726F72282D34
:10A42000312900556E6B6E6F776E20636F6D6D61B5
:10A430006E6400204572726F72004572726F720016
:10A440005F690020005742200025303264253032F9
:10A450006425303264253032642530326425303250
:10A46000642530326400683A25642C25642C256408
:10A47000206C3A256420703A256420733A25642CB8
:10A4800025642C256420633A25642C25642C2564DE
:10A4900020643A25642C25642C256420693A2564BF
:10A4A00020613A2564004E4F5F53455249414C5F4D
:10A4B0004E554D4245520068683A6D6D3A737320AF
:10A4C0005365742052656164204572722020536583
:10A4D0007420526561642045727220202053657497
:10A4E0002052656164204572722020202050202077
:10A4F00020202049202020202044202020202050DF
:10A5000020202020204920202020204420202020FE
:10A5100020502020202020492020202020442020BE
:10A5200044757479202044757479202044757479B9
:10A53000204552522320466C670A0D00202020201F
:10A54000202020202020202020426174682020200C
:10A550002020202020204F7269656E74202020204A
:10A56000202020202044727920202020202020201C
:10A5700020202020202042617468202020202020DC
:10A58000202020202020204F7269656E742020201A
:10A590002020202020202020202044727965722055
:10A5A00020202020204261746820204F72696E7440
:10A5B000204472792020202020202053796E630AC5
:10A5C0000D000A0D00616D200A0D00706D200A0D4E
:10A5D00000253032642000253032642E002532649C
:10A5E0003A0053617475726461792000467269643F
:10A5F0006179200054687572736461792000576531
:10A60000646E657364617920005475657364617963
:10A6100020004D6F6E646179200053756E6461791E
:10A6200020003230253032642020002532642C2076
:10A6300000446563656D62657220004E6F76656DDE
:10A6400062657220004F63746F626572200053650B
:10A650007074656D62657220004175677573742052
:10A66000004A756C7920004A756E6520004D61794D
:10A670002000417072696C20004D61726368200097
:10A68000466562727561727920004A616E75617209
:10A690007920000A0D0A0D000A0D48656174204FEB
:10A6A00066662E2E2E0A0D000A0D48656174204F35
:07A6B0006E2E2E2E0A0D0094
:08A6B800D9CFE6FFE1CFD9FF85
:10A6C000020EE126DE6ADD6ADECF00F0DDCF01F0AA
:10A6D000FD0EDBCF02F0FE0EDBCF03F00250005C7C
:10A6E0000350015814E2B40EE66E7AEC5FF0E552C6
:10A6F000B40EE66E7AEC5FF0E552B40EE66E7AECDC
:10A700005FF0E552DF2A010E01E3DB2ADDD7020EFE
:10A71000E15C02E2E16AE552E16EE552E7CFD9FF82
:10A720001200D9CFE6FFE1CFD9FF020EE126896AF8
:10A73000C0881F0EC16EC098926880A005D000002E
:10A74000F29E0EEF00F00000E7D8580EDE6E020E0B
:10A75000DD6E9B8CDFCF00F0DF06010EDBCF01F05A
:10A7600001E2DB060050011001E0F4D78D6890682B
:10A770008882010EE66EE66A9FDFE552E552889216
:10A780008884010EE66EE66A97DFE552E55288940A
:10A790008886010EE66EE66A8FDFE552E5528896FE
:10A7A0008888010EE66EE66A87DFE552E5528898F2
:10A7B000888A010EE66EE66A7FDFE552E552889AE6
:10A7C000888C010EE66EE66A77DFE552E552889CDA
:10A7D0008D6A906A16EC3EF01AEC3EF0AED8E66A4E
:10A7E000E66A61EC50F0E552E5526DEC40F0E66A45
:10A7F000F8EC4EF0E55201010A6F0B6B800B01E0A3
:10A800000B69A4D838EC44F049EC3BF027EC22F07B
:10A81000060EE66E010EE66E040EE66E010EE66EA4
:10A82000020EE66E010EE66E91EC27F0006E060E4B
:10A83000E15E005002C108F103C109F104C12EF12B
:10A8400005C12FF106C154F107C155F100002EECEE
:10A8500029F00000A9EC2FF085EC28F0F3CF28FFB9
:10A86000F4CF29FFFAEC28F00201A86FE66AE66A45
:10A8700001C1E6FF00C1E6FF0A0EE66EC0EC46F03D
:10A88000006E050EE15E00506BEC5AF0010EC06EDA
:10A8900004013C0EFB6FFBC4FCF4F9EC38F0050E30
:10A8A000E66EE66A09DFE552E55204013D0EFB6FF4
:10A8B000FBC4FCF4F9EC38F0050EE66EE66AFCDE4B
:10A8C000E552E5520401320EFC6F0401FB6B010EF0
:10A8D000E66EE66AF1DEE552E5524AEC3CF0480EDF
:10A8E000E66E7AEC5FF0E5524AEC3CF0010EE66E63
:10A8F000E66AE2DEE552E55218EC3EF01CEC3EF072
:10A9000026EC56F0020EE15C02E2E16AE552E16EED
:10A91000E552E7CFD9FF1200816A936A826A949068
:10A9200094829494949A956A8D6A966A97689868C6
:10A93000876A996A886A9A6A1200280EC66E1D0E86
:10A94000C86EC78E94869488C56A1200190EE66E8A
:10A95000E66A3C0EE66EC1EC5DF0E552E552E5526A
:10A9600001010151E66EE66A01010051E66EE66AF8
:10A970003A0EE66EA30EE66E000EE66E75EC5DF026
:0AA98000006E070EE15E00501200A9
:06A98A00D9CFE6FFE1CF8A
:10A99000D9FFE6520201D13504E2D0510108000E80
:10A9A000D15504E2D007000ED15B11D0010ED019B1
:10A9B00001E1D15107E14AEC3CF00201D007000E61
:10A9C000D15B05D00401FB6B0201D06BD16B80A081
:10A9D00040D03E0E8014E8407F0BDF6E0101FD5138
:10A9E00002E034EC58F00201CE51DF5C21E1DF508F
:10A9F00009E0040EDF5C06E00D0EDF5C03E0110EE3
:10AA0000DF5C15E1CC51CD110EE1050ECF5D05E205
:10AA1000410ECC6FCD6BCF2B03D0190ECC6FCD6B0D
:10AA20004AEC3CF00DD0CC07000ECD5B0AD109D129
:10AA3000DFCFCEF2410ECC6FCD6BCF6B4AEC3CF04A
:10AA40000401FB51020A6FE0030A35E0010A05E048
:10AA5000A2D0DF68CE69CF6BF4D0DF5013E10101E3
:10AA6000082B000E0923093504E208513C08000EAA
:10AA7000095503E23C0E086F096B0201A16BA26B42
:10AA800001EC2FF0040EDF5C15E101010807000E58
:10AA9000095B190E09AF02D0D89003D0085D000EF3
:10AAA000095903E2190E086F096B0201A16BA26B31
:10AAB00001EC2FF070D0DF5018E101012E2B000EB9
:10AAC0002F232F3504E22E514108000E2F5503E2AB
:10AAD000410E2E6F2F6B0201A36BA46B0201400E7F
:10AAE000D06F060ED16F01EC2FF0040EDF5C1AE17F
:10AAF00001012E07000E2F5B190E2FAF02D0D89048
:10AB000003D02E5D000E2F5903E2190E2E6F2F6B0E
:10AB10000201A36BA46B0201400ED06F060ED16F31
:10AB200001EC2FF038D0DF5018E10101542B000E5A
:10AB30005523553504E254514108000E555503E2A2
:10AB4000410E546F556B0201A56BA66B0201400EBE
:10AB5000D06F060ED16F01EC2FF0040EDF5C1AE10E
:10AB600001015407000E555B190E55AF02D0D89065
:10AB700003D0545D000E555903E2190E546F556B06
:10AB80000201A56BA66B0201400ED06F060ED16FBD
:10AB900001EC2FF000D00C0EDF5C0BE10201400E47
:10ABA000D06F060ED16F0401010EFB6F0401330E4E
:10ABB000FC6FDF040BE10201400ED06F060ED16F77
:10ABC0000401020EFB6F0401330EFC6F100EDF5CFC
:10ABD00007E182A003D018EC3EF002D016EC3EF064
:10ABE000050EDF5C09E1320E0401FC5D02E13AEC86
:10ABF0003CF00401320EFC6F090EDF5C09E1330EFC
:10AC00000401FC5D02E142EC3CF00401330EFC6FF8
:10AC1000080EDF5C0CE102019E5105E10401FB6BB3
:10AC2000C8EC3DF004D00401FB6BFAEC3DF00D0ED6
:10AC3000DF5C02E129EC44F0110EDF5C02E11AEC6A
:0CAC400044F0E552E552E7CFD9FF1200C6
:04AC4C000001FB6B9D
:10AC5000FC6BFD6BFE6B1BEC19F00FEF22F0D9CFF4
:10AC6000E6FFE1CFD9FF040EE126200E0F01E76ECB
:10AC70000019E8AE02D0E73402D0E750005D03E3EC
:10AC80006550020B01E07ED00001FB51FC1102E196
:10AC9000000E08D0FBC0E9FFFCC0EAFFEF50800BBC
:10ACA00001E0010E00096EE1A00EE66E000EE66EF8
:10ACB000600EE66E000EE66E58EC08F0E552E552C6
:10ACC000E552E552020EF3CFDBFF030EF4CFDBFFBC
:10ACD000020EDBCF00F0030EDBCF01F00001800E8F
:10ACE000011410E0FF0EE66EA30EE66E000EE66E97
:10ACF000A00EE66E000EE66E1FEC5AF0006E050E1A
:10AD0000E15E0050D950020FE96EDACFEAFFEE5053
:10AD1000ED1002E10001A06B0001FD51FE1102E106
:10AD2000000E08D0FDC0E9FFFEC0EAFFEF50800B27
:10AD300001E0010E000913E1400EE66EA00EE66E82
:10AD4000000EE66E010EE66EE66E2DEC21F0006E52
:10AD5000050EE15E0050F3CFFDF0F4CFFEF0400EA3
:10AD6000E66E600EE66E000EE66EE66A010EE66EB8
:10AD70002DEC21F0006E050EE15E0050F3CFFBF0EC
:10AD8000F4CFFCF0040EE15C02E2E16AE552E16E10
:10AD9000E552E7CFD9FF1200120012001200120094
:10ADA000F5EF5BF012001E0EE66E010EE66E87EC0C
:10ADB00020F0E552E552400EE66E600EE66E000EA3
:10ADC000E66EE66A010EE66E2DEC21F0006E050ED1
:10ADD000E15E0050F3CFFBF0F4CFFCF0120065848D
:10ADE0000001080EE06F070EE16FE007000EE15B67
:10ADF000E051E111FAE165941200D9CFE6FFE1CF0D
:10AE0000D9FFFD0EDBCF20F0FE0EDBCF21F0720E5E
:10AE1000201801E1215033E0E868201802E17F0E9C
:10AE200021182BE0740E201801E1215024E0750E4A
:10AE3000201801E121501DE0730E201801E121507E
:10AE400016E0030E201801E121500FE0020E201839
:10AE500001E1215008E0010E201801E1215001E03C
:10AE600010D0A1DF0FD09EDF0DD09ADF0BD096DF80
:10AE700009D092DF07D091DF05D091DF03D0000029
:10AE800001D000D0010E00D0E552E7CFD9FF12006B
:10AE9000D9CFE6FFE1CFD9FFE66A45EC3DF0E552B8
:10AEA000010EE66E45EC3DF0E552020EE66E45EC15
:10AEB0003DF0E552FE0EDB500101FD5D01E1CAD01F
:10AEC000FE0EDB50430A01E1B5D0020A01E1A2D037
:10AED000780A01E18FD0010A01E17DD00F0A6BE011
:10AEE000010A59E0030A47E0010A35E0070A23E0B6
:10AEF000010A12E0030A01E0ADD0FE0EDBCFE6FF4F
:10AF0000E66AE66AE66A020EE66EC0EC46F0006E9D
:10AF1000050EE15E00509ED0FE0EDBCFE6FFE66A36
:10AF2000E66A010EE66EE66E1DEC46F0006E050E5A
:10AF3000E15E00508FD0FE0EDBCFE6FFE66AE66AE8
:10AF4000020EE66E010EE66E1DEC46F0006E050E7A
:10AF5000E15E00507FD0FE0EDBCFE6FFE66AE66AD8
:10AF6000030EE66E010EE66E1DEC46F0006E050E59
:10AF7000E15E00506FD0FE0EDBCFE6FFE66AE66AC8
:10AF8000010EE66E050EE66E1DEC46F0006E050E37
:10AF9000E15E00505FD0FE0EDBCFE6FFE66AE66AB8
:10AFA000020EE66E050EE66E1DEC46F0006E050E16
:10AFB000E15E00504FD0FE0EDBCFE6FFE66AE66AA8
:10AFC000030EE66E050EE66E1DEC46F0006E050EF5
:10AFD000E15E00503FD0FE0EDBCFE6FFE66AE66A98
:10AFE000E66A010EE66EC0EC46F0006E050EE15E0C
:10AFF000005030D0FE0EDBCFE6FFE66AE66A010EB7
:10B00000E66E060EE66E1DEC46F0006E050EE15E85
:10B01000005020D0FE0EDBCFE6FFE66AE66A020EA5
:10B02000E66E060EE66E1DEC46F0006E050EE15E65
:10B03000005010D0FE0EDBCFE6FFE66AE66A030E94
:10B04000E66E060EE66E1DEC46F0006E050EE15E45
:10B05000005000D0FE0EDBCFFDF10401460EFC6F68
:10B06000E552E7CFD9FF1200D9CFE6FFE1CFD9FFF4
:10B07000020EE12602019E6B02019F6B0201A06B92
:10B0800001EC2FF00201A16BA26B0201A36BA46B78
:10B090000201A56BA66BE66AE66AE66AFDC1E6FFF9
:10B0A000080EE66EC0EC46F0006E050EE15E005044
:10B0B0000101FD6B0401320EFC6F0101010EFC6FFA
:10B0C000020EE15C02E2E16AE552E16EE552E7CF91
:04B0D000D9FF120092
:0CB0D400FF0EE3CFEAFFE552FF0EE3CFD2
:10B0E000E9FFE552E66AE66AD9CFE6FFDACFE6FF86
:10B0F000FC0EE124D96EFF0EE220DA6EE66AE66A03
:10B10000E66A200EEF5C06E0090EEF5C03E0EF66F6
:10B1100003D03FD0EE50F5D72D0EEF5C03E1FF0ECC
:10B12000E32A03D02B0EEF5C01E1EE502F0EEF640B
:10B1300024D03A0EEF6021D0D890F90EE336FA0E03
:10B14000E336FD0EDECFE3FFFE0EDDCFE3FFD8904A
:10B15000F90EE336FA0EE336D890F90EE336FA0E1E
:10B16000E336FD0EE350DE26FE0EE350DD22300E08
:10B17000EE5CDE26000EDD22D9D7FF0EE3CFE8FF1E
:10B18000E85207E0F90EE31EE32AFA0ED8B4E3060C
:10B19000E31EE552E552E552FF0EE3CFDAFFE5523A
:10B1A000FF0EE3CFD9FFE552E1CFE9FFE2CFEAFF9F
:10B1B000ED52ED52EECFF3FFEFCFF4FF1200D9CFF7
:10B1C000E6FFDACFE6FFFA0EE3CFD9FFFB0EE3CFBF
:10B1D000DAFFFD0EE35209E72D0EDE6EFC0EE31ED4
:10B1E000E32AFD0ED8B4E306E31EE652E652E65229
:10B1F000FD0EE124E76EFF0EE220E46EE652F70E4C
:10B20000E3CFE6FFF70EE3CFE6FF4FEC59F0F90E80
:10B21000E124E96EFF0EE220EA6E3FEC59F00AE10C
:10B220003CEC59F009E13FEC59F008E13CEC59F0F5
:10B2300007E108D04AEC59F045EC59F04AEC59F0D6
:10B2400045EC59F04AEC59F0DE6AF90EE126FF0EA2
:10B25000E222FF0EE3CFDAFFE552FF0EE3CFD9FF84
:10B26000E552FC0EE124E96EFF0EE220EA6EEECF1D
:10B27000F3FFEFCFF4FF1200EF380F0B1200EF5087
:10B280000F0B02E1EE52D8841200EF380F0B300F93
:10B29000DE6E1200EE500F0B300FDE6E1200FC0E51
:10B2A000E3CFE9FFFD0EE3CFEAFF100EE66EEE6A94
:10B2B000EE6AEF6AD890FD0EE336FE0EE336ED3609
:10B2C000ED36EF36FF0EE30609E070EC59F0EE5272
:10B2D00070EC59F0EE5270EC59F0EDD7E56E1200BB
:10B2E000030EEF24E8B6EF6E300EEF24E8BEEF6EEB
:02B2F000000C50
:0EB2F200D9CFE6FFDACFE6FFFA0EE3CFD9FFA1
:10B30000FB0EE3CFDAFFFC0EE3CFE9FFFD0EE3CF48
:10B31000EAFFE9CFF3FFEACFF4FFF80EE35003E1D1
:10B32000F90EE35008E0F80EE30602E2F90EE30638
:10B33000DECFEEFFF2D7FF0EE3CFDAFFE552FF0ECE
:10B34000E3CFD9FFE5521200FE0EE3CFE9FFFF0E77
:10B35000E3CFEAFFE9CFF3FFEACFF4FFFB0EE350C0
:10B3600003E1FC0EE35009E0FB0EE30602E2FC0EF3
:10B37000E306FD0EE350EE6EF1D71200D9CFE6FFE3
:10B38000DACFE6FFFA0EE3CFD9FFFB0EE3CFDAFF09
:10B39000FC0EE3CFE9FFFD0EE3CFEAFFE9CFF3FFB9
:10B3A000EACFF4FFEE66FED7ED52DFCFEEFFDE66AA
:10B3B000FCD7FF0EE3CFDAFFE552FF0EE3CFD9FF54
:10B3C000E5521200FB0EE3CFF6FFFC0EE3CFF7FFD2
:10B3D000FD0EE3CFF8FFFE0EE3CFE9FFFF0EE3CF54
:10B3E000EAFFE9CFF3FFEACFF4FFEE66FED7ED52B6
:10B3F0000900F5CFEFFFEE66FBD71200D9CFE6FFCD
:10B40000DACFE6FFFA0EE3CFD9FFFB0EE3CFDAFF88
:10B41000FC0EE3CFE9FFFD0EE3CFEAFFE9CFF3FF38
:10B42000EACFF4FFDECFEFFFEE66FCD7FF0EE3CFEF
:10B43000DAFFE552FF0EE3CFD9FFE5521200FB0E13
:10B44000E3CFF6FFFC0EE3CFF7FFFD0EE3CFF8FFEF
:10B45000FE0EE3CFE9FFFF0EE3CFEAFFE9CFF3FFF4
:10B46000EACFF4FF0900F5CFEFFFEE66FBD712003D
:10B47000FE0EE3CFE9FFFF0EE3CFEAFFF36AF46AC3
:10B48000EE5203E0F34AF42AFBD71200FF0EE3CF9B
:10B49000F8FFE552FF0EE3CFF7FFE552FF0EE3CFD3
:10B4A000F6FFE552E66AE66AE66A0900F55209E047
:10B4B000FD0EE32A05E1FE0EE32A02E1FF0EE32A78
:10B4C000F4D7FD0EE3CF1FF0FE0EE3CF20F0FF0E0A
:06B4D000E3CF21F01200A1
:0AB4D600F1849F0EE66E5EEC5FF05D
:10B4E000E552D08EF28E1200D8CFE4FFE0CFE4FF19
:10B4F000E46EDACFE4FFE2CFDAFFE652E552E5CFC1
:10B50000DAFFE550E5CFE0FFE5CFD8FF1000DACF56
:10B51000E4FFE2CFDAFFE9CFE4FFEACFE4FFF6CFC2
:10B52000E4FFF7CFE4FFF8CFE4FFF5CFE4FFF3CF7C
:10B53000E4FFF4CFE4FFFACFE4FFFBCFE4FF00EE3B
:10B5400018F0140EE80403E3EECFE4FFFBD700EE9F
:10B5500000F0180EE80403E3EECFE4FFFBD7E65259
:10B56000F2A45FD0C80EE66E830EE66E42EC5FF08A
:10B57000E552E5520201C951C92B2C6E2C0EE76E23
:10B580002C18E8AE02D0E73402D0E7502C5C0FE371
:10B590000201C96B0201BE51BF1103E10201010E9C
:10B5A000C06F0201BE2B000EBF230201BF6B020160
:10B5B000010EC76F85EC37F00201CA2B000ECB23BA
:10B5C0000201BC0ECA5D000ECB5929E30400020142
:10B5D000010EC86F0201CA6BCB6B0201C551C611C7
:10B5E00010E10401010EFA6F010E0201C56FC66B76
:10B5F0000201C25105E102019E0502E11AEC3EF092
:10B600000ED00401FA6B0201C507000EC65B0201F1
:10B61000C25105E102019E0502E11CEC3EF0F294EC
:10B6200002D089EC19F0E55200EE17F0180EE8048C
:10B6300003E3E5CFEDFFFBD700EE2BF0140EE8049B
:10B6400003E3E5CFEDFFFBD7E5CFFBFFE5CFFAFF47
:10B65000E5CFF4FFE5CFF3FFE5CFF5FFE5CFF8FF4A
:10B66000E5CFF7FFE5CFF6FFE5CFEAFFE5CFE9FF4E
:06B67000E5CFDAFF110036
:0AB67600186A26AE44EF5BF0256C65
:10B68000261EE86A2622181E21AE4CEF5BF0206CC5
:10B69000211EE86A2122181E91EC5FF021BE5CEFAA
:10B6A0005BF018AE000C206C211EE86A21221C6C95
:10B6B0001D1EE86A1D22000C18BE53EF5BF01988AE
:10B6C000FF0C21C02BF020C02AF020502502F4CF1F
:10B6D0001FF0F3CF1EF021502602F4CF21F0F3CF5C
:10B6E00020F02502F3501F26F4502022E86A212280
:10B6F0002A502602F3501F26F4502022E86A212205
:10B7000026AE87EF5BF02A50205E2B50215A2BAEDD
:10B71000000C2550205E2650215A000C20C02AF033
:10B7200020502502F4CF1FF0F3CF1EF02150260247
:10B73000F4CF21F0F3CF20F02502F3501F26F45070
:10B740002022E86A21222A502602F3501F26F450B4
:10B750002022E86A2122000C21C02BF020C02AF010
:10B760001FC029F01F502402F4CF1DF0F3CF1CF0AE
:10B7700020502502F4CF1FF0F3CF1EF02402F35027
:10B780001D26F4501E22E86A1F2229502502F3507C
:10B790001D26F4501E22E86A1F2221502402F35075
:10B7A0001E26F4501F2221502502206AE86A20221A
:10B7B000F3501F26F450202229502602F3501E2653
:10B7C000F4501F22216AE86A202221222A502602F0
:10B7D000F3501F26F4502022E86A21222B50260223
:0AB7E000F3502026F4502122000C43
:06B7EA00040120511F0BB9
:10B7F000010801E06CD0245101E069D0060E215D02
:10B8000029E12351230A25E0010A13E0030A01E09C
:10B8100021D00F0101050CE10F01F40E116FB80EDC
:10B82000126F000E136F090E156F166BC00E146F9A
:10B8300011D00F0101050CE10F01770E116FB90E48
:10B84000126F000E136F1D0E156F166BC00E146F66
:10B8500001D000D004012051600BE842E842E842E8
:10B86000E842E842010801E032D021510B0A29E008
:10B87000080A1CE0090A14E0080A07E00B0A04E0C1
:10B88000080A01E024D023D022D00F01FE0E116F50
:10B89000010E126F010E156F166BC10E146F17D0CB
:10B8A0000F01800E146F23C4FEF111D00F01FF0EA3
:10B8B000116F010E126F010E156F166B810E146F52
:10B8C00006D00F01800E146F22C4FFF100D01200C9
:10B8D0001201000200000008D8043BFC0200010233
:10B8E000000109022900010100C032090400000220
:10B8F00003000000092111010001221D000705813C
:10B900000340000107050103400001040309043A54
:10B910000354007200690061006E0067006C0065EE
:10B92000002000420069006F006D0065006400693E
:10B9300000630061006C0020005300630069006533
:10B94000006E006300650073002E03530069006DF4
:10B950000070006C00650020004800490044002091
:10B960000044006500760069006300650020004423
:10B970000065006D006F000600FF0901A1011901BB
:10B980002940150026FF00750895408100190129FE
:10B99000409100C0E2B8000BB9000FB90049B900EE
:10B9A000D9CFE6FFDACFE6FFE1CFD9FFE2CFDAFF6A
:10B9B000E652E652E652E652D950F90F006EFF0EFB
:10B9C000DA20016E020E00C0DBFF030E01C0DBFFB8
:10B9D000020EDBCFE6FF030EDBCFE6FFF90EDBCF77
:10B9E000E6FFFA0EDBCFE6FFFB0EDBCFE6FFD9501A
:10B9F000FC0FE66EFF0EDA20E66E8AEC31F0006E88
:10BA0000070EE15C02E2E16AE552E16E0050F3CF1D
:10BA1000DEFFF4CFDDFFFC0EDBCFE9FFFD0EDBCF59
:10BA2000EAFFEF6ADECF00F0DDCF01F000C0F3FFE8
:10BA300001C0F4FF040EE15C02E2E16AE552E16E4E
:0CBA4000E552E5CFDAFFE7CFD9FF120096
:04BA4C001E0EF66E66
:10BA5000100EF76E000EF86E02010900F550AF6F80
:10BA60000900F550B06F03E1AF6701D03DD0090088
:10BA7000F550AA6F0900F550AB6F0900F550AC6F97
:10BA800009000900F550E96E0900F550EA6E090059
:10BA900009000900F550AD6F0900F550AE6F0900BF
:10BAA0000900F6CFB1F2F7CFB2F2F8CFB3F2AAC2E3
:10BAB000F6FFABC2F7FFACC2F8FF0201AD5302E1E3
:10BAC000AE5307E00900F550EE6EAD07F8E2AE07A1
:10BAD000F9D7B1C2F6FFB2C2F7FFB3C2F8FF020155
:0ABAE000AF07000EB05BBFD71200E5
:06BAEA00D9CFE6FFDACF20
:10BAF000E6FFE1CFD9FFE2CFDAFFE652E652E652A7
:10BB0000E652D950FB0F006EFF0EDA20016E00C026
:10BB1000DEFFDD6EDECFE6FFDDCFE6FFFB0EDBCF27
:10BB2000E6FFFC0EDBCFE6FFFD0EDBCFE6FF3BCFF3
:10BB3000E6FF3CCFE6FF8AEC31F0006E070EE15CD9
:10BB400002E2E16AE552E16E0050020EF3CFDBFF44
:10BB5000030EF4CFDBFF020EDBCF00F0030EDBCFD2
:10BB600001F000C0F3FF01C0F4FF040EE15C02E24B
:10BB7000E16AE552E16EE552E5CFDAFFE7CFD9FFA2
:02BB80001200B1
:0EBB8200D9CFE6FFDACFE6FFE1CFD9FFE2CF61
:10BB9000DAFFAD6AAC6AFD0EDBB0AD88DBA202D085
:10BBA000AD8CAC8CDBB4AD8EDBA602D0AC8801D002
:10BBB000AC8ADBB8AD84DBBAAC86DBAC02D09D8A44
:10BBC00001D09D9ADBAE02D09D8801D09D98FB0EDE
:10BBD000DB50B06EFC0EDBCF01F001C000F0016A5B
:10BBE00000507F6EAD8AAC8E949C948EAD50100B3D
:10BBF00004E0AD50800B01E1948CE552E5CFDAFF13
:06BC0000E7CFD9FF12009E
:0ABC0600D9CFE6FFDACFE6FFE1CF69
:10BC1000D9FFE2CFDAFFFB0EDBCF00F0FC0EDBCF6B
:10BC200001F00001800E01141AE1FB0EDBCFE9FFE9
:10BC3000FC0EDBCFEAFFEECFF3FFEDCFF4FFEE2AF1
:10BC4000000EEF22F3CFE9FFF4CFEAFFFD0EDBCFCA
:10BC5000EFFFEF50016AF36E01C0F4FF10D0FB0E4E
:10BC6000DB50FE0806E1FD0EDBCFE6FFC5EC5FF022
:10BC700005D0FD0EDBCFE6FF03EC08F0E552E55200
:0ABC8000E5CFDAFFE7CFD9FF12008D
:06BC8A00D9CFE6FFDACF7E
:10BC9000E6FFE1CFD9FFE2CFDAFFFD0EDB50C96E40
:10BCA000C6AE02D0FF0E2BD00F0EC61408080FE050
:10BCB0000F0EC6140B080BE0C6889EA6FED7C75011
:10BCC000040B03E1C750010B17E0000E18D00F0E54
:10BCD000C614080804E00F0EC6140B0810E1C7B024
:10BCE000FED7C750040B01E0010E006E1F0EC514F5
:10BCF0000010F7E1C5AC02D0FE0E01D0000EE552F7
:0ABD0000E5CFDAFFE7CFD9FF12000C
:06BD0A00D9CFE6FFDACFFD
:10BD1000E6FFE1CFD9FFE2CFDAFFFB0EDBCFF3FF87
:10BD2000DB06F350000925E0E1EC5FF0E66EFC0E67
:10BD3000DBCFE9FFDB2AFD0EDBCFEAFF01E3DB2AE5
:10BD4000E552E750EF6EC5B6FED7A1A602D0FF0EB2
:10BD500011D00F0EC614080804E00F0EC6140B080D
:10BD6000DCE1FB0EDB50D9E0C59AC588C5A8D5D764
:10BD7000FDD7000EE552E5CFDAFFE7CFD9FF12007D
:10BD80001E502302F3CF1AF0F4CF1BF02402F3501D
:10BD90001B26000EF4201C6E1E502502F3501C269C
:10BDA000000EF4201D6E1E502602F3501D261F505B
:10BDB0002302F3501B26F4501C22000E1D221F509C
:10BDC0002402F3501C26F4501D221F502502F3506C
:10BDD0001D2620502302F3501C26F4501D22205013
:10BDE0002402F3501D2621502302F3501D26120079
:10BDF000FF0EE124E96EFF0EE220EA6EEDCFF4FFC4
:10BE0000EFCFF3FFF46607D0600EF36404D07B0E2F
:10BE1000F36001D0F39A1200F36AF46AFF0EE12492
:10BE2000E96EFF0EE220EA6EED6607D02F0EEF649A
:0CBE300004D03A0EEF6001D0F32A12009B
:04BE3C001D6A1C6AF5
:10BE40001B6A1A6A200EE76ED8901E361F362036FF
:10BE500021361A361B361C361D3623501A5C2450E8
:10BE60001B5825501C5826501D5809E323501A5EB4
:10BE700024501B5A25501C5A26501D5A1E2AE72EA4
:04BE8000E4D71200F1
:0CBE8400D9CFE6FFDACFE6FFE1CFD9FF0F
:10BE9000E2CFDAFFE652E652FC0EDBCFDEFFDBCF6D
:10BEA000DDFF010EDB50D76EDF50D66EE552E55256
:0CBEB000E552E5CFDAFFE7CFD9FF120022
:04BEBC00D9CFE6FFF5
:10BEC000DACFE6FFE1CFD9FFE2CFDAFFFD0EDB509C
:10BED0007F0BD56ED76AD66AF294FD0EDBAE02D028
:10BEE000F28A01D0F29AD58EE552E5CFDAFFE7CF9C
:04BEF000D9FF120064
:0CBEF400FF0EE3502E6EEF0E01D0F30E97
:10BF0000E76EE72E81EF5FF00C0E2D6EE76AE72EED
:10BF100087EF5FF02D2E86EF5FF02E2E7FEF5FF024
:02BF200012000D
:0EBF22001D6A1C6A100EE76ED890203621367C
:10BF30001C361D3625501C5C26501D5805E3255027
:0EBF40001C5E26501D5A202AE72EF0D7120054
:02BF4E00400EA3
:10BF5000F36E00EE00F00F0E01D81200EA6002D07E
:0EBF6000EE6AFCD7F350E9601200EE6AFCD7DF
:02BF6E001EEEC5
:10BF700000F02EEE00F0F86A199C26EC5DF007EC5C
:0ABF800008F001EC48F0FBD71200B6
:06BF8A00FF0EE350ADBA0A
:10BF900004D0B06AAC8EAD8A949CADA2FED7AE6ED2
:06BFA000F36EF46A1200CA
:0ABFA600FF0EE3502E6E1B0E00D0BC
:10BFB00001D0200EE76EE72EFED72E2EFAD700D046
:02BFC00012006D
:0EBFC2000F0EC614080804E00F0EC6140B087C
:0CBFD00001E1C586C7A0FED7C9501200D1
:04BFDC00FF0EE35021
:10BFE000E84E1200000000D000D000D0E82EFAD7B2
:02BFF00012003D
:0EBFF2003031323334353637383961626364AA
:03C0000065660072
:07C003000000010000001421
:06C00A0000000000000030
:0BC01000000000000000000000000025
:05C01B00000000000818
:0EC020000000000010000000002000000000E2
:02C02E004100CF
:04C03000FF004006C7
:07C034000100000000000004
:05C03B0070A3006BA3DF
:01C0400000FF
:0FC041000000000000F5A23598F14987CD59B2F3
:0AC0500025901449DA82B979379E71
:03C05A00000100E2
:03C05D00000000E0
:10C0600000000000000000000000000000000000D0
:10C0700000000000000000000000000000000000C0
:10C0800000000000000000000000000000000000B0
:10C0900000000000000000000000003132333435A1
:07C0A0003600003200000031
:020000040001F9
:01FFF800BA4E
:01FFF900F710
:01FFFA003DC9
:01FFFB00FF06
:01FFFD00F70C
:00000001FF
